:020000040800F2
:1000000000000220E9100C086D110C08AD0D070866
:100010006D110C086D110C086D110C08000000002A
:100020000000000000000000000000006D110C083E
:100030006D110C08000000006D110C08794E0508C8
:100040006D110C086D110C086D110C086D110C0868
:100050006D110C086D110C0871110508751105085A
:10006000791105087D11050881110508B5420408BC
:10007000C9420408DD420408F142040805430408AB
:10008000194304082D4304086D110C086D110C0868
:100090006D110C086D110C086D110C088511050807
:1000A0006D110C086D110C086D110C08314D040810
:1000B000454D0408594D04086D4D0408D135040818
:1000C000C535040805360408F93504086D110C0817
:1000D0006D110C0805570408115704081D57040832
:1000E000891105086D110C0800000000A94D0408D5
:1000F000F94D0408214E0408954D040841430408B5
:100100006D110C0859660408814D04086D110C0826
:10011000295704086D110C086D110C08797A040830
:1001200055430408694304087D43040891430408C7
:10013000A54304086D110C086D110C086D110C0815
:1001400000000000000000000000000000000000AF
:10015000B9430408CD430408E143040835570408B3
:10016000393604082D3604086D110C086D110C0881
:100170006D110C086D110C086D110C0800000000C9
:100180006D110C086D110C08415704084D570408F7
:100190006D110C086D110C086D110C086D110C0817
:1001A0006D110C086D110C086D110C086D110C0807
:1001B0006D110C086D110C086D110C086D110C08F7
:1001C0006D110C086D110C086D110C086D110C08E7
:1001D0006D110C08896604086D110C086D110C086E
:1001E0006D110C086D110C086D110C086D110C08C7
:1001F0006D110C086D110C086D110C086D110C08B7
:100200006D110C086D110C086D110C086D110C08A6
:10021000BD4D0408D14D0408E54D04086D110C08CE
:100220006D110C086D110C086D110C080000000018
:100230005D6604086D110C08000000006D110C08CB
:100240006D110C086D110C086D110C086D110C0866
:100250006D110C086D110C086D110C086D110C0856
:100260006D110C086D110C086D110C086D110C0846
:100270006D110C086D110C086D110C0800000000C8
:100280006D110C08000000006D110C08000000004A
:08029000000000006D110C08D4
:0802980088000C0001000000C9
:1002A00008AB0124020100000200140028AB012465
:1002B000020200000200140048AB0124020A000000
:1002C0000200140068AB01240203000004001400C3
:1002D00088AB01240208000004001400A8AB01242C
:1002E000010B000000017700C8AB0124010C0000E5
:1002F00000017600E8AB0124011000000001760047
:1003000008AC0124010D01000001770028AC012494
:10031000011200000001760048AC01240114000025
:1003200000001E0068AC0124011A000000000D004E
:1003300088AC0124011B000000002C00A8AC0124A3
:100340000115000000000C00C8AC012401160000DB
:1003500000000C00E8AC0124011C000000000E00AD
:1003600008AD0124011D000000001E0028AD01247D
:100370000117000000000C0048AD01240118000026
:1003800000000E0068AD01240119000000000C00FF
:1003900088AD0124011F000000000C00A8AD01245D
:1003A0000120000000000C00C8AD0124012901005B
:1003B00000011800E8AD01240121000000014800FF
:1003C00008AE0124012200000001490028AE0124EA
:1003D0000123000000014A0048AE0124012400006E
:1003E00000014B0068AE01240125000000014C0013
:1003F00088AE01240126000000014D00A8AE0124B2
:100400000127000000014E00C8AE012401280000B1
:1004100000014F00E8AE0124012C0000000029007B
:1004200008AF0124012D01000000290028AF01249C
:10043000012E01000000700048AF012401300000CF
:100440000000310068AF0124012F010000005200BC
:1004500088AF01240131010000012800A8AF012468
:100460000132010000012800C8AF0124013500005D
:1004700000003C00E8AF012401380000000020002B
:020000040804EE
:10000000836B5A6D12F0500F5A6D1AD1196842F471
:1000100000725A650A6812F0080FCA6816D012F406
:10002000406F15D1CA68920412D45A6D22F48072BE
:100030005A655A6DD1040BD45A6D42F001025A65CB
:100040007047D20604D4DB6CDB6C18479007ECD009
:10005000704700BF704700BF836B5A6D42F040028B
:100060005A659A6D42F004029A65704702685549D4
:1000700038B5554B554D564CAA4218BF9A420CBF45
:10008000012300238A4208BF43F001033031A2421A
:1000900008BF43F0010330348A4208BF43F0010334
:1000A0003031A24208BF43F0010330348A4208BF16
:1000B00043F0010301F55C71A24208BF43F0010364
:1000C00004F55C748A4208BF43F001033031A24258
:1000D00008BF43F0010330348A4208BF43F00103F4
:1000E0003031A24208BF43F0010330348A4208BFD6
:1000F00043F001033031A24208BF43F001038A42BA
:1001000008BF43F0010313B9324B9A4208D10423CC
:1001100080F83530136823F001031360002038BDE8
:100120002D4B2E4D1168AA4218BF9A422C4C21F03B
:100130000E0105F13C050CBF012300231160A24212
:1001400008BF43F0010311682834AA4208BF43F0F6
:10015000010321F00101A24208BF43F0010314345E
:100160001160A24208BF43F001031E498A4208BF42
:1001700043F0010313B91C4B9A4217D10123856D3B
:10018000D0E91714226801F01F0122F480728B401D
:1001900022606B60C36ED0E91921516033B11A68D7
:1001A000D0E91C1422F480721A604C6001210022F4
:1001B000036D80F8351080F83420002BAED09847BE
:1001C000ACE700BF4000024010000240280002409F
:1001D00058000240B80402401C5402580854025807
:1001E0003054025880540258945402580168002236
:1001F0000B6880F842205A0410B40ED50B6823F423
:1002000080430B6090F84130292B10D090F841309A
:100210002A2B24D05DF8044B70471B04F2D50B68E1
:1002200023F400430B6090F84130292BEED12822B3
:10023000212380F841200022036390F841300C68AC
:1002400003F02803282B14BF6FF0F2036FF0420372
:1002500023405DF8044B0B6080F840207047282253
:10026000222380F841200022036390F841300C687B
:1002700003F02803282B14BF6FF0F4036FF044033E
:1002800023405DF8044B0B6080F84020704700BFAE
:100290000023202210B4174C4363C462036380F828
:1002A000412080F842304B07026811D5526A436AF8
:1002B0001A70436A028D013343624AB1438D013A99
:1002C000013B02859BB24385436C43F004034364C6
:1002D0000368102490F84120002190F841201A680A
:1002E00022F0FE021A60DC615DF8044B80F84010D9
:1002F000704700BF0000FFFF70B5574B002590F816
:100300004120044680F84250283AC3624585436C38
:10031000022A41EA0301036841642FD890F8411092
:1003200090F84120282001F0280102F02802282915
:1003300014BFF6214621282A1A680CBFC9436FF062
:10034000F6010A4045491A6084F84100A06B226B0F
:10035000616318B1112A42D0212A40D0E06B18B154
:10036000122A51D0222A4FD094F84130602B4FF0FE
:1003700000032DD0236384F8403070BD90F84120F5
:1003800090F841201A6822F0FE021A609A699207DA
:1003900000D59D629A69D60703D49A6942F001029A
:1003A0009A6194F84120602A10D0202284F84120DC
:1003B0009A6995060AD59A69D00605D51022DA61A0
:1003C000626C42F0040262642022DA610021BDE71F
:1003D000202284F8403084F84120236370BD1A68DD
:1003E00051042CD490F83530012BBDD000221C4B89
:1003F000036584F8402090F83520022A24D080221A
:100400004265BDE8704018471A68120403D51A689F
:1004100022F400421A6090F83530012BA4D000225B
:100420000F4B036584F8402090F83520022AE6D16E
:10043000FFF71CFE0028A0D0E06B036DE1E71A680F
:1004400022F480421A60CDE7FFF710FE002894D016
:10045000A06B036DD5E700BF0000FFFFDD040408BB
:100460002D08040803689A69196810B4D40528D5C2
:100470000C0606D4416C11F00B0F1FD15DF8044B34
:100480007047416C4FF4807441F0010141645105A3
:10049000DC6120D5416C4FF48064920541F0080185
:1004A0004164DC61E6D5426C4FF4007142F0020217
:1004B0004264D961416C11F00B0FDFD05DF8044B41
:1004C0001AE7540502D50906E4D4D3E79405D1D53B
:1004D0000906E8D4CEE79205E5D4CBE7F8B590F865
:1004E00040300D46C16A012B00F008810123AE06A1
:1004F000044680F8403001D5900656D4EB0619D555
:10050000D70617D5638D9BB2002B40F0F98094F885
:100510004130B1F1007FDBB240F0D580282B40F0B4
:10052000D28029462046FFF7B3FE0023184684F800
:100530004030F8BD68071AD42F0701D516074AD4F2
:10054000A807F2D59307F0D5638D9BB2002B00F07E
:10055000FA80616A236811F8010B228D9862638D1D
:10056000013A6162013B22859BB26385DDE7530757
:10057000E2D5638D9BB26BB12268636A526A1A70CE
:10058000638D606A228D013B0130013A9BB260624B
:1005900022856385638D9BB2002BC6D111F5803F08
:1005A000C3D02046FFF722FEBFE72368202118684A
:1005B000E66A94F84120D961213A092A1ED8DFE879
:1005C00012F0C70015001D001D001D001D001D00BC
:1005D000F000C700150094F84130226803F02803AA
:1005E000282B00F0C5800823D3619EE794F84120B2
:1005F0001A6822F0FC021A60222222635A68894992
:1006000042F400425A605A680A405A609A69910757
:1006100001D500229A629A69D20703D49A6942F0FE
:1006200001029A6147047BD51A6822F480421A605D
:10063000A26B1AB111684A6892B262856A070BD53B
:100640005A6A25F00405636A1A70636A01336362AB
:10065000238D002B40F08580638D9BB21BB1636CB2
:1006600043F004036364EB061AD5C70618D5638DFF
:100670009BB2002B40F0AA8094F84130282B03D184
:10068000B6F1007F00F0C98094F8413016F5803F44
:100690002268DBB202D0292B00F0AD801023D36199
:1006A000002384F84230666C6363002E40F084803F
:1006B000E36A5D4DAB423DD194F84130202384F88C
:1006C0004130266331E794F841202368292A4FF00E
:1006D0001002DA617FF429AF11F5803F3FF425AFB6
:1006E0009A69960701D500229A629A69D5073FF563
:1006F00058AF9A6942F001029A6152E70220F8BDB0
:1007000023681022DA61636C43F00403636431F000
:1007100080737FF40AAF616C2046FFF7EDFD04E7BC
:1007200001048BD51A6822F400421A60E26B002A99
:1007300080D183E72046FFF759FD2023E56284F846
:1007400041302663F1E631F080737FF4EEAE28E7A6
:1007500094F841201A6822F0FA021A6021222263DA
:100760004CE7013B2385638D013B9BB2638573E7B7
:10077000E1689369022990699368D56836D1C3F31B
:10078000C21383EA104313F006032FD1A16C013189
:10079000A164A16C02297FF4C8AE0821A364D161D1
:1007A000C3E694F8412094F841201A6822F0FE0232
:1007B0001A600022226321E7616C2046FFF79CFD4E
:1007C00094F84130282B7FF4B0AEAAE623681022BB
:1007D000DA61636C43F00403636436F080737FF482
:1007E0005FAF616C2046FFF787FD59E7136823F080
:1007F000B803136099E61023D3619369980701D574
:10080000002393629369D90703D4936943F00103EA
:1008100093612046FFF7EAFC42E729462046FFF7AE
:1008200037FD3DE700E800FE0000FFFF836B9A6B99
:100830000AB100211165DA6B0AB10021116593F844
:100840004120602A05D000221A63002283F840204C
:1008500070470022202183F841101A63002283F898
:1008600040207047016870B4CC072DD5914A1369B8
:10087000926A03F03803102B00F0E180182B00F08F
:10088000D9804368B3F5803F00F00581002B00F06C
:100890005A81B3F5A02F874B1A6800F0678222F4C3
:1008A00080321A601A6822F480221A60824B41F268
:1008B000883C804C1D6804E01A68521B624500F2B7
:1008C0003F8122689603F7D58A0768D4CD0631D5D3
:1008D000784A1369926A03F03803082B00F0C0804D
:1008E000182B00F0B880C369724C002B00F05F81B8
:1008F0002268714B42F0800222601D6804E01A6891
:10090000521B022A00F21C812268D205F7D56B4BDC
:10091000026A1D6841F20303B3EB154FC0F0448235
:100920006368202A23F0F8430CBF43F0804343EA76
:10093000826363600D0713D543695E4C002B00F0A2
:100940001881626F5C4B42F0010262671D6804E02F
:100950001A68521B022A00F2F380626F9207F7D5E1
:100960008C0613D58369534C002B00F0118122684B
:10097000514B42F4805222601D6804E01A68521BF9
:10098000022A00F2DD8022689204F7D5490700F1BF
:100990008880436A002B40F0BC80002059E0454A23
:1009A0001369926A13F038032BD1424AC368126864
:1009B000520701D5002B4BD03E4C226822F0190281
:1009C0001A433D4B22601D6804E01A68521B022A3C
:1009D00000F2B68022685607F7D5384B02691D68C9
:1009E00041F20303B3EB154F6368C0F0028123F4B7
:1009F0007C33402A0CBF43F4003343EA0233636084
:100A000064E7182B00F0F180C3682A4C002B00F03B
:100A1000DD80226822F019021A43274B22601D68EC
:100A200004E01A68521B022A00F28A8022685207E8
:100A3000F7D5D2E702F00302022A7FF422AF1D4B62
:100A40001B689B037FF540AF4368002B7FF43CAFEE
:100A5000012070BC704702F00302012A7FF443AF0B
:100A6000144B1B68DC0502D5C369802BF0D1134CF5
:100A700041F20303026A2468B3EB144FC0F0BF8055
:100A8000202A00F09E810B4C636823F0F84343EA70
:100A9000826363604EE7074A136843F48033136050
:100AA00004E70749044B0A6842F480720A601C6834
:100AB0000CE000BF00440258002E00240010005C2F
:100AC000004802581A68121B642A39D80A68D505EA
:100AD000F8D58268012A00F06E81002A00F04E816C
:100AE000052A9F4A116F00F0748121F001011167FE
:100AF000116F21F0040111671D6841F28834984993
:100B000003E01A68521BA2421AD80A6F9207F8D55E
:100B10003FE793490A6902F03802182A00F0D580AD
:100B20000A68022B8F4B22F080720A606FD018681F
:100B30000A6892017FF531AF1A68121A022AF7D9B2
:100B4000032070BC7047864C41F28835854B226883
:100B500022F480322260226822F4802222601E6801
:100B600003E01A68921BAA42EAD822689203F8D4DA
:100B7000AAE6626F7B4B22F0010262671D6803E008
:100B80001A68521B022ADBD8626F9607F8D4E7E690
:100B90002268744B22F4805222601D6803E01A68B8
:100BA000521B022ACCD822689604F8D4EEE62268BA
:100BB0006C4B22F0800222601D6803E01A68521B11
:100BC000022ABDD82268D605F8D4B3E62268654B60
:100BD00022F0010222601D6803E01A68521B022AFB
:100BE000AED822685607F8D470E694077FF40CAFAD
:100BF000DBE623F0FE4343EA0263636066E6584C9B
:100C0000E36823F07C5343EA0263E36092E61C68E6
:100C100003E01A68121B022A92D80A689501F8D4D8
:100C20008C6A514A2240846A2243C46A42EA04120E
:100C30008A62D0E90D24013A013C5202240492B2A6
:100C400004F4FE042243046B013CC4F30804224371
:100C5000C46B013C240604F0FE4422430A63CA6AC2
:100C600022F00102CA624A6B846C6FF3CF0242EA3F
:100C7000C4024A63CA6A046C22F00C022243384C54
:100C8000CA62CA6A406C22F002020243CA62CA6A9D
:100C900042F48032CA62CA6A42F40032CA62CA6A44
:100CA00042F48022CA62CA6A42F00102CA620A6839
:100CB00042F080720A601968226890013FF56DAEBB
:100CC0001A68521A022AF7D93AE7012B8A6A0D6B81
:100CD0003FF4BEAE02F00303846AA3427FF4B8AED1
:100CE000C2F30512C36A9A427FF4B2AE036BC5F336
:100CF0000802013B9A427FF4ABAE436BC5F3462238
:100D0000013B9A427FF4A4AE836BC5F30642013BDC
:100D10009A427FF49DAEC36BC5F30665013B9D42CD
:100D20007FF496AE4B6B816CC3F3CC0399423FF4D6
:100D300034AE0B480B4BC26A22F00102C2621A6841
:100D400018688242FCD0064A536B6FF3CF0343EA24
:100D5000C1035363D36A43F00103D3621DE600BFAE
:100D600000440258002E00240CFCFFFF42F48022B5
:100D70001A601A6842F480321A6097E5194941F204
:100D800088350A6F22F001020A670A6F22F0040216
:100D90000A671C6804E01A68121BAA423FF6D0AE2C
:100DA0000A6F9607F7D4F4E5E36823F07C5343EA2F
:100DB0000263E360BEE50B490A6F42F001020A6775
:100DC0009AE6084A536823F0F84343F0804353609F
:100DD000B0E541F004011167116F41F001011167A5
:100DE0008AE600BF00440258334B30B4996A9C6ACB
:100DF000DD6A14F47C7F5A6BC4F3051036D0C2F35D
:100E0000CC0205F0010501F0030107EE900A05FB95
:100E100002F20129B8EEE77A06EE902AFAEEE96AC4
:100E200002D0022942D019B3DFED247A87EE876A17
:100E30001B6BC3F3080307EE903AF7EE005AF8EE87
:100E4000E77A77EEA67A77EEA57A67EE867A1A4B7E
:100E50001B6BC3F34623013307EE103AF8EEC76A63
:100E600087EEA67AFCEEC77A17EE900A30BC704780
:100E70001A6892061DD51968F7EE005A104A1B6BC6
:100E8000C1F3C101C3F30803CA4007EE903A06EE6E
:100E9000102AF8EEE77AB8EEC66A77EEA66AC6EED2
:100EA000077A36EEA57A67EE877AD0E7DFED057A26
:100EB000BCE7DFED057AB9E7004402580024744A24
:100EC0000090D00320BCBE4B0024744CF0B5354AD2
:100ED000B0F1804F344DA0EB02020368A0EB050E89
:100EE0004C69B2FA82F28F68BEFA8EFE0E684FEA43
:100EF00052124FEA5E1E1FD0F2B9DFF8B8C060454B
:100F000037D00CF5806C604533D00CF5806C6045B3
:100F100012D0BEF1000F0FD1244D254A904218BFC8
:100F2000A8422AD002F58062904226D023F08003A6
:100F3000C76286621C4314E04D6823F07003D1F849
:100F40000CC02B43C762866223F4407343EA0C0350
:100F500023F080031C4312B9BEF1000F16D00B69B9
:100F600003630368012243F00403036042610460E9
:100F7000F0BD23F070034A681343CA6823F440733A
:100F8000C7621343866223F080031C43074A084B61
:100F9000984218BF9042E2D003F580639842DED0B9
:100FA000DFE700BF000001400004014000400140B5
:100FB0000044014000040040836A1A0710B406D5BB
:100FC0000168846B4A6822F4004222434A60DC07CD
:100FD00006D50168C46A4A6822F4003222434A6096
:100FE000990706D50168046B4A6822F480322243CF
:100FF0004A605A0706D50168446B4A6822F4802289
:1010000022434A60DC0606D50168C46B8A6822F474
:10101000805222438A60990606D50168046C8A686A
:1010200022F4005222438A605A060AD50168446CB1
:101030004A68B4F5801F22F4801242EA04024A6032
:101040000BD01B0606D50268C16C536823F400233D
:101050000B4353605DF8044B70474A68846C22F47C
:10106000C00222434A60ECE70022836BA3F85E20B3
:10107000704700BF124B41F2883C124A01461B6880
:10108000A2FB03235B0A0CFB03F33BB14A6B12F098
:10109000450F01D0920404D5013BF7D14FF0004039
:1010A00070474B6B5B0707D4486B10F0010014BF0F
:1010B0000123054B8B637047042318468B637047ED
:1010C00000000024D34D6210C5002000036942686F
:1010D0001F2B70B430D9A3F1200520215468A940FA
:1010E000214227D08169087C022835D048681F2B0F
:1010F000C9681B4D4E680169C1F30324194951F8B1
:10110000244015F804C0056856F80C4024F001048A
:1011100046F80C40407901EB4001088CE96800F486
:10112000F05021EA0001E96010D9A3F12001202349
:101130008B40D36070BC70472021146899402142D5
:10114000F8D08169087C0228D0D105E0202101FA7D
:1011500003F370BC9360704700200874C6E700BFBB
:10116000389D0C08089C0C08D0E907239A423CBF24
:10117000C1685218D01A7047D0E9092300699A4211
:1011800038BF12180138D31AC01A7047D0E90902C3
:10119000101AB0FA80F04009704700BF016A034698
:1011A00040694A1C405CD9688A4228BF00221A6202
:1011B000704700BF436A826910B4D154436A416BDF
:1011C000046901330A68A34228BF00235DF8044B79
:1011D00042F0800243620A60704700BF436BD869E7
:1011E00010F0100002D0102201201A62704700BFD8
:1011F000704700BF704700BF704700BF01207047B5
:10120000014B5868704700BF002E0024074B93F82D
:10121000A422012A01D10020704793F8A402A0F172
:101220000300B0FA80F04009704700BF002E002490
:10123000012380F849307047EFF31182702383F364
:1012400012880849D2B2D1E9B93182F31188581E07
:101250008B42A0EB01008CBF0023012300EB033085
:10126000704700BF002E002470B5D0F8D442D0F8EB
:10127000C86200EB840EDEF8C05245B301F00F04E3
:101280000A4604EB840C00EB8C0CDCF818306BB9CC
:10129000DEF8C43200211B69C5F8141223B105F52C
:1012A0000471D5F808029847002070BD04EBC4040F
:1012B00006EB8406F469B3FBF4F604FB1633002B4B
:1012C000E6D11A46CCF818307DF0D0FCECE70320CC
:1012D00070BD00BFD0F8D42200EB820210B5D2F866
:1012E000C042ACB101F00F03D0F8C802D2F8C4225A
:1012F00004F5037103EBC303D26800EB8303D4F856
:101300000402D3F86832C4F80C329047002010BDB4
:10131000032010BDD0F8D43200EB830010B5D0F814
:10132000C04284B1D0F8C4325BB194F80002FF2807
:1013300007D09B68214694F801229847FF2384F840
:101340000032002010BD032010BD00BF30B52B4C73
:1013500086462379E5889D4242D9184604341946C9
:101360001A4602E0954246D921780C440A44617835
:1013700092B20529F6D1A1788229F3D19C461A466A
:101380001F4903E0AA4234D291F800C0614462448C
:1013900091F801C092B2BCF1050FF3D191F802C0EF
:1013A000BCF1010FEED1164A02E0A8421DD213781B
:1013B0001A44034492F801C098B2BCF1050FF4D16D
:1013C0009378812BF1D10CB11023A37119B10020B6
:1013D000022308714B711AB100210223117153715C
:1013E00043230748AEF8003030BD0022002CEBD17B
:1013F000ECE70021D7E70024C0E700BF000000248D
:101400000400002430B52B4C86462379E5889D42A4
:1014100042D91846043419461A4602E0954246D984
:1014200021780C440A44617892B20529F6D1A1785A
:101430008229F3D19C461A461F4903E0AA4234D2BE
:1014400091F800C06144624491F801C092B2BCF1CD
:10145000050FF3D191F802C0BCF1010FEED1164A8D
:1014600002E0A8421DD213781A44034492F801C046
:1014700098B2BCF1050FF4D19378812BF1D10CB166
:101480001023A37119B10020402348710B711AB1C8
:10149000002140235171137143230748AEF80030F7
:1014A00030BD0022002CEBD1ECE70021D7E700246F
:1014B000C0E700BF0000002404000024A2E700BF32
:1014C00003460A2201481A80704700BF48000024E2
:1014D000064B4FF0120C064AA3F11400526DA1F80E
:1014E00000C0022A18BF1846704700BF68000024D9
:1014F00000400058042301480B8070477C00002402
:101500001D48D0F80038D0F8082830B59B184FF0A7
:101510001A040C8001D1194830BD184A0024D0F8B3
:10152000040802F1100511464FEA137EB3F1204F73
:10153000CC7001F102010EF1370C38BF0EF1300C06
:101540008D424FEA031381F800C0EDD102F1080586
:101550000024010FB0F1204FD47402F1020201F116
:10156000370338BF01F1300395424FEA001013747E
:10157000EFD1024830BD00BF00E0F11F8000002421
:10158000122301480B80704754000024554B002162
:10159000554A1B685548A2FB032330B5DB0C544C5D
:1015A00083B0013BC4F8FC12C4F8F41242F20F718C
:1015B00094F82923C4F8EC02C4F8F812C4F8F03205
:1015C000002A00F08A8002254A49484884F82953B5
:1015D000FFF77CFC0123484A0621372084F8343386
:1015E00084F82A3384F82B3384F82C3384F82D3391
:1015F00084F82E3384F82F3384F8303384F8313371
:1016000084F8323384F8333384F82933D2F8E8305D
:1016100043F02003C2F8E830D2F8E83003F02003AA
:101620000193019B74F07AFF344B4FF400025A602F
:1016300094F82933012B3BD1D4F8EC22304B3148BC
:10164000B2F1804F18BF9A4284F82953D1680CBF79
:101650000123002341F00101824208BF43F001034E
:1016600000F58060D160824208BF43F0010300F5BD
:1016700080602549824208BF43F0010300F57840AD
:10168000824208BF43F001038A4208BF43F00103CE
:1016900013B91E4B9A4207D191681D4B0B40062B84
:1016A00006D0B3F5803F03D0136843F00103136005
:1016B000D4F8DC3204EB8303D3F8C83243B11548C5
:1016C0000021154AC3F80802C3F81012C3F8042217
:1016D0000020C4E9CE0003B030BD02F0FF0084F862
:1016E000280370E70000002483DE1B430014004041
:1016F000002E0024F03000240044025800E100E0F5
:10170000000001400004004000180040004001407B
:1017100007000100C84D0024C83D00242DE9F04712
:10172000046982B0C3681C4046D0814688464FF0A9
:10173000004501F1500701F13806B4FA84F325FAA7
:1017400003F21B3BD2431440C9F81020B8F1000F3C
:101750005FD0042B2ED8DFE803F052483D3203005F
:10176000D8F81030D9F82CA033B19B6823B11FFAF8
:101770008AF108F108009847D8F8283033B19B68FF
:1017800023B11FFA8AF108F120009847D8F84030B9
:1017900033B19B6823B11FFA8AF108F138009847EA
:1017A000D8F8583033B19B6823B11FFA8AF108F199
:1017B00050009847002CC0D102B0BDE8F087D8F89F
:1017C000103008F10800D9F834105B689847002CF5
:1017D000B3D1F1E7D8F8283008F12000D9F8381053
:1017E0005B689847002CA8D1E6E7D8F8403030462F
:1017F000D9F83C105B689847002C9ED1DCE7D8F8FC
:1018000058303846D9F840105B689847002C94D17E
:10181000D2E7042B07D8DFE803F01903140F0A00FE
:10182000D9F83C300193019B002C86D1C4E7D9F84C
:101830002C300193019BF7E7D9F834300193019BD9
:10184000F2E7D9F838300193019BEDE7D9F8403041
:101850000193019BE8E700BF0A49D1F840334A6889
:101860005BB1002AFCD0013A10B513F8014B4A6075
:10187000C1F8403312B1204610BDFEE775F014FAEE
:10188000204610BD002E0024F8B50E4E96F8A43266
:10189000012B00D1F8BD96F8A432032BFAD10D46E6
:1018A0001446D6F8447308E008F0F0F8D6F844334C
:1018B000241A0544DB1B322BECD8002C2146284689
:1018C000F2DCF8BD002E0024F8B590F848305D1C1D
:1018D0000344EDB280F8485083F8341090F8493052
:1018E00053B1132D07D9002380F84830104F97F8D3
:1018F000A432012B05D1F8BD80F84830002DF5D178
:10190000F8BD97F8A432032BF5D1D7F8446300F162
:1019100034042946204608F0B9F8D7F844332D1A84
:1019200004449B1B322BE6D8002DF2D1F8BD00BF3A
:10193000002E0024F8B5002390F84850A0F8483055
:1019400005B9F8BD0D4F97F8A432012BF9D097F8DF
:10195000A432032BF5D1D7F8446300F134042946AF
:10196000204608F093F8D7F844332D1A04449B1B03
:10197000322BE6D8002DF2D1F8BD00BF002E002496
:101980002DE9F041012104464FF4077087F082FEF3
:10199000054600286CD0D4F8D46204EB8606C6F85D
:1019A000C002237CC4F8BC02002B40D0402302229A
:1019B000812120467CF0CCFE0121402302222046DA
:1019C00021877CF0C5FE4FF0010808230322822105
:1019D0002046A4F878817CF0BBFE294B0027E36405
:1019E000D6F8C432C5F804721B689847D5F80402CB
:1019F000C5F81472C5F8187200283ED0227CD4F8BD
:101A0000C83222BBC3F88C224FF400749A7903F5D4
:101A10001E71C3F88402012AA3F87882C3F88842B1
:101A200023D018687DF012F80020BDE8F081204630
:101A30004FF40073022281217CF08AFE01214FF4D1
:101A400000730222204621877CF082FEBBE79A7950
:101A5000402403F51E71C3F88C72012AC3F8840276
:101A6000A3F87882C3F88842DBD1C3F89402D8E7A0
:101A7000D4F8D432B03344F823000220BDE8F0811A
:101A800001001000F8B5D0F8C85240F20112044627
:101A900095F894342A87012B3ED001260027286828
:101AA0003246314685F894647DF060F927873A46DE
:101AB00031462868A5F8786285F894647DF056F977
:101AC0004FF48173A4F8787132460221286885F8B2
:101AD0009464A5F85C307DF049F985F89474D4F8E5
:101AE000D432002504EB8303E564D3F8C0228AB125
:101AF000D3F8C4325B689847D4F8D432B03354F882
:101B0000230086F057FED4F8D432B03344F8235083
:101B1000C4F8BC520020F8BD00224FF48171028746
:101B2000A5F87832A0F87821A5F85C10D7E700BFB7
:101B3000D0F8D43200EB8303F0B5002683B0D3F89D
:101B4000C0728DF80560ADF806605FB191F800C015
:101B500004460D461CF060022FD0202A05D02046F6
:101B60007CF03AFF032003B0F0BDCA884878002A11
:101B700042D01CF0800F00F08380D3F8C432394685
:101B80009B689847EA8802234FF48071072AC4F8BB
:101B9000943228BF0722D4F8C832C4E906225A6218
:101BA0009A79998203F11401012A1F629E6200D181
:101BB0001F6318687CF04AFF22E04B780B2BCED8CD
:101BC00001A252F823F000BF051C0408011C040800
:101BD0005F1B04085F1B04085F1B04085F1B0408ED
:101BE0005F1B04085F1B04085F1B04085F1B0408DD
:101BF000451C04083B1C0408D3F8C4329B68984772
:101C00000020B0E790F89C32032BA8D10222D0F834
:101C1000C8320020C4F8942203F11401C4E906225A
:101C20000DF106049862C3E908424FF480729A826B
:101C30009A79012ABDD11C63BBE790F89C32032B33
:101C4000DED08CE790F89C32032B88D10122022150
:101C5000D0F8C832C0F8941203F11401C0E906228A
:101C60000DF10500C3E908024FF4807200209A824A
:101C70009A799862012A9CD10DF10500186398E7C2
:101C8000402A4FF0030387F8000228BF402287F85C
:101C90000122C4F89432D4F8C832C4F85821C4F8E8
:101CA0005C2103F51571C3F864229A79C3F8607258
:101CB000012AC3F86862A3F8546208BFC3F87072BF
:101CC00077E700BF08B520B9044873F031FF044836
:101CD00008BD044873F02CFF014808BDA0460D085C
:101CE00048310024C4460D08024808B573F020FFAF
:101CF000014808BDE8460D0848310024024808B5EF
:101D000073F016FF014808BDF0460D084831002465
:101D1000024808B573F00CFF014808BDFC460D08E9
:101D20004831002408B520B9044873F001FF044885
:101D300008BD044873F0FCFE014808BD0C470D08BF
:101D4000483100242C470D08024808B573F0F0FE16
:101D5000014808BD4C470D0848310024024808B529
:101D600073F0E6FE014808BD58470D0848310024CD
:101D700070B5124D124A2B68A2FB03239B09013B4D
:101D8000B3F1807F01D3012070BD4FF0E0220D49F7
:101D900000240F2853614FF0F003064681F82330EA
:101DA0004FF0070394611361EDD801464FF0FF3007
:101DB00074F0B4FB2046C5F89C6070BD00000024A0
:101DC000D34D621000ED00E03749024603688B42B4
:101DD00033D01831591AB1FA81F1490969BB334836
:101DE000834240D01830834240D01830834236D0EE
:101DF000183083423DD01830834240D0183083429F
:101E00002CD000F55670834237D029498B4233D00D
:101E100018318B4236D018318B4236D018318B4274
:101E200036D018318B4236D018318B4236D018312B
:101E30008B4236D023F0FF0013E0DBB21D491E4871
:101E4000103B10B41D4CA4FB03435DF8044B01EBA5
:101E5000131393F82810C2E9160170471621184889
:101E6000D1659065704710211348F9E71621124893
:101E7000F6E706211248F3E706211248F0E71021A1
:101E80000F48EDE710210F48EAE716210D48E7E774
:101E900000210D48E4E706210B48E1E710210A483C
:101EA000DEE716210848DBE7100002404000024050
:101EB00028040240089C0C0800000240ABAAAAAA11
:101EC000040002400004024004040240F0B50C4645
:101ED000114602688646936913F0100C72D04FF0D9
:101EE000000C102338486546D36193699E065FD481
:101EF00045B903685B1AA3423DD893699F06F8D59C
:101F00002023D3614CF0040C01209369D90552D5EC
:101F10004FF480715F054CF0010CD16104D54FF492
:101F200080614CF0080CD1619D0504D54FF400731D
:101F30004CF0020CD3619369990701D50023936299
:101F40009369DB0703D4936943F0010393615368FA
:101F500020241E4901200B4000215360DEF844304C
:101F60008EF8401043EA0C03CEF844308EF841401E
:101F70008EF84210F0BD57689EF842309669DBB289
:101F8000360408D57E0406D4202B04D0536843F4CD
:101F900080435360016893699F06A6D403685B1A67
:101FA000192BF8D993694FF0200C01259E069FD577
:101FB000002DA5D0A6E75E05B1D49C05B6D40028B7
:101FC000B9D1F0BD6046A0E7002E002400E800FE75
:101FD0002DE9F04707689A46089EBB6931EA03037A
:101FE0000CBF01230023934220D180460C461546A6
:101FF000DFF85C90324651464046FFF767FF20BB52
:10200000D9F80030A3EB060CD44507D9BB6934EAF4
:1020100003030CBF01230023AB420AD0BB6934EA9F
:1020200003030CBF01230023AB42E3D00020BDE833
:10203000F087D8F84430202288F840001343C8F8CD
:10204000443088F8412088F842000120BDE8F0873C
:10205000002E00240C4A136903F03803102B0DD016
:10206000182B09D063B913689B060BD51368074872
:10207000C3F3C103D8407047FEF7B6BE04487047AB
:102080000448704701487047004402580090D0034C
:1020900040787D0100093D00184A136903F03803B8
:1020A000102B10B524D0182B09D01BBB13689B062E
:1020B00022D513681248C3F3C103D84001E0FEF7EC
:1020C00093FE0E490F4A8B698969C3F303230E4CB3
:1020D00001F00F0113440A4493F8301092F83030A5
:1020E00001F01F0203F01F03D0402060D84010BD54
:1020F0000648E6E70648E4E70148E2E700440258FC
:102100000090D003089C0C080000002440787D015A
:1021100000093D00474A70B4946A956AD66A15F47E
:102120007C3FC5F30533D16B5BD0C1F3CC01C6F363
:10213000001604F0030407EE903A06FB01F1012CAF
:10214000B8EEE77A06EE901AFAEEE96A03D0022CAE
:102150006AD0002C4AD0DFED387A87EE876A936B1D
:10216000C3F3080307EE903AF7EE005AF8EEE77A69
:1021700077EEA67A77EEA57A67EE867A2D4AB7EEE5
:10218000006A936BC3F3462307EE103AB8EEC77AA2
:1021900070BC37EE067AC7EE876AFCEEE66AC0EDE1
:1021A000006A936BC3F3064307EE103AB8EEC77AA2
:1021B00037EE067AC7EE876AFCEEE66AC0ED016A82
:1021C000936BC3F3066306EE903AF8EEE66A76EE9A
:1021D000866A87EEA67AFCEEC77A17EE903A83609D
:1021E000704770BCC0E900338360704713689B067A
:1021F0001DD51468F7EE005A936B1049C4F3C10261
:10220000C3F30803D14007EE903A06EE101AF8EE39
:10221000E77AB8EEC66A77EEA66AC6EE077A36EEB9
:10222000A57A67EE877AA9E7DFED057A95E7DFED16
:10223000057A92E7004402580024744A0090D003C3
:1022400020BCBE4B0024744C474A70B4946A956A13
:10225000D66A15F07C7FC5F30553516C5BD0C1F392
:10226000CC01C6F3002604F0030407EE903A06FB07
:1022700001F1012CB8EEE77A06EE901AFAEEE96A5F
:1022800003D0022C6AD0002C4AD0DFED387A87EEDA
:10229000876A136CC3F3080307EE903AF7EE005A0F
:1022A000F8EEE77A77EEA67A77EEA57A67EE867A89
:1022B0002D4AB7EE006A136CC3F3462307EE103ABB
:1022C000B8EEC77A70BC37EE067AC7EE876AFCEEC6
:1022D000E66AC0ED006A136CC3F3064307EE103ADA
:1022E000B8EEC77A37EE067AC7EE876AFCEEE66A82
:1022F000C0ED016A136CC3F3066306EE903AF8EE84
:10230000E66A76EE866A87EEA67AFCEEC77A17EE64
:10231000903A8360704770BCC0E9003383607047B7
:1023200013689B061DD51468F7EE005A136C10490C
:10233000C4F3C102C3F30803D14007EE903A06EE9E
:10234000101AF8EEE77AB8EEC66A77EEA66AC6EE1D
:10235000077A36EEA57A67EE877AA9E7DFED057A88
:1023600095E7DFED057A92E7004402580024744AAD
:102370000090D00320BCBE4B0024744C02698368DB
:1023800070B5044605681343C069626986B0296860
:102390001343AC4A03430A40616A1343E2682B606B
:1023A0006B6823F440531343A2696B60A64B9D42B4
:1023B00000F06681236AAE681A43A44B33401A4387
:1023C000AA60EB6A23F00F030B43EB62A04B9D4224
:1023D00028D0A04B9D421AD09F4B9D4217D09F4BB7
:1023E0009D4214D09E4B9D4211D09E4B9D4219D0D0
:1023F0009D4B9D420BD09D4B9D4208D00120002358
:102400004FF001126367A266A36706B070BD984BD8
:102410005B6D03F00703052BF0D8DFE803F09F7F27
:102420008A925F79924B5B6D03F03803282BE5D8D5
:1024300001A252F823F000BFE5250408FD2304089B
:10244000FD230408FD230408FD230408FD230408DC
:10245000FD230408FD2304081D250408FD230408AA
:10246000FD230408FD230408FD230408FD230408BC
:10247000FD230408FD23040833250408FD23040874
:10248000FD230408FD230408FD230408FD2304089C
:10249000FD230408FD23040843250408FD23040844
:1024A000FD230408FD230408FD230408FD2304087C
:1024B000FD230408FD230408DD240408FD2304088B
:1024C000FD230408FD230408FD230408FD2304085C
:1024D000FD230408FD23040811250408B0F5004F6E
:1024E000644853D0644B626803EB4103B3F8403057
:1024F000B0FBF3F000EB52004FF6EF73B0FBF2F0DD
:10250000A0F110029A423FF679AFE860002076E72A
:10251000B0F5004F3AD04FF40040E3E7B0F5004F7C
:102520002DD003A8FFF7F6FD04980028EED0616ACD
:10253000D8E7B0F5004F71D06846FFF785FE0198E7
:10254000F3E7B0F5004F5ED0494B1A68920639D5D3
:102550001B684A48C3F3C103D840C3E7B0F5004F36
:1025600032D0FFF799FD424A434BD269C2F30212BF
:10257000134493F8303003F01F03D840D5E703A885
:10258000FFF7C8FD04980028C0D0616A3A4B626822
:1025900003EB41034FF6EF71B3F84030B0FBF3F0BB
:1025A000530803EB4003B3FBF2F3A3F110028A429A
:1025B0003FF624AF23F00F02C3F3420392B213435A
:1025C000EB60A3E72D488DE7FFF766FD284A2A4B0D
:1025D000D269C2F30212134493F8303003F01F03A0
:1025E000D840D0E7B0F5004F1DD0FFF755FD204A89
:1025F000214BD269C2F30222134493F8303003F026
:102600001F03D84091E71A4B1A68900640F1A58045
:102610001B681A48C3F3C103D840B7E76846FFF701
:1026200013FE0198AFE7FFF737FD114A124BD2694D
:10263000C2F30222134493F8303003F01F03D84052
:10264000A1E700BFF369FFCF000C0058FFF4FF11B2
:10265000001001400044004000480040004C004091
:10266000005000400014014000780040007C004011
:102670000044025800093D00089C0C080090D0035B
:10268000A868374B03401343364AAB60EB6A23F02C
:102690000F030B43EB62936D03F00703052B3FF62B
:1026A000ADAEDFE803F0413C3303524F2D4B1A68C7
:1026B00095064CD42C482D4B656803EB410305EB84
:1026C0004501B3F84020B0FBF2F399423FF696AED5
:1026D000B3EB053F3FF692AE002319467EF0EAFCCD
:1026E0002A460902030241EA1061680818184FF0EF
:1026F000000341F100017EF0DDFC1D4BA0F54072AE
:102700009A423FF67BAE1B4BD860FFE66846FFF768
:102710009BFD019800283FF4F9AE616ACBE703A85E
:10272000FFF7F8FC0498F5E7FFF7B6FC0D4A0F4BEE
:10273000126AC2F30212134493F8303003F01F03FD
:10274000D840E7E74FF40040B5E70B48B3E71B6814
:102750000548C3F3C103D840ADE7034816E700BFFF
:10276000FFF4FF11004402580090D003089C0C08AD
:10277000FFFC0F00000C005800093D00474A70B4F0
:10278000946A956AD66A15F47C7FC5F30513516B7C
:102790005BD0C1F3CC0106F0010604F0030407EEA0
:1027A000903A06FB01F1012CB8EEE77A06EE901A9A
:1027B000FAEEE96A4ED0022C6DD0002C4DD0DFED40
:1027C000387A87EE876A136BC3F3080307EE903AF3
:1027D000F7EE005AF8EEE77A77EEA67A77EEA57A6A
:1027E00067EE867A2D4AB7EE006A136BC3F3462371
:1027F00007EE103AB8EEC77A70BC37EE067AC7EE2D
:10280000876AFCEEE66AC0ED006A136BC3F3064309
:1028100007EE103AB8EEC77A37EE067AC7EE876A47
:10282000FCEEE66AC0ED016A136BC3F3066306EEC5
:10283000903AF8EEE66A76EE866A87EEA67AFCEEC5
:10284000C77A17EE903A8360704770BCC0E90033D6
:1028500083607047DFED137AB3E713689B06AED54C
:102860001468F7EE005A136B0F49C4F3C102C3F3A7
:102870000803D14007EE903A06EE101AF8EEE77A18
:10288000B8EEC66A77EEA66AC6EE077A36EEA57A85
:1028900067EE877AA6E7DFED057A92E700440258F3
:1028A0000024744C0024744A0090D00320BCBE4B1A
:1028B000344A136830B423F08063334C13602568C6
:1028C00003E023685B1B022B54D813681B01F8D468
:1028D000936A056823F47C3343EA05339362836883
:1028E000C568013B013D5B022D049BB205F4FE056A
:1028F0002B434568013DC5F308052B430569013DA0
:102900002D0605F0FE452B439363D36A456923F0FA
:10291000C0032B43D362D36A856923F020032B4382
:10292000D362D36A23F01003D362D36BC0696FF311
:10293000CF0343EAC003D363D36A43F01003D362E7
:10294000D36AD1B101290CBF43F4801343F40013BF
:10295000D3620C4A136843F080631360216803E07C
:1029600023685B1A022B05D813681B01F8D50020D9
:1029700030BC7047032030BC704743F40023D3625F
:10298000E7E700BF00440258002E0024344A1368D1
:1029900030B423F08053334C1360256803E0236880
:1029A0005B1B022B54D813689B00F8D4936A05680C
:1029B00023F07C7343EA055393628368C568013B47
:1029C000013D5B022D049BB205F4FE052B434568D7
:1029D000013DC5F308052B430569013D2D0605F0B2
:1029E000FE452B431364D36A456923F440632B43AC
:1029F000D362D36A856923F400732B43D362D36A0D
:102A000023F48073D362536CC0696FF3CF0343EA3E
:102A1000C0035364D36A43F48073D362D36AD1B1E1
:102A200001290CBF43F4000343F08073D3620C4AC6
:102A3000136843F080531360216803E023685B1A36
:102A4000022B05D813689B00F8D5002030BC7047D6
:102A5000032030BC704743F48003D362E7E700BF34
:102A600000440258002E0024026810B452E8003FCF
:102A700023F4907342E800310029F7D1144C02F19D
:102A8000080353E8003F234002F1080C4CE80031F2
:102A90000029F4D1C36E012B08D0002320225DF859
:102AA000044BC0F88C204367C366704752E8003F70
:102AB00023F0100342E800310029EED052E8003F35
:102AC00023F0100342E800310029EFD1E5E700BF11
:102AD000FEFFFFEF436BDA69F0B5970683B004465B
:102AE00042D5586AE36AC0B2002B00F09580216B92
:102AF0009847636B1A681D4622F480721A609A68C0
:102B000022F001029A609A6942F008029A61DA6939
:102B1000D6072DD4DA69900701D502221A62DA6944
:102B2000510701D504221A62DA69120701D5082279
:102B30001A62DA69170612D5D4F8BC20212A0ED001
:102B4000D4E909128A4273D0A169895C0132C9B201
:102B500099622169B2FBF1F001FB1022A262DA69ED
:102B6000560608D403B0F0BDDA691D46D607D1D5A4
:102B700001221A62CEE7DA6940F60F0C1E6804F1F2
:102B8000340012EA0C0F996836D0B24F0F4040F073
:102B9000BB80DFF8CCC216EA0C0F40F06381D4F89A
:102BA000A050012D4CD0D50202D54F0200F1678113
:102BB000150606D501F4000106F080050D4340F02E
:102BC00043815106CED57206CCD553E8002F22F0B2
:102BD000400243E8002141B1626B52E8003F23F01C
:102BE000400342E800310029F7D120220023C4F835
:102BF000BC20C4F8AC30B5E79506D0D506F020056A
:102C000001F080573D43CAD0D4F8A830002BA9D09A
:102C100003B0BDE8F0401847E3696269D054E36946
:102C2000E2680133B3FBF2F102FB1133E36160E7C9
:102C30000022A4F88A201A6822F080021A608EE727
:102C4000D706B0D5F506AED51022B4F890501A626A
:102C50009A68570640F11D81D4F8B40001684A68AB
:102C600092B2002A00F05081AA4280F04D81C169E1
:102C7000A4F89220B1F5807F40D053E8002F22F4D1
:102C8000807243E8002141B1626B52E8001F21F4D9
:102C9000807142E80015002DF7D103F1080252E8D7
:102CA000002F22F0010203F1080545E80021002968
:102CB000F3D103F1080252E8002F22F0400203F1A1
:102CC000080545E800210029F3D12022C4F8C020DE
:102CD000C4F8A01053E8002F22F0100243E80026A9
:102CE000002EF7D15C490D6840B190F83530022BC9
:102CF00000F01381802380F8346043650223C4F818
:102D0000A430B4F892302DE712F0010F0CD016F475
:102D1000807F09D04FF0010CC3F820C0D4F8C4C0A4
:102D20004CF0010CC4F8C4C012F0020F7BD112F0B9
:102D3000040F0CD011F0010F09D04FF0040CC3F8B0
:102D400020C0D4F8C4C04CF0020CC4F8C4C012F0C7
:102D5000080F0CD006F0200C5CEA070C07D00827FF
:102D60001F62D4F8C47047F00807C4F8C470170590
:102D70000AD5770108D54FF400671F62D4F8C43034
:102D800043F02003C4F8C430D4F8C430002B3FF41F
:102D9000E9AE92060CD506F0200601F080510E43F4
:102DA00006D0D4F8A8301BB101909847656B019804
:102DB000D4F8C420AB6802F0280203F040031343A8
:102DC00061D0FFF751FEAB685B067FF5CBAE05F136
:102DD000080353E8003F23F0400305F1080141E8F0
:102DE000003262B1626B02F1080353E8003F23F046
:102DF000400302F1080040E800310029F3D1D4F883
:102E0000B40000283FF4AEAE90F83520134B022AF0
:102E100003653BD1FDF72AF900283FF4A3AED4F8AF
:102E2000B400036DF4E611F0010F90D04FF0020CE6
:102E300012F0040FC3F820C0D4F8C4C04CF0040C46
:102E4000C4F8C4C083D078E7D4F8AC30002B7FF44A
:102E5000DFAE87E601000010002E00246910040890
:102E60002001000412F0010F3FF471AF16F4807FCF
:102E70007FF450AF12F0020F7FF469AF57E74FF4C1
:102E800080121A626EE6C4F8C4306BE68022426596
:102E9000BEE6B4F89220B4F8921092B289B2AA4277
:102EA0003FF460AE00293FF45DAE53E8002F22F4FA
:102EB000907243E8002141B1626B52E8001F21F497
:102EC000907142E800100028F7D1954803F10802FC
:102ED00052E8002F024003F1080545E800210029CF
:102EE000F4D12022C4F8A810C4F8C020C4F8A0105F
:102EF00053E8002F22F0100243E800210029F7D107
:102F00000223C4F8A4302DE6AA427FF42BAEC36995
:102F1000B3F5807F7FF426AEF2E70368814A824EE4
:102F2000824FB34218BF934206F118060CBF01222C
:102F30000022B34208BF42F001021836B34208BF74
:102F400042F001021836B34208BF42F001021836BF
:102F5000B34208BF42F0010206F55676B34208BFFD
:102F600042F001021836B34208BF42F0010218369F
:102F7000B34208BF42F001021836B34208BF42F024
:102F800001021836B34208BF42F001021836B342BC
:102F900008BF42F001021836B34208BF42F00102F6
:102FA000A6F59266BB4218BFB34207F592670CBF05
:102FB00001260026BB4208BF42F0010256EA020782
:102FC00079D0D3F800C02CF01E0CC3F800C0D3F8A1
:102FD00014C02CF0800CC3F814C0D0F860C076BBCD
:102FE000D0F860C0DCF8006026F48076CCF8006091
:102FF0001A6822F001021A6003E00A68521B052ACF
:1030000024D81A68D607F8D4D0E9165101F01F0168
:103010002FB33F238B40AB60C36ED0E919215160C1
:1030200033B11A68016F22F480721A60436F4B60EB
:103030000122002380F8352080F834305EE6DCF889
:10304000002022F48072CCF80020D1E72021032256
:103050000023416580F8343080F835204EE6344A4C
:10306000344EB34218BF934206F114060CBF01223E
:103070000022B34208BF42F001021436B34208BF37
:1030800042F001021436B34208BF42F00102143686
:10309000B34208BF42F00102012606FA01F169605D
:1030A00025498B4208BF42F00102002AB4D1234ACD
:1030B0009342B1D0BCE71E4EDFF878C0634518BF1D
:1030C000B3420CF1140C0CBF01260026634508BF67
:1030D00046F001060CF1140C634508BF46F00106EA
:1030E0000CF1140C634508BF46F001060CF1140CFA
:1030F000634508BF46F00106D3F800C02CF00E0C63
:10310000C3F800C0DFF830C0634508BF46F00106D1
:10311000002E7FF465AF094EB3423FF461AF67E71D
:10312000FEFFFFEF4000024058000240280002402E
:10313000085402581C54025880540258945402589F
:103140004B4B10B41B684B4CA4FB03435B0A03FBC3
:1031500002F25AB18446531E4748DCF83420013B42
:10316000024201D0920406D55C1CF6D14FF000401B
:103170005DF8044B7047DCF834305C0741D4DCF870
:103180003430D80709D43D4BCCF83830DCF8103057
:10319000DBB2994205D00120EAE70123CCF83830B0
:1031A000F9E7DCF81430364818400028E0D0002B4E
:1031B0002CDB5A002DD49C002DD4D9002DD41A011B
:1031C0002ED45C012FD4D90130D41A0231D45C0240
:1031D00032D499023CD4DA0237D45C0332D4990356
:1031E0002DD4DA0340D41C043BD4590436D49A04B9
:1031F00031D413F0080F0CBF4FF480304FF40000AF
:10320000B6E704231846CCF83830B1E74FF0007029
:10321000AEE74020ACE78020AAE74FF48070A7E734
:103220004FF40070A4E74FF48060A1E74FF4006012
:103230009EE74FF480509BE74FF4005098E74FF41F
:10324000802095E74FF4003092E74FF400408FE77D
:103250004FF480408CE74FF4800089E74FF4001072
:1032600086E74FF4801083E74FF4002080E700BF2B
:1032700000000024D34D621045002000C50020004E
:1032800008E0FFFD82B00023019302E00369002BF8
:1032900009DB019B01330193019BB3F1706FF5D9F9
:1032A000032002B070478901002341F020010193FF
:1032B000016103E0036913F0200307D0019B013390
:1032C0000193019BB3F1706FF4D9E9E7184602B09E
:1032D000704700BF82B00023019302E00369002B16
:1032E00009DB019B01330193019BB3F1706FF5D9A9
:1032F000032002B07047002210230192036103E013
:10330000036913F0100307D0019B01330193019B64
:10331000B3F1706FF4D9EBE7184602B0704700BF05
:1033200082B00023019302E00369002B09DB019BBB
:1033300001330193019BB3F1706FF5D9032002B003
:10334000704700230193036943F00103036103E025
:10335000036913F0010307D0019B01330193019B23
:10336000B3F1706FF4D9E9E71846E8E72DE9F843BF
:10337000056807460C46C5F31009B9F1000F39D1AD
:103380008A4B4FF6FF72B3F88030934256D0002B31
:1033900054D0874A02EA432808F10068454534BF03
:1033A0004FF001084FF00208824B9D4206D903F509
:1033B00000339D4200F2CF804FF001097E4E96F817
:1033C0005C34012B12D00123B8F1010F86F85C3474
:1033D0004FF00003C6F8603436D0022073F04AF88C
:1033E000002800F09980002386F85C344FF0FF300D
:1033F000BDE8F883704E96F85C34012B4CD0012365
:1034000086F85C3405F17843B3F5801F48D3A5F105
:103410000163B3F5801F3FD200230220C6F8603459
:1034200073F028F8002870D1644A4FF00208D2F8EF
:103430000C3143EA0803C2F80C313FE0B5F1016FEB
:1034400067D3052011F0C6FD404673F013F800283D
:10345000C9D14046DFF86481D8F80C3023F4E66324
:10346000C8F80C30D8F80C3043EA092343F0A40321
:10347000C8F80C3072F0FEFFD8F80C20504B134007
:10348000C8F80C300028AED105F178430122B3F51D
:10349000801F86F85C2403D36FF00100BDE8F88339
:1034A00000230120C6F8603472F0E4FF68BB434A91
:1034B0004FF00108D36843F00203D360BFF36F8F6E
:1034C000BFF34F8F04F1200254F8043B944245F8B7
:1034D000043BF9D1BFF36F8FBFF34F8F404672F0BB
:1034E000C9FFB8F1010F354A30D0D2F80C3123F0C2
:1034F0000203C2F80C31002386F85C340028CBD1DB
:103500003B6820333B60BDE8F883002386F85C34D9
:10351000C2E74FF0010847E7DFF8A0800220D8F8A3
:103520000C3123F4E663C8F80C31D8F80C3143EAC7
:10353000092343F0A403C8F80C3172F09BFFD8F8BC
:103540000C211F4B1340C8F80C319BE7D36823F0C4
:103550000203D360CFE703F500339D4211D903F591
:1035600000339D4210D903F500339D4206D903F57F
:1035700000339D420BD84FF005091FE74FF00409B7
:103580001CE74FF0020919E74FF0030916E703F5AE
:1035900000339D4206D9B5F1016FBFF452AF4FF031
:1035A00007090BE74FF0060908E700BF00E8F11F25
:1035B00000FE1F00FFFF0108002E00240020005223
:1035C000FBF8FFFF0148FCF74DBF00BF6832002445
:1035D000084810B4D0F86834D0F89C4499691A6847
:1035E0002CB1234600F58D605DF8044B18475DF85B
:1035F000044B7047002E00240148FCF733BF00BF86
:10360000C0320024084810B4D0F8C034D0F8F444D4
:1036100099691A682CB1234600F598605DF8044B4F
:1036200018475DF8044B7047002E00240148FCF752
:1036300019BF00BF18330024084810B4D0F818355B
:10364000D0F84C4599691A682CB1234600F5A3605F
:103650005DF8044B18475DF8044B7047002E0024BA
:103660002DE9F04FDFF8649300EB400583B0430091
:1036700009EB85050093D5F8A0300193002B00F0ED
:1036800062818046B5F8A60072F080FA95F8A40031
:103690000DF02AFE044695F8A5000DF025FE08F170
:1036A00001030746DBB2002C00F0728140F60C12D9
:1036B000A1882372E2802268002800F05D810372F5
:1036C00040F60C23C38091613B68BA889A6111214E
:1036D000204609260DF0C4FD112138460DF0C0FD2D
:1036E0006525002C00F032812268A38811690B4205
:1036F00000F02C811B04936111F010FC05468B46F1
:1037000011F00CFC401B61EB0B01052871F100016D
:10371000F6D314B12368A2889A6111F0FFFB054625
:103720008B4611F0FBFB401B61EB0B01052871F18F
:103730000001F6D3013ED3D11CB1A38822681B043B
:10374000936111F0EBFB05460E4611F0E7FB401BC1
:1037500061EB0601052871F10001F6D31FB1BB88AA
:103760003A681B04936111F0D9FB05460E4611F02F
:10377000D5FB401B61EB0601052871F10001F6D372
:1037800014B12368A2889A6111F0C8FB05460E4661
:1037900011F0C4FB401B61EB0601052871F100012B
:1037A000F6D317B13B68BA889A61009B20463E2148
:1037B000434409EB830393F8AB4022460DF072FDBE
:1037C000224638463E210DF06DFD7A4C5823019A71
:1037D00003FB0843C3F86824774B9A4200F0C78084
:1037E000FEF75AFC754BDA69C2F30212744B1344AC
:1037F00093F8303003F01F03D840009B434409EB9B
:10380000830393F8A830022B00F0BD80032B00F057
:10381000B580012B14BF4FF4C8714FF4487172F09A
:1038200043FA03465822002102FB0842C2F87014F2
:10383000C2F87814C2F87C14C2F88414C2F8881450
:103840000121C2F86C34C2F8741492F8A91401F082
:10385000FF00002900F0A480582123F07062242684
:103860004FF4004701FB08415648D1F8683481F80D
:10387000A9641D6825F001051D601A619A6822F48B
:1038800000429A609F605A6822F400625A605A6847
:103890001043D1F8802458601202D86820F4004008
:1038A000D860DA6000221A60186840F001001860E1
:1038B0002020C1F8AC2481F8A904C1F8982481F82B
:1038C000AA2491F8A9042028C5B217D191F8A80418
:1038D000012813D081F8A964186820F0010018604D
:1038E000186820F48050186018681860186840F054
:1038F0000100186081F8A95481F8A824009B0221D6
:103900000126314F434409EB830999F8AA50284610
:1039100072F004FE05F01F036A0999F8A95006FA2F
:1039200003F30221284647F8223072F0F7FD5823AE
:1039300003FB084405F01F036D0906FA03F347F87B
:10394000253084F8646403B0BDE8F08F013D2AD0CF
:1039500011F0E4FA83468A4611F0E0FAB0EB0B006E
:1039600061EB0A01052871F10001F5D3B9E6FEF714
:1039700093FB124B1A6A37E79161A8E6C82172F0EF
:1039800093F903464EE7642172F08EF9034649E746
:1039900000283FF49CAE037240F60C23C38093E6EC
:1039A00082F8A80458E7002C3FF4A6AEA38822684A
:1039B000A0E600BF002E0024001C0058004402585E
:1039C000089C0C080080000200E100E000000024D8
:1039D0002DE9F04F441C85B017469DF83C202DD0B2
:1039E0005824DFF8A8831E46054600FB04F408EBC4
:1039F000040393F86494B9F1000F1FD044444900C4
:103A0000FF2F04F58D64039100D0EEB9002A40F039
:103A1000C680582303FB058393F8A924202A04D1E8
:103A2000B6B94FF40072C3F8AC24B8F86C35284628
:103A300001339BB2A8F86C35FFF712FE4FF0000976
:103A4000484605B0BDE8F08F93F8A934202BECD19F
:103A50004FF0580A0AFB058A9AF8A834012BE4D0E3
:103A60000122D8F800B019234FF400418AF8A824A5
:103A70002046CDF800B0FEF7ABFA0028D5D10E9B5A
:103A8000DAF86814CAF88C342123BA4A8AF8A934BF
:103A90004023CAF89C048AF8AA34CAF8AC04204629
:103AA000AAF892644B681340039A1343B24A1A432C
:103AB0004A60594672F0B0FC0246002840F0FB8094
:103AC000DAF86834802120469F620A23CDF800B0DE
:103AD000FEF77EFA002840F0EE80BAF892349BB2EE
:103AE000FF2B40F21681DAF86814FF23A348AAF8E6
:103AF00090344B68A24A0340039803431A434A6038
:103B00005826DDF80CA05F46039506FB058605E008
:103B1000B6F892349BB2002B00F010813946204653
:103B200072F07AFC002840F0F280D6F88C14D6F8B7
:103B3000685411F8012BB6F89034AA62C6F88C14B8
:103B4000013BB6F892149BB20139A6F8903489B2C1
:103B5000A6F89214B6F8921489B2002BD8D1002995
:103B6000D6D002460A23802120460097FEF730FA7D
:103B7000FF22002840F0CB80B6F892349BB29342EB
:103B800040F2A080D6F86814A6F890244B687B4ACF
:103B900013407B4A43EA0A031A434A60B8E74FF0EE
:103BA000580A0AFB058A9AF8A934202B7FF43DAF06
:103BB0009AF8A834012B3FF438AF0122D8F80070EE
:103BC00019234FF400418AF8A82420460097FEF7F5
:103BD000FFF900287FF429AF0E9BCAF89C04CAF8AD
:103BE0008C3421238AF8A93410238AF8AA34CAF81D
:103BF000AC04AAF89264BAF892349BB2FF2B00F29C
:103C0000C780BAF892349BB2AAF89034002B40F0E7
:103C1000F180DAF8681457484B685A4A0340039811
:103C200003431A434A605826AA4606FB0586B6F89F
:103C3000923439469BB2002B00F0D480204672F0BB
:103C4000EBFB002878D1D6F88C14D6F8685411F81C
:103C5000012BB6F89034AA62C6F88C14013BB6F872
:103C600092149BB20139A6F8903489B2A6F8921446
:103C7000B6F8921489B2002BD9D10029D7D00246C8
:103C80000A23802120460097FEF7A2F9FF22002890
:103C900052D1B6F892349BB2934225D9D6F8681423
:103CA000A6F890244B68354A1340039A1343344ACC
:103CB0001A434A60BBE75823002203FB058383F8BD
:103CC000A824B2E6B6F89234D6F868249BB22B4802
:103CD0005168A6F89034DBB201404AEA03430B4333
:103CE00043F00073536013E7B6F89234D6F86814C3
:103CF0009BB2039A2148A6F89034DBB242EA034310
:103D00004A680240134343F000734B608FE7039D02
:103D10008BE6BAF89234DAF868149BB2039A174823
:103D2000AAF89034DBB242EA03434A6802401343E4
:103D300043F000734B60E3E6554676E6394620468D
:103D4000039D72F03BFB00287FF46FAED6F8683419
:103D500020210D4CD9615A6822405A605823002214
:103D600086F8A91403FB058386F8AA0483F8A8241F
:103D700066E600BF009800FC00200101009C00FCEA
:103D80000000FF010020000200E800FE002E0024D9
:103D9000FF234FF47F00FE224FF08076AAF8903484
:103DA000039BDDF838E01E4358231EF801AB03FBEC
:103DB0000583DFF850C0D3F86814C1F828A0A3F831
:103DC0009024B3F89224C3F88CE4013A92B2A3F899
:103DD00092244B6803EA0C033343034343F4005338
:103DE0004B6020E72046554672F0E8FA00287FF441
:103DF0001CAEABE7013B4FF000769AB2501CC0B24C
:103E00000004CDE7009800FC2DE9F04F441C85B07C
:103E100099469DF83C3000F096805825C64C0646E1
:103E200000FB05F504EB050B9BF864A4BAF1000F49
:103E300000F089802544FF2A90464FEA410705F5A6
:103E40008D6540F08680002B00F083809BF8A934BC
:103E5000202B6FD19BF8A834012B6BD00122D4F812
:103E6000008019234FF400418BF8A8242846CDF890
:103E70000080FEF7ADF800285CD10E9BCBF89C04C7
:103E8000CBF88C3422238BF8A93410238BF8AA3476
:103E9000CBF8AC04ABF89294BBF892349BB2FF2BF6
:103EA00000F21781BBF89234DBF868149BB2A34888
:103EB0004A68ABF89034DBB2024047EA034313434D
:103EC0009F4A1A434A604FF0580909FB0649B9F85E
:103ED00092349BB2002B00F08A81D9F868349A6939
:103EE000520700F1378142460A212846FDF7EEFFCE
:103EF000002840F0FB80D9F868349A69910640F1B7
:103F000000819A699A6912F0100200F0F88010227C
:103F100020218C4DDA610422C9F8AC24D9615A6899
:103F20002A405A6089F8A91489F8A80489F8AA04D3
:103F300022689B69B4F86C35304601339BB2A4F813
:103F40006C35FFF78DFB4FF0000A504605B0BDE819
:103F5000F08F4FF0580B0BFB064B9BF8A934202B2E
:103F6000E8D10E9B002B00F0AC80B9F1000F00F0FF
:103F7000A8809BF8A834012BDCD0236801224FF4E1
:103F8000004128468BF8A824039300931923FEF7D9
:103F90001FF80028CED12223DBF868140E9A8BF884
:103FA000A9344023CBF88C248BF8AA34CBF8AC048A
:103FB000ABF89294DFF884914A68CBF89C042846C9
:103FC00002EA09023A4342F490324A60039972F0DD
:103FD00023FA0246002840F036814023284619463D
:103FE000DBF86834C3F82880039B00930A23FDF7AD
:103FF000EFFF002840F02781BBF892349BB2FF2BE3
:1040000040F22881DBF86814FF234F4AABF8903464
:104010004B6803EA09033B431A434A604FF05808D0
:10402000B946039F08FB064805E0B8F892349BB2F6
:10403000002B00F021810A2300220421284600974A
:10404000FDF7C6FF00287FF475AFD8F86834596AC9
:10405000D8F88C341970B8F89214D8F88C34013927
:10406000013389B2C8F88C34B8F89034A8F89214A7
:10407000013BB8F892149BB289B2A8F89034002999
:10408000D3D0002BD1D102460A23802128460097A5
:10409000FDF79EFFFF2200287FF44CAFB8F8923462
:1040A0009BB2934240F2BD80D8F86814A8F89024DF
:1040B0004B68264A1340264A43EA09031A434A60DA
:1040C000B3E758234FF4007203FB0643C3F8AC2454
:1040D00030E7DBF86814FF231848ABF890344B68DE
:1040E000194A03403B431A434A60ECE6582303FB5A
:1040F0000643D3F868349A6922689B691AE7C9F8BD
:10410000AC242268A2EB08020A2A7FF6E8AE9A697C
:1041100012F004027FF4E3AE582101FB0641D1F80E
:10412000AC0481F8A824202240F02000C1F8AC049F
:1041300081F8A9249B69FDE6002E0024009800FC6C
:104140000024000200E800FE0024FF01009C00FCA7
:104150000000FF015A6AD9F88C341A70B9F8923409
:10416000D9F88C24013B01329BB2C9F88C24A9F800
:104170009234B9F89034B9F89224013B92B29BB2D0
:10418000A9F89034002A3FF4A2AE002B7FF49FAE32
:104190000A23002280212846CDF80080FDF718FF71
:1041A00000287FF4C7AEB9F892349BB2FF2B0CD92C
:1041B000D9F86814FF233B48A9F890344B683A4A71
:1041C00003403B431A434A6081E6B9F89234D9F878
:1041D00068149BB233484A68A9F89034DBB20240B5
:1041E00047EA0343134343F000734B606FE64146D5
:1041F000284672F0E3F800287FF49CAED9F86834C2
:1042000020212A4DD9615A682A405A6089F8A91498
:1042100089F8AA045822002302FB064484F8A83433
:1042200093E6B8F89234D8F868249BB21D485168D8
:10423000A8F89034DBB2014049EA03430B4343F052
:1042400000735360F1E65823002203FB064383F812
:10425000A8246FE6BBF89234DBF868149BB24A6876
:10426000ABF89034DBB202EA090247EA0343134396
:104270000F4A1A434A60D1E60399284672F09EF825
:10428000034600287FF456AED8F868242020074D56
:10429000D06151682940516088F8A90488F8AA348F
:1042A000B8E700BF009C00FC0000FF0100E800FE32
:1042B000002400020348D0F8D0300BB1C4301847B6
:1042C000704700BF000000240348D0F8F0300BB165
:1042D000E4301847704700BF000000240348D0F8BE
:1042E000103113B100F582701847704700000024A8
:1042F0000348D0F8303113B100F592701847704779
:10430000000000240348D0F8503113B100F5A2702A
:1043100018477047000000240348D0F8703113B1EB
:1043200000F5B27018477047000000240348D0F829
:10433000903113B100F5C270184770470000002497
:104340000348D0F8B03113B100F5D2701847704768
:10435000000000240348D0F8D03113B100F5E2701A
:1043600018477047000000240348D0F8F03113B11B
:1043700000F5F27018477047000000240348D0F899
:10438000103213B100F50170184770470000002487
:104390000348D0F8303213B100F509701847704760
:1043A000000000240348D0F8503213B100F511701A
:1043B00018477047000000240348D0F8703213B14A
:1043C00000F5197018477047000000240348D0F822
:1043D000903213B100F52170184770470000002497
:1043E0000348D0F8B03213B100F529701847704770
:1043F0000000002410B41C46436884466FF30F038A
:1044000023434360036843F001030360036843F4FC
:1044100000730360002C3AD040F2E930DCF814302D
:104420009B0748D5002A49D012F8013B40F2E930F9
:104430008CF82030DCF81430DB0720D40138F9D1B7
:10444000214B9C450CD0A3F578439C4538D003F50F
:1044500080639C4536D003F578439C450BD10320FF
:104460001A4A00EB400002EBC002B2F8D832013326
:104470009BB2A2F8D83200205DF8044B70479CF83C
:104480003000C0B209B101F8010B013CC4D1DCF825
:1044900014301B07FBD5DCF8183001205DF8044B05
:1044A00043F01003CCF81830DCF8003023F001039F
:1044B000CCF8003070470138B0D1C1E7FF23B5E731
:1044C0000120CDE70220CBE70030014000000024AE
:1044D0002DE9F84300242C4E8046036856F83450EA
:1044E000AB4209D001340E2CF8D1284A0021052016
:1044F00006F0DAFF002019E0254B03EB8409D9F818
:104500007075AFB198F8051000204B1C01EB41020B
:1045100003EB430307EBC202DB00C2F80C80C2E9E5
:104520000400F854182303FB01700830BDE8F88339
:104530000721682007F03EF80146C9F87005F0B180
:104540003946682284F0FEF9D9F8701506EBC404E8
:104550003B4689600C6009628963096556F833201F
:10456000954205D001330E2BF8D14F600F46C9E7B5
:10457000084F4C2202FB03774F600F46C2E7064A02
:10458000052006F091FFB5E7609C0C0868470D0810
:10459000002E0024A833002490470D0830B40C4CA2
:1045A0000022234603E0013214330E2A0CD093F884
:1045B00004C08445F7D1DD68294201D10029F2D138
:1045C000142303FB024000E0002030BC704700BF12
:1045D00024030024F0B54468A37913F002025FD0ED
:1045E00002224FF0080C036864795B689B48204402
:1045F00093F83C40012C90F8C80050D0012483F877
:104600003C40142848D8DFE810F015004700470068
:10461000470084004700470047003B014700470030
:104620004700BB00470047004700F2004700470033
:1046300047004D0018688A4C056A8A4E25F002052D
:10464000B04242EA0502056A25F0010505624768A5
:10465000856904EA050444F0600407D0824DA8424D
:1046600004D005F57055A84240F04D8122F00802B3
:1046700047F440774CEA020222F00402476084616A
:1046800041630262826942F008028261826922F01B
:104690000402826182698261002283F83C20F0BDBD
:1046A0009446A0E718686F4E046AB04224F40014E0
:1046B00044EA0252046A24F4801404626B4C456894
:1046C000476D04EA070444F4C0440ED006F5806642
:1046D000B0420AD0664F06F58046B04218BFB842D5
:1046E00003D006F58066B04201D145F480254560CF
:1046F0004465C1650262426D42F400624265426DEA
:1047000022F480624265426D4265002283F83C20BB
:10471000C5E71868574C056A524E25F02005B0428F
:1047200045EA0215026A22F01002026247688269B5
:1047300004EA020444F4C04400F0DE804A4A904295
:1047400000F0DA804A4E4C4A904218BFB04203D083
:1047500002F58062904201D147F44067476084616E
:1047600081630562826942F400628261826922F497
:104770008062826182698261002283F83C208EE738
:104780001868384E046AB04224F4005444EA0232F5
:10479000046A24F480540462364C4568C76904EA0C
:1047A000070444F4C0440ED006F58066B0420AD037
:1047B0002F4F06F58046B04218BFB84203D006F529
:1047C0008066B04201D145F480454560C461016412
:1047D0000262C26942F40062C261C26922F480626C
:1047E000C261C269C261002283F83C2057E71868A1
:1047F0001C4E046AB04224F4003444EA0242046AC3
:1048000024F4803404621D4C4568476D04EA0704B3
:1048100044F060040ED006F58066B0420AD0144F12
:1048200006F58046B04218BFB84203D006F5806650
:10483000B04201D145F4803545604465816502622E
:10484000426D42F008024265426D22F00402426568
:10485000426D4265002283F83C2020E7089C0C084A
:104860008CFFFEFF0000014000040140FF8FFFFEAF
:1048700000400140FF8CFFFE004401408FFFFEFF1F
:104880001868264C056A264E25F4007EB0424EEA92
:104890000225026A22F4807202624768C26904EA51
:1048A000020444F0600420D01E4A90421DD01E4EE7
:1048B0001E4A904218BFB04203D002F58062904277
:1048C00001D147F440574760C461C1630562C269C2
:1048D00042F00802C261C26922F00402C261C269E8
:1048E000C261002283F83C20D9E625F4006E4EEA2E
:1048F0000C2E2EF48065E4E725F0800545EA0C15C2
:1049000025F0400528E705F58065A8423FF4AEAEE6
:1049100005F58065A8427FF4B1AEA7E68CFFFEFFE7
:1049200000000140000401400040014000440140FB
:1049300042685379032B0FD8DFE803F00B08050218
:1049400010684030704710683C307047106838304D
:10495000704710683430704700207047D0E900027B
:10496000064B517992790B44406893F8C81053076D
:1049700001D57AF0B9BA7AF033BB00BF089C0C08B5
:10498000F0B54468374A2469C368C4F303245B68FC
:1049900052F82460EFF31184102585F312884568DE
:1049A000314F95F805E0D0F80CC002EB4E02D5F877
:1049B00000E0158CDEF80C2005F4F05522EA050223
:1049C000CEF80C2017F806E0DCF8102053F80E5053
:1049D0001F2A25F0010543F80E5039D9203A202529
:1049E000DCF804C005FA02F2CCF80C20E2B282F343
:1049F0001188BA5DDFF874C003EB020E46684569A2
:104A0000DEF8044004EA0C0C4CEA0101CEF8041074
:104A10007179032924D8DFE801F0181512023168F2
:104A20004031CEF80C500124CEF80810995841F0CE
:104A3000100199509958214399500474F0BD316880
:104A40003C31EEE731683831EBE731683431E8E783
:104A50002025DCF804C005FA02F2CCF80820C5E7EE
:104A60000021DEE7089C0C08389D0C080000FFFFC1
:104A700003681A7E012A2ED0002293F830100129F3
:104A800009D093F8481001290ED093F8601001293D
:104A90001BD02ABB7047022142F4806283F8301099
:104AA00093F84810012904D1022142F4006283F8EE
:104AB000481093F86010012907D01B6800211B687B
:104AC0005962D9680A43DA607047022142F4805281
:104AD00083F86010F1E702214FF400721976CCE7F9
:104AE0004FF40072E9E700BF08B5204B98420ED0A2
:104AF00003F5806398420AD01D4A03F5804398422B
:104B000018BF904203D003F5806398421BD1FDF794
:104B1000C3FA1849184BCA69C969C2F30222C1F322
:104B200002211A4492F8302002F01F02D040114AAC
:104B30001269C2F3C03241EAC202134493F8CC3086
:104B400003FB00F008BDFDF7A7FA0A490A4BCA6942
:104B5000C969C2F3021CC1F3021103EB0C0292F803
:104B6000302002F01F02D040E1E700BF000001400A
:104B70000040014000440258089C0C0870B50E46E5
:104B800005EE102AD0E90031013E1A680868B6B275
:104B90005C681568FFF7A8FF07EE900AB8EE455A63
:104BA0009FED5D7AF8EE677A87EE850A30EE070AA8
:104BB0007EF042FE23680138AB4280B268D0C4E97F
:104BC000005000238022E660A360A261C4E90433A0
:104BD00094F83D3003F0FF02002B78D00223211D12
:104BE000284684F83D30FCF771F94C4A0123B5F1B1
:104BF000804FA5EB020284F84830B2FA82F284F8C2
:104C00003E3084F83F304FEA521284F8403084F846
:104C1000413084F8423084F8433084F8443084F8DA
:104C2000453084F8463084F8473084F83D3034D03D
:104C30009ABB3B4B9D420CD003F580639D4208D04C
:104C400003F580639D4245D003F578439D4241D0F2
:104C500070BD94F83C30012BFAD00222314B012177
:104C600084F83D20A8680340AB6084F83D1084F8C8
:104C70003D206B68A96823F0700321F080010122B8
:104C80006B600023A96084F83D2084F83C3070BD3F
:104C9000636883423AD0606093E794F83C30012B1C
:104CA000D6D002211F4B002084F83D10A9680B408C
:104CB0000121AB6084F83D10022384F83D306B681D
:104CC000A9680AB90028D6D023F47003D3E784F882
:104CD0003C2083E794F83C30012BB9D00221114BE2
:104CE000114884F83D10A968281A0B40B0FA80F0EA
:104CF0000121AB600023400984F83D1084F83C306A
:104D00000A4B9D42D8D00028D6D170BDE368B3428B
:104D10007FF457AF70BD00BF0AD7233C00000140AD
:104D2000000400408800CEFF00040140000C004059
:104D3000024B0348D3F87015FCF7F0BC002E00249A
:104D400000000140034B4FF08040D3F87415FCF78E
:104D5000E5BC00BF002E0024024B0348D3F87815B1
:104D6000FCF7DCBC002E002400040040024B03488A
:104D7000D3F87C15FCF7D2BC002E002400080040BC
:104D8000024B0348D3F88015FCF7C8BC002E002462
:104D9000000C0040024B0348D3F88C15FCF7BEBC56
:104DA000002E002400040140024B0348D3F89C1558
:104DB000FCF7B4BC002E002400180040024B03484E
:104DC000D3F8A815FCF7AABC002E0024004001402F
:104DD000024B0348D3F8AC15FCF7A0BC002E00240E
:104DE00000440140024B0348D3F8B015FCF796BCD1
:104DF000002E00240048014010B5064C0648D4F8A7
:104E00008C15FCF78BFCD4F8A0150448BDE81040C5
:104E1000FCF784BC002E002400040140001C00406C
:104E200010B5064C0648D4F88C15FCF777FCD4F87E
:104E3000A4150448BDE81040FCF770BC002E002407
:104E40000004014000200040BFF34F8F0549064B8E
:104E5000CA6802F4E0621343CB60BFF34F8F00BF18
:104E6000FDE700BF00ED00E00400FA05002101208D
:104E700008B50EF037F872B6FFF7E6FF2DE9F043FC
:104E8000BFB0BFF35F8FA14C0023626A22F480326F
:104E90006262C4F894309DF843109DF844C009063E
:104EA0009DF842200F9841EA0C7141EAC2419DF8F9
:104EB000452041EA82419DF8462041EA42419DF861
:104EC000472041EA02419DF8412041EA02219DF834
:104ED000402041EA4201C4F898300133D4F8A020C0
:104EE000112B22F00102C4F8A020C4F89C00C4F8E1
:104EF000A010F0D10523C4F89430636A43F48033E2
:104F00006362BFF34F8FBFF36F8F8148814A82493D
:104F1000121A82F0EFFB814B5A6D012A00F0DF80FC
:104F2000D4F8881000227E4B012041F47001C4F8AF
:104F3000881018601A61196841F0800119601968B9
:104F400001431960196841F480311960196841F40E
:104F5000805119609A61DA611A629A62DA621A63A0
:104F60005A639A63DA631A645A64196821F48021D7
:104F700019601A664FF000636A49C1F80801A3601E
:104F80007BF046F9684AD36813F0040FD36840F009
:104F90009480664B0021644A0591D96A21F0010191
:104FA000D962DB6A03F001030593936943F440433C
:104FB0009361936903F440430593059B93699E04B1
:104FC000FCD54C2200210EA8594C83F0BBFC594A59
:104FD00042F20303A4F110011268B3EB124F4FF039
:104FE00000024FF00C0308BF0C460892E268A37061
:104FF000002A4FD04D4BD96A21F00101D962DB6AFA
:10500000494903F0010308938B6923F44043134398
:105010008B618B6903F440430893089B424A936970
:105020009D04FCD53E4B4FF4403543480321D3F853
:10503000E02042F08002C3F8E0200122D3F8E03003
:1050400003F080030793079B85610D9BCDE9001357
:1050500000237AF08BFF022301204FF48031A288D5
:10506000CDE917330C231993A379CDE90E01E0792B
:10507000217A1C900EA81D91CDE91A230822002345
:10508000CDE91E23FBF7EEFB032800F06082002829
:1050900058D0FEE7244A254B916941F44041916183
:1050A000926902F440420892DA6A42F00102DA623E
:1050B000DB6A03F001030893AFE723F007031F4CFB
:1050C00043F00203D360216805E023685B1AB3F55F
:1050D0007A7F3FF65EAF53689F04F6D559E7104AD2
:1050E000002017495865D2F8F43043F00203C2F8A3
:1050F000F430D2F8F43003F002030E930E9B0B68E9
:1051000083F308884B689847FEE700BF00ED00E096
:1051100000000000B0370000E0C60D080040005855
:105120000044025800800051004802580004005812
:105130004C0400240010005C001C0258002E0024C7
:105140000098F01F754B1A6812F00E0F0BD11A68F9
:1051500022F00F0242F002021A601B6803F00F03F4
:10516000022B40F0F6816E4A936903F070033F2BE7
:1051700005D8936923F0700343F040039361684AB4
:10518000D36903F070033F2B05D8D36923F0700374
:1051900043F04003D361624AD36903F4E063B3F59B
:1051A000806F05D2D36923F4E06343F48063D36155
:1051B0005B4A136A03F070033F2B05D8136A23F090
:1051C000700343F040031362554B9A69140705D4EA
:1051D0009A6922F00F0242F008029A61504A9369DC
:1051E00023F4706393611368980130D5136941F219
:1051F00088314C4C23F0070343F00303136120680C
:1052000004E023681B1A8B4200F2AC81136903F09F
:105210003803182BF5D1936903F00F03082B05D938
:10522000936923F00F0343F0080393613B4A13682B
:1052300003F00F03022B0BD9136823F00F0343F085
:1052400002031360136803F00F03022B00D0FEE784
:10525000334A936903F07003402B05D9936923F017
:10526000700343F0400393612D4AD36903F0700348
:10527000402B05D9D36923F0700343F04003D36179
:10528000274AD36903F4E063B3F5806F05D9D36986
:1052900023F4E06343F48063D361214A136A03F08B
:1052A0007003402B00F256811D4EFCF7D3FE1E4DBD
:1052B000B269B369C2F303221C4B134493F8303034
:1052C00003F01F0320FA03F3D5F89C002B60FCF7D2
:1052D0004FFD002840F08D811023159017900EA8E7
:1052E0000E93FBF7BFFA002840F030813368104A74
:1052F00043F080033360D6F8F43043F00203C6F87D
:10530000F430D6F8F43003F002030493049B136ADC
:1053100043F001031362074B216810E000200052A4
:1053200000440258002E002400000024089C0C08B1
:105330000004005880380100013B00F00881226819
:105340009142F9D0226823689B1A0A2BFBD90021CD
:105350004FF48020A74C4FF44013002600273093D1
:105360004FF00208CDE90E010EA879F025FFD4F820
:10537000EC30A14941F2030243F002030EA8C4F845
:10538000EC30D4F8EC3003F002030393039BD4F821
:10539000943043F00203C4F89430D4F8943023F0EE
:1053A0000203C4F894300B689449B2EB134F944B4A
:1053B000944A28BF0A465A601A6822F47C5242F482
:1053C00000521A601A6842F060021A600322002339
:1053D000CDE92C67CDE90E2379F0EEFE4FF4E042E3
:1053E00000230EA8CDE9266700270326CDE90E236A
:1053F0003A9779F0E1FE182200230EA82F973497F0
:10540000CDE90E2379F0D8FE4FF4803200230EA8A8
:105410001797CDE90E2305224FF4FA73CDE9102337
:10542000042314934FF48033CDE915772293CDE90B
:10543000128679F0C1FED4F8E03042464FF4807114
:1054400043F001037048C4F8E030D4F8E03003F0D2
:1054500001030993099B3B46CDE900677AF086FD7D
:1054600023694246694823F0FE7343F08873236141
:10547000D4F8E03043F00403C4F8E030D4F8E0306E
:1054800003F0040306933B4606994FF40071CDE9FF
:1054900000677AF06BFD236923F07E4343F0FC4301
:1054A0002361FCF7D7FD2860BFF35F8F584C3E4661
:1054B000584D4FF00108636A23F480336362C4F8E7
:1054C000947028E0002A4CD02F686B7A103515F8BC
:1054D000061C1B0643EA017343EA420315F8052C38
:1054E00043EA824315F8042C43EA424315F8032C9F
:1054F000C4F89860013643EA0243D4F8A020032E92
:1055000043F0010322F00102C4F8A020C4F89C700B
:10551000C4F8A03027D06B682A7A002BD2D02F682D
:10552000002AD2D127F01F02A3EB0209B9F1200F04
:1055300038BF4FF02009484682F052F8421E08FA60
:1055400002F1894508BF0246D2B2BEE7FEE7FFF787
:105550008DFC7CE6136A23F0700343F04003136272
:10556000A2E6FEE773E60523C4F89430636A43F4C9
:1055700080336362BFF34F8FBFF36F8FBFF34F8FE3
:10558000BFF36F8F0022C4F85022BFF34F8FBFF3D9
:105590006F8F636943F400336361BFF34F8FBFF3D1
:1055A0006F8FC4F88420BFF34F8FD4F8805043F638
:1055B000E0761749C5F34E34C5F3C905640104EA22
:1055C00006002B4640EA8372013BC1F86022F9D203
:1055D000203C14F1200FF2D1BFF34F8F4B6943F4FD
:1055E00080334B61BFF34F8FBFF36F8F3FB0BDE888
:1055F000F0832CE6004402580010005C7FBB2200C0
:10560000008400407FBB223000000258000802588E
:1056100000ED00E05C0400242DE9F843374E984685
:1056200006EB8003D3F8DC40002C65D004F1D203F4
:10563000FC360546B4F8D202A36104F5E97366604E
:105640001746E3614FF48073261DE160C4E904331B
:105650002368C4F8CC30A36300284AD194F8D10061
:105660000BF042FE18F0080F94F8D09034D1BA072E
:1056700023D4FB0711D4052194F8D60270F04EFF15
:1056800094F8D63201221E4903F01F005B098240C4
:1056900041F823203046BDE8F883013548460BF039
:1056A00023FEEDB218B140F206630572C38094F890
:1056B000D42202210BF0F6FDDDE76B1CDBB218B142
:1056C000037240F20653C38094F8D52202210BF0F6
:1056D000E9FDFB07CFD5E0E70135EDB218B140F2A7
:1056E00006730572C38094F8D52202210BF0DAFD0F
:1056F000C1E770F04BFAB1E72646CBE7089C0C08EF
:1057000000E100E00148FDF7E5B900BF9004002486
:105710000148FDF7DFB900BF680700240148FDF725
:10572000D9B900BF400A00240148FDF7D3B900BF32
:10573000180D00240148FDF7CDB900BFF00F00247B
:105740000148FDF7C7B900BFC81200240148FDF7A2
:10575000C1B900BFA015002470B52422456B0023F9
:105760008168C0F8BC2004462A6800F1340622F0A3
:1057700001022A602B606B60AB608279C0F8C43094
:1057800080F8B830C0F8BC30C364C0F8C03043659E
:10579000C0F8A030C0F8A4309302816303F48053B2
:1057A0004179C363130303F400530364130203F446
:1057B00080634364C36D01F00200C90745D400282B
:1057C0007ED1A06412F0080254D0D4F8BC20002A84
:1057D00000F08A802422C4F8BC202A6822F001024A
:1057E0002A60002B7CD13046FCF7C8FD012812D07E
:1057F0006B68304623F490436B60AB6823F0220360
:10580000AB60AB6843F00803AB602B6843F0010367
:105810002B6079F009FB6279D6070DD5D4F8C83032
:10582000196841F480711960996841F0010199602B
:10583000196841F020011960950705D5D4F8C820F2
:10584000136843F08003136070BD0421A16470B33A
:105850000C21D007A164B5D54FF4803143F0020389
:10586000616643F001034FF40031E365216612F0F5
:105870000802AAD1D4F8BC1009B194F8B82084F871
:10588000B8202422C4F8BC202A6822F001022A6031
:1058900013BB3046FCF772FD0128BCD06B68304664
:1058A00023F490436B60AB6823F02A03ACE7D10785
:1058B00088D543F002034FF48031E365616681E7E8
:1058C0000821A164D1077FF57DAF43F001034FF4B8
:1058D0000031E3652166CAE73046FBF76DFBD8E788
:1058E0003046FBF769FB7EE784F8B82072E700BF1B
:1058F000816031E741712FE781712DE738B5134D94
:1059000041F20D13124941F28832D5F8140AD5F844
:10591000D0490004A060E068014020460B430D21FF
:10592000E360FDF70DFC38B1D5F8042A03460020EA
:105930001343C5F8043A38BD606900F4F050A0F58F
:105940000060B0FA80F0400938BD00BF002E00248E
:10595000C0E0FEFF2DE9F04FA64D7C2200219BB058
:1059600005F51D63184682F0EDFF4FF40031034644
:10597000D5F84C4A4FF48030226819610221C5F8ED
:10598000D409596195F8003AC5F8D029002B00F0E8
:1059900088800422984B85F8002ADA6C1B68D603AD
:1059A0000DD5180100F1D98001224FF0006385F870
:1059B000002AC5F8043A01201BB0BDE8F08F9C0115
:1059C000F2D50AAB18460193FCF7D8FE0B990029D3
:1059D000EAD0D5F8D0490A0A884B6668A3FB0232A0
:1059E000874B884F33401009B94243EA1213636072
:1059F000236843F00303236040F2F6804300824AA9
:105A0000B1FBF3F3B2FBF3F2296802322B685B1AA5
:105A10009A42FBD800237D4A0493A3607C4BE16843
:105A200017680B4043F48053E3607A4BA3FB0737BE
:105A300041F288337F0A03FB07F73B46002B00F057
:105A4000C880626B013B1106F8D5734B704AA363A3
:105A50004FF4D573A360E3681A4041F2081313436F
:105A6000E3604FB13B46626B12F0450F02D09204E7
:105A700040F1DA80013BF6D10023C5F80C3AA3606F
:105A8000634BE268134043F48053E3603B46002BD2
:105A900000F09F80626B013B1106F8D55E4BA3635B
:105AA000E1E05E4B9A425FD05D4B9A4200F00D817F
:105AB00095F8580A0BF018FC834695F85A0A0BF033
:105AC00013FC824695F8500A0BF00EFC814695F8BF
:105AD000520A0BF009FC804695F8540A0BF004FCBE
:105AE000074695F8560A0BF0FFFB95F8592A06462B
:105AF0000E2158460BF0D6FB504695F85B2A0E2136
:105B00000BF0D0FB484695F8512A0E210BF0CAFB4A
:105B1000404695F8532A0E210BF0C4FB95F8552A00
:105B200038460E210BF0BEFB0E2195F8572A304661
:105B30000BF0B8FB0221B4F9040070F0EFFCB4F9EB
:105B40000430002BFFF625AF03F01F0001225B0994
:105B50003449824041F823201BE70AAB18460193E1
:105B6000FCF7D8FA0C9932E7234BD3F8D42022F46F
:105B70008032C3F8D420D3F8D4200243C3F8D42011
:105B8000D3F8D42002400392039ADA6F0243DA6713
:105B9000DA6F22F48032DA678AE72A684FEA134E16
:105BA000A2EB09027346824213D8002B40F03281E7
:105BB000C4F808E0E36803EA0A030B43E3603B46EA
:105BC000626B12F0450F02D0920440F1F180013B6C
:105BD000F6D14FF00040012385F8003AD5F8043A99
:105BE0000343C5F8043AE6E6074AB2FBF1F2296836
:105BF0000BE700BF002E002400440258598B4F01D0
:105C0000002CC0FFFF340C00102101000000002414
:105C1000C0E0FEFFD34D6210C500200000700052AE
:105C20000024024800E100E0636B5B0700F16F8332
:105C3000636BDE0769D4636B580601D54023A36309
:105C40000123704A37212046C5F80C3A0023A3608F
:105C5000E3681A4041F23713134341F28832E3609C
:105C6000FDF76EFA70BB049A4FF6FE739A4200F28B
:105C70003982DFF890A1DFF89881634E002241F26B
:105C8000371337212046A260E26802EA0A02134372
:105C900041F28832E360FDF753FA00289BD1C4F843
:105CA000088041F22913E26802EA0A021343E36022
:105CB00047B13B46626B12F0450F01D0920427D5E5
:105CC000013BF7D14FF0805085E7504BD3F8DC20F3
:105CD00022F40072C3F8DC20D3F8DC2042F4007216
:105CE000C3F8DC20D3F8DC2002F400720292029A9E
:105CF000D3F8842042F40072C3F88420D3F88420BF
:105D000022F40072C3F88420D2E60123A36397E74C
:105D1000636B5B0758D4A6636269049B002A03F196
:105D200001030493049B03DB4FF6FE718B42A5D95C
:105D300004994FF6FE73994200F21782500040F129
:105D4000D4814FF00108D5F80090C5F8088A23687F
:105D5000990700F0C4810023DFF8A8A02046A360C3
:105D600041F20233E26802EA0A021343E360FBF7FE
:105D700081F900287FF42FAF636941F20311C5F860
:105D80003C3AA369C5F8403AE369C5F8443A236A46
:105D9000C5F8483AA060E36803EA0A030B43E360EE
:105DA000002F3FF416AFDFF860C041F2873006E7FE
:105DB000636B5B0722D4636BDE071CD42369DBB201
:105DC000032B06D0012006E704234FF08050A36385
:105DD00001E7C4F838C0636913F4604F3FF4DDAEE7
:105DE000590400F19D8213F4004F0CBF4FF4803032
:105DF0004FF48050EFE60123A363E3E70423184642
:105E0000A363E8E6C0E0FEFFC5002000004402589E
:105E1000000010C14FEA0E49C5F814EAD44A2046E2
:105E2000C4F80890E3681A4041F209331343E36071
:105E3000FBF720F900287FF4CEAE6269C5F82C2A62
:105E4000A369C5F8303AE769C5F8347A216AC5F81C
:105E5000381AD4F818C04FEA1C5CC5F810CA4FEACB
:105E6000927C8DF828C0C2F3836C8DF829C0C2F3F0
:105E7000016C8DF82AC0C2F3074C8DF82BC0C2F319
:105E8000072CD2B28DF82CC08DF82D201A0DADF84C
:105E90002E20C3F303428DF83020C3F3C0328DF8B7
:105EA0003120C3F380328DF83220C3F340328DF8B5
:105EB0003320C3F300328DF834208DF83500B8F16B
:105EC000000F00F01F811B0403F47C1343EA174307
:105ED0000E934FF40073C5F81C3A0E9B01339B02DE
:105EE000C5F8183AC5F8203AC7F380334FF4007A62
:105EF00020468DF84130C7F3C61307F07F07C5F879
:105F000024AA8DF84230CB0F8DF8437001278DF80D
:105F10004430C1F341738DF84530C1F382638DF88D
:105F20004630C1F383538DF84730C1F340538DF8A9
:105F3000483000238DF84930C1F300438DF84A30D2
:105F4000C1F3C0338DF84B30C1F380338DF84C3042
:105F5000C1F340338DF84D30C1F300338DF84E302E
:105F6000C1F381238DF84F30C1F30123C1F3460102
:105F70008DF8503041F207138DF8511007218DF83C
:105F80005270C4F80890DFF8E891E26802EA09026A
:105F9000134341F28832E360FDF7D2F800287FF422
:105FA0001AAEC4F808A041F2101BE36841F288322F
:105FB0001021204603EA090343EA0B03E360FDF7DF
:105FC000BFF8002840F0948095F8003A032B3FF486
:105FD000F2AC2F6863699A017ED44FF0400A41F217
:105FE000883210212046C4F808A0E36803EA0903B8
:105FF00043EA0B03E360FDF7A3F8002843D1D5F88B
:10600000143A372120461B04A36041F23713E2689B
:1060100002EA0902134341F28832E360FDF790F887
:1060200088BB4FF0FF330D216362C4F828A0E36AF8
:1060300023F0FF0343F06303E36241F20D13A0601A
:106040002046E26802EA0902134341F28832E36023
:10605000FDF776F8B8B9019E04E02B68DB1B01332D
:1060600000F08A80636B13F4957F636B40F0878048
:106070001B04F2D506F12002D4F8803046F8043B28
:10608000B242F9D1E9E7D5F8043AC5F8043A394BF8
:106090000122A363D5F8043A18434FF40073C5F8FE
:1060A000040A204685F8002AA36041F21013E16833
:1060B0002F4A0A401021134341F28832E360FDF772
:1060C0003FF800283FF477AC2A4A0123A263C5F8C1
:1060D000040A85F8003A6EE44FF40060D7E74FF009
:1060E000806078E5049A9A423FD84FF000082AE68B
:1060F000204BA363D5F8043A0343C5F8043A85F866
:10610000007A58E440F6FC7202EA830343EA97738C
:106110000E93C7F3C2638DF83C30C7F302638DF86A
:106120003D30C7F342538DF83E30C7F382438DF8BC
:106130003F30C7F3C2338DF8403001230E9A9DF8EB
:1061400040001A4400F00700023082409DF8300001
:1061500000F00F00C5F8182A8340C5F81C3A5B0A06
:1061600002FB03F3C5F8203ABEE64FF0807032E53B
:10617000C0E0FEFFFF0FE01F4FF0004087E7180769
:1061800000F1C880636B990700F1C880636B9A06C1
:1061900008D5C1E0D4F880202B6846F8042BDB1B1F
:1061A0000133E9D0636BDB04F4D40A9B5E4AA2633B
:1061B000C3F381128DF81420C3F340128DF815201B
:1061C0001A0A22F0FF0242EA1362DDE90B1392B2CF
:1061D00009BAADF81620DAB206918DF81C20C3F387
:1061E00007229DF83B108DF81D20C3F303521B0CB2
:1061F0008DF81E200D9A23F0FF03D0B203432046F2
:10620000ADF82030C2F385238DF82230C2F301238C
:106210008DF82330C2F3031302F00F028DF82430FF
:106220004FF400738DF825208DF826101021A360FF
:106230003E4AE3681A4041F21013134341F2883298
:10624000E360FCF77DFF00287FF43EAF9DF824302B
:10625000B8F1010F9DF82520DBB2D2B205D113436E
:1062600014BF4FF400784FF48078D5F8DC09C5F8F6
:10627000288A6FF0A5FF00287FF49DAB2C6803E00F
:106280002B681B1B013330D06FF078FF0428F7D147
:1062900000230121D5F8182AC5F8043AC5F8FC39BD
:1062A00085F8001A002A3FF486AB4FF480406FF067
:1062B00087FF00287FF47FABD5F8083AF3B1012BB4
:1062C0007FF479AB02201A4C85F85C0AA4F1340300
:1062D0000FCB84E80F00A4F1240310340FCB84E823
:1062E0000F0000201BB0BDE8F08F4FF000420123EB
:1062F000C5F8042A85F8003AFFF75DBBD5F80C3ADB
:10630000002BE0D0012B7FF456AB1846DBE70423CB
:10631000A36395E40820BAE62020B8E60220B6E69A
:106320004FF4005057E400BF3A0F0018C0E0FEFFE2
:1063300060380024C74BD3F8601AD3F8642A70B5CC
:106340008C0F93F85C5A100EC2F3072C83F8884A1E
:10635000C1F383640001012D83F8894AC1F301640C
:1063600083F88A4AC1F3074483F88B4AC1F30724B0
:10637000C9B283F88C4AC2F3035483F88D1AA3F888
:106380008E0AC2F3C030B3F88E1A89B241EA040112
:10639000C2F30344A3F88E1AC2F3403183F8904A43
:1063A000C2F3803483F8910A4FF0000083F8924AD8
:1063B00083F8931AC2F3003183F8941AD3F8681A59
:1063C00083F8950A40F2EF80022D00F0C3802A2066
:1063D0004FEA4C0C83F8A14AC1F3C01201F07F01CF
:1063E0000CF07E0C83F8A2CA4FF0010C93F8A24A7D
:1063F0001443D3F86C2A83F8A24AD40F83F8A31A63
:10640000910D83F8A44AC2F3417401F00C01C2F368
:10641000815583F8A54AC2F3826483F8A64A83F8BB
:10642000A71A93F8A71AD3F8704A294383F8A71A32
:10643000C2F3405183F8A81A002183F8A91AC2F3C5
:10644000004183F8AA1AC2F3C03183F8AB1AC2F331
:10645000803183F8AC1AC2F3403183F8AD1AC2F32D
:10646000003183F8AE1AC2F3812183F8AF1AC2F368
:106470000121C2F3460283F8B01AC4F3074183F83E
:10648000B12A220E090283F8B2CA83F8B42AC4F3EF
:106490000722A3F8B61A2406B3F8B61A89B2114334
:1064A000A3F8B61AD3F8741AC3F8B84A0C0ED3F886
:1064B000B82A42EA0442C3F8B82A0A0AD3F8B84A0A
:1064C00002F47F422243C1F30724C9B2C3F8B82AB9
:1064D000D3F8B85AD3F8782A2C43C3F8B84A83F8CB
:1064E000BC1A110E83F8BD1A110C0906C3F8C01AA4
:1064F0001102D3F8C04A0A4601F47F01214392B247
:10650000D3F87C4AC3F8C01AD3F8C01A0A43C3F8B8
:10651000C02AC4F30352D3F8C01A41EA1461C3F885
:10652000C01A93F8C41A1143C4F3072283F8C41A9B
:10653000210A01F47061A3F8C61AB3F8C61A89B229
:106540001143C4F34602A3F8C61A83F8C82A83F895
:10655000C9CA70BD1204C1F3072C0D0E02F47C12DF
:10656000C3F8982AC1F30742D3F8984A44EA0524AD
:10657000C3F8984AD3F8984A22434FF40074C3F8FA
:10658000982AD3F8982AC3F8D84A013240F1000477
:10659000A40244EA92549202C3F8D44AC1F380346C
:1065A000C3F8D02A14E74FEA8C2CC1F3C2659400DB
:1065B0000CF44062C1F3072C04F47F74C3F8982AEA
:1065C000D3F8982A1443CA0BC3F8984A02F006027B
:1065D000D3F8984A44EA9174C3F8984AC1F3026424
:1065E00083F89C5A012583F89D4AC1F3425483F8ED
:1065F0009E4AC1F3824483F89F4AC1F3C03483F8B2
:10660000A02A93F8A02A224383F8A02AD3F8984A14
:1066100093F8A02A93F8906A023205FA02F2B54084
:10662000D617A2FB052EC3F8D85A05FB06EE04FBCD
:106630000EEE0134A2FB0424A644520AC1F38034B6
:1066400042EACE52C3F8D02A4FEA5E22C3F8D42AD7
:10665000BEE600BF002E00246FF0ECBB6FF0EABB7B
:1066600010B51C200AF040FE044611210AF0F8FD86
:10667000204607F07DF9C8200EF07EFC2046BDE8DC
:10668000104007F06FB900BF2DE9F04FDFF8B4B349
:106690008BB0DBF8E0AADAF8143013F0010902D06D
:1066A0000BB0BDE8F08FDAF81420DAF818301A428F
:1066B000F6D0DAF808280AF50061DAF81430C2F3E7
:1066C0000D220291CBF8B42FDAF8182013409D0761
:1066D00005D5DAF8143003F00203CAF81430DAF8FA
:1066E0001430DAF818201340DC061BD5DAF818301D
:1066F00023F01003CAF81830DAF8203003F4F0124F
:1067000003F00F05B2F5802F00F04985B2F5402F58
:1067100000F02583CDF804A0019A936943F010039B
:10672000936101E0CDF804A0019A53699269134086
:10673000180300F19C82019A5369926913405F0328
:1067400000F1D281019B5A699B691A4200F1EA80EB
:10675000019A5369926913401B0509D5029B9B68F6
:10676000DF0700F16485019A536903F40063536104
:1067700001994B698A6913401E0116D54B6903F0D4
:1067800000634B619BF8AC3F002B00F0C282DBF84A
:10679000C03F93F89C22042A04D093F89C22D2B2E2
:1067A00083F89D22042283F89C22019A53699269FE
:1067B0001340DD0400F14881019A53699269134046
:1067C0009C0400F1D780019A53699269134019071C
:1067D00000F1C38001994B698A6913401A067DD480
:1067E0004B698A691340DB0228D59BF8E48AB8F12B
:1067F000010F1ED9924D0AF51267012604E00136F9
:1068000020372435464514D095F83C303A68012BA2
:10681000F5D1002AF3DA66F07F0085F83B30C0B28C
:1068200070F088F9EBE7019A536992691340DA0234
:1068300004D5019A536903F480135361019A536993
:10684000926913409F0231D59BF8E47A012F28D931
:106850000AF532627A4B012103E0B94203F12403C5
:106860001FD093F87C020131146820320128F4D142
:10687000002CF2DADBF8B45F85EA1445EE07ECD4BD
:1068800083F87B02DAF8180040F08000CAF818009C
:10689000DAF814000506E0D4029A536843F4007352
:1068A0005360019A536903F400135361019A5369C9
:1068B000926913405C0000F1BD8001994B698A69BF
:1068C000134058077FF5ECAE4C68610700F1BF84B8
:1068D000DBF8E03A5A6814435C60E1E6DAF8183015
:1068E0009BF8E48A23F08003B8F1010FCAF818304E
:1068F00099D9534D01262F4603E0013624374645EA
:1069000007D097F87B32012BF7D1F0B270F012F973
:10691000F3E7019B5A699B691340DB028ED59BF814
:10692000E48A68E7029A536823F0010353609BF8F6
:10693000AC3F012B00F00182DBF8C03F93F89C22B2
:10694000042A04D193F89D22D2B283F89C22019AA2
:10695000536903F000435361FAE6DBF8C00F90F887
:106960009C32032B00F0ED81019A536903F0080378
:1069700053612FE7019AD2F800396FF30A03C2F886
:10698000003902F50063D2F8042842F480725A609C
:106990009B68980700F1F78113F0060F0CBF0023E6
:1069A0000F238BF8E73AFBF777FB9BF8E76A022E99
:1069B00000F06F844FF410530199003EDBF8C05F84
:1069C000CA6818BF012622F47052CA60CA6813430D
:1069D000CB600123002185F89C32D5F8B83269607C
:1069E000C5F8A41285F8A012C5F894121BB15B6813
:1069F0000BB1284698470022402401274023114626
:106A0000284677F0A5FE2346002280212846C5F8B7
:106A10006041A5F8647177F09BFEDBF8C03FDBF8BE
:106A2000E02AAF842C621E745369019203F4005370
:106A30005361C8E6019A536903F0804353613CE710
:106A4000E0380024002E0024029A10210198536897
:106A500023F001035360FCF715FC9BF8E40AE0B156
:106A60000AF510634FF67F31996009F101091A6840
:106A70002033814522F4001243F8202CC3F8E8119A
:106A8000D3F8E02122F40012C3F8E021D3F8E0218A
:106A900042F00062C3F8E021E6D1029AD36943F0E4
:106AA0000113D3619BF8EF3A002B00F03B81029A6F
:106AB000D2F8843043F00B03C2F88430536C43F0B7
:106AC0000B035364DAF80038019C23F4FE63B44AE4
:106AD0002046CAF800389BF8E61A77F0BBFE6369D7
:106AE00003F48053636167E6019AD2F81878D2F80C
:106AF0001C381F40BFB2002F3FF424AE0AF51061CE
:106B00004FF00008CDF80CA01346A64D44468A4627
:106B1000CDF8109008E07F0804F1010405F1240588
:106B20000AF1200A00F03181FE07F4D5D3F81028CD
:106B300004F00F01D3F834684FEA4419CE40F6014F
:106B4000F6B2164303F5106202EB44129268164047
:106B5000E2B2F007019221D50120029ADBF8C08F42
:106B6000526B00FA01F122EA010202994A639BF892
:106B7000E61ACAF80800814200F078832B6A059370
:106B8000002C40F0FA82D8F89432022B00F0E8830F
:106B900098F8A03213B1002388F8A032320702D54A
:106BA0000823CAF80830F30602D51023CAF80830C3
:106BB000700602D54023CAF80830B10700F11081F1
:106BC0003206DBF8E03AA6D5D5E909068642A2D816
:106BD000811BEA6903F5106E8A42CE4428BF0A463B
:106BE000DEF81810033289B2B1EB920F31D39BF863
:106BF000E68A03F5805C019442460CEB043C98461F
:106C00001346B04240F29083811BEA69914228BF4B
:106C100011462A6A01F103094FEA990973B98CB246
:106C20000334A4080AD002EB840452F8040BA242F5
:106C3000CCF80000F9D12A6AD5E909060A440E44C5
:106C40002A62DEF81820AE6292B29145D9D9019C31
:106C50004346B0423FF65FAF04F00F02012191407E
:106C6000D3F8342822EA0102C3F8342853E7019804
:106C7000D0F81838D0F81C2813405FEA13483FF4C6
:106C80005AAD484B0AF53066CDF80CA000279A465D
:106C9000CDF8149008E05FEA580807F1010706F103
:106CA00020060AF1240A74D018F00109F3D0FBB2CF
:106CB00000F530627D01019302EB47139C68D0F828
:106CC00014180C40E1076FD4210700F19580E50608
:106CD00001D51023B360A0070FD5039B5B6919068C
:106CE00004D5029A536843F4806353609AF857328C
:106CF000012B00F01C830223B360A20601D52023E0
:106D0000B360A30402D54FF40053B360DBF8E00A8C
:106D1000C1E701238BF8AC3F4B6DC3F38303CBF882
:106D2000B03F42E5029942F22B034A6913434B619B
:106D30000B6943F00B030B61C4E600238BF8AC3FF7
:106D400005E6D0F8B832002B3FF40EAEDB69002B1D
:106D50003FF40AAE9847DBF8E03A019304E605EB0E
:106D6000C5020AF58051C3F30A130BEB8202D2F875
:106D7000480D03440868CBF87C0F0968C2F8483D09
:106D8000CBF8801FC6E402230BE6DDE903A90193DB
:106D9000D8E4DDF80CA0DDF814900190CBE400BF3E
:106DA0007C3D0024E03800240121B1609BF8E61A04
:106DB000D0F840E00129D3F808C000F0A582B64918
:106DC0008E4500F09B83DBF8443D3B4300F0498453
:106DD000DAF860220199DBF8C00F77F06DFF73E7F6
:106DE00021460398FCF74EFAEB7D012B00F09183CE
:106DF0000223CAF80830E3E6DBF8E02A0823B36090
:106E000002F53063126C2B4410460492A34A996831
:106E1000904204D90A0402D54FF400429A60DBF88C
:106E2000C05F01219BF87C3F05F2AA2085F8AA32B9
:106E30009BF87DEF079085F8ABE2BBF87E2FA5F8B5
:106E4000AC22BBF880CF0692A5F8AEC2BBF8822F69
:106E5000C5F8941203F01F01A5F8B0220129C5F866
:106E6000982200F0A582022900F00783002940F053
:106E7000DE8203F06003202B00F0E983402B00F05A
:106E8000E683A3B9BEF1090F11D8DFE81EF0E800D0
:106E9000C1001000D80010007D00640010003E000A
:106EA0002300D5F8B4325B69002B40F0C285284638
:106EB00077F092FD794B049A9A427FF608AF9BF8DF
:106EC000E61A01297FF403AF754ADBF8E00A77F090
:106ED000C1FCFCE69DF81890B9F1010F8BF8C49F36
:106EE000E5D895F89C32DAB2022B069200F00385C1
:106EF000032A00F0D784284677F06EFDD5F8B83223
:106F0000494628465B689847D4E7012ACFD195F8CF
:106F10009C120229CBB200F2A684002BC7D0D5F870
:106F2000C832002128464FF0020C40F8081FC5F86F
:106F300094C2C5E90622C3E9092118624FF48072A0
:106F400003F114019A829A79012A08BF186318681C
:106F500077F07CFDAEE7069B00221B0AADF82620E9
:106F6000013B062BA3D801A252F823F04D7104086F
:106F70003171040807710408AF6E0408AF6E04088D
:106F8000A57004085F71040852EA0C0C8FD1069BAF
:106F90007F2B8CD895F89C32032B88D00698D5F897
:106FA000C8325FFA80F985F89E9293F89424012AFA
:106FB00012D01A684FF0000C83F81190D2F8001824
:106FC00021F4FE61C2F80018D2F8001841EA00115D
:106FD000C2F8001883F894C40422002003F11401BD
:106FE000C5F894224FF48072A8619A829A799862C7
:106FF000012AC3E9080008BF1863186877F026FD66
:10700000B9F1000F40F07284012385F89C3251E7FA
:1070100095F89C32013B022B3FF649AF069B012BB2
:107020007FF448AF0020D5F8C832C5F8A402A861A3
:107030000422C5F894229862C3E908007EE7069B03
:10704000012B00F06F84069B022B7FF430AF4FEAD8
:107050001C2CD5F8C832002085F8A0C2E7E795F8C7
:107060009C32013B022B3FF622AF022A7FF41FAF76
:10707000D5F8A4322846002B18BF4FF0030940F87A
:107080000C9FD5F8C832C5F89422C5E90622C3E999
:10709000080200229A6251E70A31544F0A30544FD5
:1070A0007C3D00242B7C002B7FF401AFD5F8B83257
:1070B0000DF126005B6B98470346B5F8B002002837
:1070C00000F03884BDF82620002A3FF4F0AE82425A
:1070D0004FF0020128BF0246D5F8C802C5F8941245
:1070E00000F11401C5E90622C0E9083200228262DB
:1070F0004FF4807282828279012A08BF036300689C
:1071000077F0A4FCD6E69DF8180005283FF6CFAE30
:1071100001A353F820F000BF6B7A04085D7A0408DD
:107120004F7A0408417A0408A36E0408277A0408F9
:107130002A7CD5F8B832002A40F072849B6A0DF19F
:1071400026009847022203464270B6E7D5F8B432CB
:107150000DF12601287C1B6898470346ADE72B7C80
:10716000002B7FF4A4AED5F8B8320DF126001B6BCE
:1071700098470722034642709FE798F89C32032BFA
:107180007FF40CADD8F8B8325B69002B3FF406AD44
:10719000002240460199C8F8D4229847FEE447F6F9
:1071A000F07213423FF4B6AA05EBC502C3F388148C
:1071B0004FEA131CC3F301130BEB8202EE00D2F86B
:1071C000407D002C00F000830AF5805E00223946E5
:1071D0000132DEF80000944241F8040BF8D107EBCD
:1071E0008404002B00F0BC810AF58052234410680F
:1071F000002220FA02F1083204F8011B9C42F8D167
:1072000073190BEB8303D3F8407DDBF8E03A01936D
:107210007319CCF30A0C0BEB83036744D3F8482DA6
:10722000C3F8407D6244C3F8482DFFF775BADBF818
:10723000C03F93F89C22042A04D093F89C22D2B237
:1072400083F89D22042283F89C22FFF78CBADBF896
:10725000C00F0122D0F8B83280F89C22002B3FF4F6
:1072600037AB5B6801799847FFF732BBD5E9070276
:1072700002442A62002C80D1DBF8000BDBF8042BDF
:107280000590002A7FF47FAC1846B74A77F0E2FAFF
:1072900079E4B64BB64A0344934240F25281B54B6F
:1072A000B54A0344934240F25781B44BB44A034475
:1072B000934240F23582B34BB34A03449342C0F049
:1072C0006B82B24BB24A0344934240F29182B14B7B
:1072D000B14A03449342C0F08F82B04BB04A03449A
:1072E0009342FFF467ABAF4BAF4A03449342C0F005
:1072F000D582AE4BAE4A034493422CBF4FF4C053E9
:107300004FF4E053FFF758BB1CF0080F00F01D814D
:10731000A84A96457FF6D8AC1CF4004F3FF4D4AC95
:107320004FF400429A60CFE4019C434694E400236A
:107330008AF85732DBF8C00FD0F8D432AE3350F8A9
:107340002330002B3FF4D7AC90F89C22032A7FF423
:10735000D2AC5B6A002B3FF4CEAC01999847CAE4EB
:10736000D8E90732934200F2278100F0988198F81B
:107370009C32032B00F0C8818021404677F0F0FA60
:1073800005230020C8F89432D8F8C8329A7903F55A
:107390001571C3F86802012AA3F85402C3E99800E2
:1073A00008BFC3F87002186877F050FBFFF7F0BB16
:1073B00003F060025B0602D5402A7FF478AD95F8B1
:1073C0009C32013B022B3FF672AD5FFA8CFCBCF1A4
:1073D000030F3FF66CADD5F8B8329B68002B3FF435
:1073E00069AD4FF0000907992846C5F8D49298472F
:1073F000B5F8B022002A7FF45DAD00287FF45AADC5
:107400000422D5F8C832C5F81890C5F894224FF474
:10741000807203F11401C3F828909A829A79012AA4
:10742000C3E908997FF493ADC3F830908FE51B064C
:10743000D5F8C85200F12D81002385F8553205F5A5
:10744000157301224FF000099A7083F8009095F8A7
:10745000941491423FF42EAD286885F894245A780C
:107460001978069077F042FA069805F29C42A979BD
:1074700077F0F0F985F894941CE503F06003202B75
:1074800000F07C81402B00F07981002B7FF40FAD60
:10749000BEF1010F5FFA8CF100F04681BEF1030FDF
:1074A00000F07E81BEF1000F7FF401AD95F89C32B3
:1074B000022BDAB200F0A481032A7FF4F8AC01F0C9
:1074C0000F0314221CF0800F02FB035340F0B28123
:1074D000B3F86431002B3FF4EAAC02FB015202F531
:1074E000AA70002940F02B8200230360D5F8C8322F
:1074F0000222C5F89422C5E90622C8E51CF4004F13
:107500007FF40EAF1CF0200F3FF462AC20229A6093
:107510005EE40023EB75DBF8C00FD0F8D432AE3355
:1075200050F82330002B3FF463AC90F89C22032AE0
:107530007FF45EAC1B6A002B3FF45AAC019998476C
:1075400056E44FF47053FFF737BA1CF0200F60D0A9
:1075500020229A60FFF7B8BB4FF46053FFF72CBAB4
:10756000CDF804A054E600BF7C3D0024405327FF23
:10757000FF340C00401E1BFF3F420F0000DC0BFFDE
:107580007F4F1200808CF9FE20D6130060B6E5FE16
:107590005FE3160000D3CEFE40771B00C05BB3FE56
:1075A000C091210000CA91FE20753800E05459FEB8
:1075B000E09C41000A30544F9A1AD8F8C832C8E902
:1075C00006225A6203F11401059A1A6200229A6295
:1075D0004FF480729A829A79012A01D10598186332
:1075E0001868CDE9050377F031FA069B00209A79F7
:1075F00003F51571C3F86802012AA3F85402C3E920
:10760000980008BFC3F87002059877F01FFAFFF7DB
:10761000BFBAC64A964503D91CF4004F7FF480AE2A
:107620001A69DAF87432C2F312029B1ACAF8683285
:10763000002F7FF4CDABDBF8442D002A00F0D28080
:10764000DBF8402D1A44CBF8402DFFF7C1BBD5F82D
:10765000D43228460799AE3355F823309B689847B3
:1076600028E4016CB14B994203D91368002BFFF653
:10767000AFAB00231361136943F400231361136953
:1076800043F018031361136943F0C0431361FFF71C
:107690009FBB4FF001036B7505F11403D1E6D8F8D9
:1076A000182093423FF663AED8F898329A42BFF45E
:1076B0005EAED8F8C83200204FF48072C8F81800C7
:1076C00003F114019A829A799862012AC3E90800A9
:1076D00008BF18631868CDE9050377F0B7F9069B72
:1076E0004FF0000C059803F51571C8F898C29A7907
:1076F000C3F868C2012AA3F854C2C3E998CC7FF446
:1077000053AEC3F870C24FE6D8F8B832DB68002B2E
:107710003FF432AE00224046C8F8D42298472BE608
:107720004FF45053FFF748B995F89C32022BDAB268
:107730004CD0032A7FF4BBAB069B002B7FF4BAAB83
:107740004806D5F8C89240F006810422002309F1CA
:107750001401D9F80000C5F894224FF48072AB618F
:10776000A9F8142099F80620C9F82830012AC9E997
:10777000083308BFC9F8303077F068F9D5F8B83267
:1077800000229B68C5F8D422002B3FF493AB0799E5
:1077900028469847FFF78EBB4FF44053FFF70CB9CC
:1077A00095F89C32022B5FFA83FC0FD0BCF1030FDB
:1077B0007FF47DAB480603D0069B134300F0C780DF
:1077C000D5F8C832002032E43C460AE54B0628468C
:1077D0003FF46EAB77F0C4F82846802177F0C0F80C
:1077E000FFF768BB524A012177F034F8FFF7F0BA8F
:1077F0004FF43053FFF7E0B84FF42053FFF7DCB8F5
:107800004A067FF454AB1CF0800FD5F8C8324FF015
:1078100002024FF0000114BF05F1140005F5AA7033
:107820000160C5F89422C5E90622C3E9092118625E
:10783000FFF784BB9B8C002B3FF439AB01F07F0139
:10784000481C00EB800005EB800000293FF44CAEA3
:107850002422D5F8C83202FB01318A7D003A18BFD4
:107860000122026044E6032B7FF421ABD5F8C83235
:107870000221C5E90622C5F8941204355A62002295
:1078800003F114011D629A624FF480729A829A7910
:10789000012A7FF45CAB1D63FFF759BB4FF4005323
:1078A000FFF78AB8B9F1000F00F0AE8069680129CE
:1078B00086D0D5F8B832C9B228465B6898479BF89D
:1078C000C41FD5F8B8326960002B3FF479AF1B684C
:1078D0002846984700283FF473AF284677F07CF895
:1078E000D5F8B832297928465B689847022385F88D
:1078F0009C32FFF7DFBAB9F1000F3FF481AD0121EF
:10790000D5F8B8326960002B5AD01B6828469847D2
:10791000002855D0284677F05FF8069B85F89C3202
:10792000FFF7C8BAC5F8A4324AE700BF0A30544F7F
:107930007C3D0024D5F8C832A861FFF779BB24222A
:10794000D5F8C83202FB013191F8562286E7284665
:1079500077F006F834E701F00F0199F804308B4214
:10796000FFF4F3AE01EBC1031CF0800F4FEA830379
:1079700041D103F51573002209EB030C242303FB0B
:10798000019383F855224FF000038CF800108CF817
:10799000023099F89434012B3FF4D7AE0123D9F883
:1079A000000089F894349CF804309CF801209CF87D
:1079B000001076F075FF4FF0000389F89434C4E6A8
:1079C0000422D5F8C8320020C5F894224FF4807202
:1079D000A86103F114019A829A799862012AC3E995
:1079E000080008BF1863186877F030F8032385F89B
:1079F0009C32FFF75FBA1433012209EB030C2423F6
:107A000003FB01935A75BEE7022349462846C5F891
:107A1000049085F89C32D5F8B8325B689847EFE45B
:107A2000DB6AFFF78CBBD5F8B4329B69002B3FF4BF
:107A30003EAA0DF12601287C98470346FFF73DBB7F
:107A4000D5F8B4321B69002BF3D1FFF730BAD5F863
:107A5000B432DB68002BECD1FFF729BAD5F8B43289
:107A60009B68002BE5D1FFF722BAD5F8B4325B68EA
:107A7000002BDED1FFF71BBA2DE9F0474A4FD7F8AC
:107A8000EC52EE682C69A30701D5B00736D4610724
:107A900001D572072AD4230701D530071ED4E10689
:107AA00001D5F20612D4E30701D5F0073BD414F454
:107AB000025F2BD031066CD4600601D571066ED4FE
:107AC000A20601D5B30629D4BDE8F0876FF01003F4
:107AD0002B610023EA6987F80833E4E76FF00803B5
:107AE0002B610023EA6987F80833D8E76FF00403B5
:107AF0002B610023AA6987F80833CCE76FF00203F3
:107B00002B610023AA6987F80833C0E7E305D3D5C2
:107B10003706D1D56FF480732B61CDE76FF020036A
:107B20002B61BDE8F0876FF001032B611F4B9D4275
:107B3000BDD1D7E9B9839845B9D098BFA3EB08095F
:107B4000D7F8DC321A4A88BFC8F5805907EB83039F
:107B50004244D3F8C832002BA9D0D3F814A2C3F8FA
:107B60000822C3F81092BAF1000FA0D10121C84435
:107B70001048C3F814124B468121C7F8349077F0AF
:107B800075F8B8F5805F14BF43465346C7F8E43232
:107B90008DE76FF40253E2052B618DD5BAE76FF0E4
:107BA00040032B618CE700BF002E0024001400402E
:107BB000C84D0024082E002400207047212808B555
:107BC00023D0222815D0202811D181B1072A0ED127
:107BD000144A154B0868B1F804C012688979186016
:107BE000A3F804C0997112B101460020904700200B
:107BF00008BD0029FBD0022AF9D10C4B1B68002BD1
:107C0000F5D0098800209847F1E70029EFD0072A2E
:107C1000EDD1054B18689A889B79086000208A800E
:107C20008B7108BD3C3100247818002438310024C1
:107C300000207047034B93F82400003818BF012040
:107C4000704700BFE05D0024034B93F82400032835
:107C500094BF002001207047E05D00240048704779
:107C6000085E0024164B002030B493F82A4014B16B
:107C7000DD698D4205D0013010330828F5D130BCC4
:107C80007047104BB2B1196F01EB40218A4201D10C
:107C9000022C08D093F8102212B9012283F8102286
:107CA000012283F8592003EB0013012283F882207C
:107CB00030BC704703EB001383F88220DFE700BF7E
:107CC000385E0024E05D002430B40023194C04F138
:107CD000580084F8FC3003E001331030082B1BD02F
:107CE000C5698D42F8D190F82AC0BCF1030FF3D1D9
:107CF000A2B1216F01EB43218A4208D094F81022EF
:107D000012B9012284F81022012284F8592004EBD0
:107D10000314012384F8823030BC7047D4F8F82073
:107D200004EB03130421013283F88210C4F8F82015
:107D3000F2E700BFE05D0024C0B1836823B10F4BC0
:107D4000072283F85A2070470C4A042192F8580001
:107D500082F86C30032882F85A10C2E9193314BF34
:107D60004FF480738023C2E917337047034B01221D
:107D700083F8102283F85920704700BFE05D00248B
:107D8000244910B54C8991F808C0644531D963463F
:107D90000831E646624603E0944238D991F800E0A3
:107DA0007144724491F801E092B2BEF1050FF3D133
:107DB00091F802E0BEF1810FEED1174A03E0A34231
:107DC0001BD292F800C06244634492F801C09BB297
:107DD000BCF1050FF3D192F802C0BCF1010FEED156
:107DE00019B1002402230C714B710021022311717F
:107DF000537120230380084810BD0029F9D00223C5
:107E000000224B7120230A710380034810BD00211A
:107E1000D3E700BF7818002480180024244910B547
:107E20004C8991F808C0644531D963460831E6466B
:107E3000624603E0944238D991F800E071447244FC
:107E400091F801E092B2BEF1050FF3D191F802E092
:107E5000BEF1810FEED1174A03E0A3421BD292F884
:107E600000C06244634492F801C09BB2BCF1050FAC
:107E7000F3D192F802C0BCF1010FEED119B1002488
:107E800040234C710B710021402351711371202349
:107E90000380084810BD0029F9D0402300220B714F
:107EA00020234A710380034810BD0021D3E700BF9F
:107EB0007818002480180024244910B54C8991F8C2
:107EC00008C0644531D963460831E646624603E09E
:107ED000944238D991F800E07144724491F801E07D
:107EE00092B2BEF1050FF3D191F802E0BEF1810F1D
:107EF000EED1174A03E0A3421BD292F800C06244BD
:107F0000634492F801C09BB2BCF1050FF3D192F823
:107F100002C0BCF1010FEED119B1002440234C7115
:107F20000B710021402351711371202303800848F5
:107F300010BD0029F9D0402300220B7120234A7183
:107F40000380034810BD0021D3E700BF7818002448
:107F50008018002403460A2201481A80704700BF97
:107F6000A0180024D0F8D42200EB82022DE9F041C1
:107F7000D2F8C0420646002C4ED0B4F8643204F168
:107F80001007D4F870520846D2F8C422394603FBD1
:107F900005F5D2F81080B5F5007FD4F86C2228BF23
:107FA0004FF40075B5FBF3F39BB2C04700281BDB11
:107FB0002B463A468121304676F058FEB4F86422CA
:107FC000B5FBF2F2D4E99B1311449B1AD4F8382282
:107FD000521BC4E99B13C4F8382213B10020BDE83A
:107FE000F08103232372F9E7D6F8D432B03356F880
:107FF00023208AB192F861320424112003F1480150
:108000000133DBB202F8314002EBC101A3428880A8
:1080100008BF002382F861324FF0FF30DFE700BF76
:1080200038B5084BD3F8803253B1DB6914460D469E
:1080300098474FF40073026800202A60238038BDFF
:108040001B68FFDEE05D002408B5064BD3F88032E4
:1080500023B11B699847013840B208BD4FF0FF308B
:1080600008BD00BFE05D002400207047002070477D
:10807000704700BF704700BF03685A1C0260197048
:10808000704700BF03685A1C02601970704700BF38
:10809000024BD3F8840203681B681847E05D002494
:1080A0002DE9F0413A4E33787E2B03D00027384635
:1080B000BDE8F08108214FF4FC4341F221041AB2DB
:1080C0005B00002A84EA42009BB2B8BF83B2013948
:1080D000F5D1B6F80140002C37D02E4A2E4DAA42D9
:1080E000E4D2052CA2F106028CBF0027012714441C
:1080F000AC4228BF47F00107002F47D141F2210EC3
:10810000A24214D0501E04F1FF3810F8011F0822BB
:1081100083EA012319B25B0000298EEA410C9BB26D
:10812000B8BF1FFA8CF3013AF4D14045EDD1218854
:1081300061B1A21DAA42BAD2052904EB0100224670
:10814000B5D9A842B3D20446DAE7144C671E41F20F
:108150002105BC4617F8012F83EA0223082219B231
:108160005B00002985EA41009BB2B8BF83B2013AA7
:10817000F5D16445EDD16788094AFF1A231DB7FA86
:1081800087F79B1B7F09A2F8883290E70F468EE79E
:1081900000000208070002080000040801000208AD
:1081A000E05D002410B50B68054A064C13602060A2
:1081B0000BB1002010BD6EF077FD002010BD00BF98
:1081C000042E002440310024F8B51F4FD7F8B02505
:1081D000B7F8B415D7F8803291614BB39B699847D3
:1081E00030B30026D7F8803213B11B69984790B995
:1081F000B6F57A7F24D00CF091FE013604460D4688
:108200000CF08CFE001B61EB0501B0F57A7F71F17B
:108210000001F5D3E6E7B6F57A7F4FF0FF3018BFDF
:108220000020B7F8B435D7F8B0251B049361F8BD2A
:10823000064B03F134025B6BC7F880229847D0E706
:108240004FF0FF30EDE700BFE05D00247818002418
:108250002DE9F84F344E90469A46B6F8C025D6F828
:10826000BC451304A361BAF1000F50D0C8EBC8534A
:10827000C24406F5CC6901EB432B41F28937D6F8AD
:1082800080225AB100235468494640461A46A04706
:10829000A8B9D6F880320BB11B699847013F3AD094
:1082A0000CF03CFE04460D460CF038FE001B61EB62
:1082B0000501B0F57A7F71F10001F5D3DFE741F2F6
:1082C0008937D6F8803213B11B69984780B9013FCE
:1082D00021D00CF023FE04460D460CF01FFE001BBF
:1082E00061EB0501B0F57A7F71F10001F5D3E8E7A4
:1082F0000BEB482008F101084FF4007249467FF06B
:10830000F9F9D045B9D1D6F8BC45B6F8C02500205A
:10831000A261BDE8F88FD6F8BC354FF0FF30B6F853
:10832000C0259A61BDE8F88FE05D00242DE9F84F83
:10833000364E90469A46B6F8C025D6F8BC4513048A
:10834000A361BAF1000F54D0C8EBC853C24406F57C
:10835000CC6901EB432B4FF400720BEB48214846EC
:108360007FF0C8F9D6F880220AB341F2893700239A
:10837000D468494640461A46A047D6F88032B8B17C
:108380000BB11B699847013F37D00CF0C7FD04467D
:108390000D460CF0C3FD001B61EB0501B0F57A7FC3
:1083A00071F10001F5D3D6F88022002ADFD1002335
:1083B00041F2893713B11B69984790B9013F1CD02E
:1083C0000CF0ACFD04460D460CF0A8FD001B61EB63
:1083D0000501B0F57A7F71F10001F5D3D6F880324E
:1083E000E8E708F10108D045B5D1D6F8BC45B6F8A4
:1083F000C0250020A261BDE8F88FD6F8BC354FF04B
:10840000FF30B6F8C0259A61BDE8F88FE05D002422
:1084100010B50E4C236D23B119689A880B691A4266
:1084200008D0FDF797FA28B9237E0133DBB2072B7A
:10843000237603D9002384F8243010BD044A012395
:10844000126884F82430626110BD00BFE05D002432
:108450004431002410B50B4C236D23B119689A8860
:108460000B691A420AD0FDF775FA38B9064B01229A
:1084700020831B6884F82420636110BD002384F8E6
:10848000243010BDE05D00244431002470B5164D49
:108490000021164E6B6C2C681B043162144A0D21AE
:1084A000A3602046E3681A4041F20D13134341F2E2
:1084B0008832E360FAF744FE50B16B6B03436B63A1
:1084C0000C4A09230020126886F82430726170BDBE
:1084D000636903F4F053B3F5006FF1D10423022074
:1084E00086F8243070BD00BFD0370024E05D002442
:1084F000C0E0FEFF4431002470B50C4D04460E462A
:1085000095F82430042B0AD0082B06D1EB6983425E
:108510000AD0FFF7BBFF022801D0012070BD08235D
:10852000C5E9074685F82430022070BDE05D0024CF
:1085300070B57D4C94F824506B1E082B1BD8DFE8D7
:1085400003F06A5E6E1A4605321A2400774B5B6AA6
:10855000002B5ED1764B0722E5681B6884F8242047
:108560006361002D55D023690120D4E90021A8477B
:1085700094F824506B1EDBB2022B44D9042D18BF93
:10858000082D0CBF0120002070BDFDF7B7F90028B1
:1085900040F0BF80664A63691268FA339342EDD2B5
:1085A000FFF736FFC6E7FDF7A9F90028F2D0236AE6
:1085B0000022012B227640F2B080E269013B0821C3
:1085C0000132236284F82410E261012070BD574B10
:1085D0001E6A002E63D1FDF791F9002866D00423AE
:1085E000E568267684F82430002DEED023693046E5
:1085F00022686168A84794F824506B1EBBE76DF0B1
:10860000BDFD04285ED04A4B62691B689B1AC82BCB
:1086100074D8002070BD022384F824308AE7FDF767
:1086200089FE0028EFD1434B0421206293F82C20CF
:1086300084F82410D88D196B84F82E20090E1A6B3B
:10864000A085120C84F82F10196B186B84F8302059
:10865000090A84F8320093F8340093F8352084F83E
:108660003110120984F8330093F8350084F838206B
:10867000996B00F00F00DD8FDA8F6163D98FC2F341
:108680000B1384F8390043EA152301F00F0203F0BD
:108690000F0384F83C2003F5FA6363874AE7244A12
:1086A0006369126864339342BFF468AFFFF7B0FEAA
:1086B000E568002D3FF43EAF002223696168104653
:1086C000A84737E7FDF736FE00289CD11A4B1B78E8
:1086D000002BA3F10203B3FA83F308BF01255B0962
:1086E000A576E376FDF726FE00287FF459AF114BFF
:1086F00003229B6C84F82420A3621BE7FFF788FE0B
:1087000094F82400042818BF08280CBF012000207A
:1087100070BD042384F8243057E7FAD1FFF7B6FE82
:1087200094F824506B1E26E7E05D00246038002496
:1087300044310024883800245C3800242DE9F041BD
:1087400006460D4690461F465D4C94F824100429B9
:1087500005D0082900F088800120BDE8F0810622BC
:108760000123C4F80C8084F82420564A23725362F3
:10877000EB062761C4E9005662D1BFF34F8F524A1E
:1087800005F500712B46C2F8683220338B42FAD1CE
:10879000BFF34F8FBFF36F8F002D00F08A80DFF89B
:1087A000348198F83030012B4AD1731CD8F850101E
:1087B00000228B42C8F834206DD80323D8F800700B
:1087C000C8F81C50182188F830304FF40073FA6252
:1087D0003846C8F82030D8F838303C4A012B4FF0E2
:1087E000FF337B624FF4007318BF7602BB62FB6AF3
:1087F00023F0FF0343F09003FB62FB6843F0400368
:10880000FB609023BD6501253D65C8F82C30BE6036
:10881000FB681A4041F21813134341F28832FB609F
:10882000FAF78EFC00283DD0294B0022BB63D8F814
:1088300034300343C8F8343088F83050C8F82C205E
:10884000637E022B1AD8013363760CF067FB044673
:108850000D460CF063FB001B61EB0501B0F57A7F60
:1088600071F10001F5D377E7E369B3423FF477AFE5
:10887000FFF70CFE02283FF468AF6DE7002666762E
:10888000FFF7C6FDE56825B123693246616801201E
:10889000A847032061E7D8F8343043F00073C8F8E4
:1088A0003430CDE7FB6B607643F48D73FB63BDE83A
:1088B000F081084A536B43F000635363C0E700BF85
:1088C000E05D00246038002400ED00E0C0E0FEFF21
:1088D000FF0FE01FD03700242DE9F84F614F0C4601
:1088E0008046164697F824101D46042908D008290A
:1088F00002D00020BDE8F88FFFF7C8FD0228F8D1AC
:1089000014F01F016AD10122574B58489A60026245
:108910004FF40072C7F860485A60002C00F0948051
:10892000DFF858B19BF83030012B57D108F1010026
:10893000DBF85030CBF83410984200F28B800323E0
:10894000DBF800A04FF001098BF830305046DBF81F
:108950003830CAF82C101121012B4FF0FF33CBE92E
:108960000942CAF824304FF4007314BF4FEA48227A
:108970004246CAF82830DAF82C3023F0FF0343F0DF
:108980009203CAF82C30DAF80C3043F04003CAF8EE
:108990000C308123CAF85840CAF85090CBF82C30DC
:1089A000CAF80820324ADAF80C301A4041F21113A2
:1089B000134341F28832CAF80C30FAF7C1FB034680
:1089C00070B32C4ACAF83820DBF834201343002255
:1089D000CBF834308BF83090CBF82C207B7E022BF8
:1089E00010D801337B760CF099FA04460D460CF052
:1089F00095FA001B61EB0501B0F57A7F71F100017A
:108A0000F5D376E700257D76FFF702FDFC68002CA4
:108A10003FF46FAF3B692A4679682846A04768E76C
:108A200005227B76DAF83C30484687F8242043F468
:108A30009573114AFE60CAF83C3013683D617B6152
:108A4000C7E90048BDE8F88F0C4A536B43F0006358
:108A50005363C3E7DBF8343043F00073CBF83430B2
:108A6000BCE700BFE05D00244066002460380024BD
:108A7000C0E0FEFFFF0FE01F44310024D037002488
:108A8000D0F8D432B03370B550F823402CB3002660
:108A9000124B054684F83C12C4F8303204F50C72CF
:108AA00026720D23812104F5047476F0DFF8D5F8E1
:108AB000C8321F220121C3F88C62A3F8781203F593
:108AC0001E711868C3E9A1429A79012A08BFC3F848
:108AD0009442BDE8704075F0B9BF70BD5553425324
:108AE000D0F8D42200EB82022DE9F041D2F8C04246
:108AF0000646002C67D0B4F8643204F11007D4F8AD
:108B000070520846D2F8C422394603FB05F5D2F864
:108B10001480B5F5007FD4F86C2228BF4FF400759F
:108B2000B5FBF3F39BB2C047002834DBD4F838021E
:108B3000B4F86422401BB5FBF2F5D4E99B13C4F8EA
:108B4000380229445B1BC4E99B13FBB1D6F8C80269
:108B500002FB03F301220021B3F5007FC0F8847209
:108B6000A0F87822827928BF4FF40073C0F88C12E5
:108B700000F51E71012AC0F8883208BFC0F894724F
:108B8000006875F063FF0020BDE8F08119463046AB
:108B9000FFF776FFF7E7D6F8D432B03356F8232044
:108BA0008AB192F861320424032003F148010133B1
:108BB000DBB202F8314002EBC101A342888008BF5A
:108BC000002382F861324FF0FF30DDE7D0F8D43275
:108BD00000EB83032DE9F043D3F8C04283B0002CAF
:108BE00000F0B7801646127805460F465A2A5FD81D
:108BF0005A2A00F29B80DFE812F0470199009900A1
:108C00005B019900990099009900990099009900D9
:108C100099009900990099009900990099008F0195
:108C20009900990099009900990099009900AD0167
:108C3000CE01990099003E01990099009900990090
:108C400011029900370299009900FA0099005F0219
:108C50009900990099009900E20199009900990002
:108C6000990099009900990099009900990099003C
:108C7000990099009900990099009900990099002C
:108C8000990099009900990099009900990099001C
:108C9000990099009900990099009900990099000C
:108CA0009900990099009900990099009900F101A3
:108CB000A82A53D0AA2A00F065829E2A36D1D3F87A
:108CC000C432084604F5197204F51A715B689847B6
:108CD0000146002840F0098394F86232022B00F02C
:108CE0000483D6F80A301ABAE2601BB104F110000E
:108CF0007FF028FED4F868320022013B190E61F3A0
:108D00000702190C61F30F22190A61F31742B4F834
:108D1000641263F31F624BBA63830023626123838F
:108D2000D6F80A301BBAE360002014E094F8612200
:108D3000052620250221531C4832DBB204F832609C
:108D400004EBC200042B858008BF0023617284F805
:108D500061324FF0FF3003B0BDE8F08394F8088033
:108D6000B8F1000F7DD194F91C22002A80F205830E
:108D700094F86222022A00F08083D3F8C4320846B5
:108D80009B689847002840F0DE82D6F80230D5F87C
:108D9000D4121BBAB031C4F86C32D6F8062055F89C
:108DA000211012BAC4F870220029D2D01344D1F88D
:108DB0006802834200F24783B4F8643202FB03F393
:108DC000D4F818229A424AD091F861320524202022
:108DD00003F148020133DBB201F8324001EBC20279
:108DE000042B908008BF002381F86132B1E794F82A
:108DF0000880B8F1000F34D194F91C22002A80F2C7
:108E0000BC8294F86222022A00F03783D3F8C4327D
:108E100038469B689847002840F09582D6F8022093
:108E2000D5F8D41212BAB031C4F86C22B6F80730B3
:108E300055F821105BBA9BB2C4F87032002988D073
:108E40001A44D1F86862B24200F27383B4F8642223
:108E500002FB03F3D4F818229A4240F0E182022385
:108E600023724FF4007339462846E36003B0BDE82F
:108E7000F043FFF777B8337900229B1AE26018BFFE
:108E8000012384F862324FE7D4F81822002A40F018
:108E9000388294F86212022900F04583D3F8C43274
:108EA00038469B689847002840F0D282E0603BE754
:108EB000D4F81832002B00F024827021002294F89C
:108EC000603221740C21C4F81520E17594F8611208
:108ED000C4F811209942C4F81920C4F81D2084F860
:108EE000212011D004EBC30191F84012A17404EBCE
:108EF000C3010133B1F84412DBB2A183042B14BFC8
:108F000084F8603284F860221223E36032799A4256
:108F100098BF1346E36007E7D4F81822002A00F050
:108F2000F0817278D20740F1B081B378002B00F065
:108F3000CE81802B40F0DF810821CC4A04F1180358
:108F400004F11000E16012F8011D03F8011D8342D5
:108F5000F9D1E9E6D3F8C4323846DB6898470028EF
:108F600040F074813279042A134628BF0423E36059
:108F7000002A3FF4D9AE013BBC4A04F1100099B27B
:108F800001F111030A44234412F8011903F8011DE9
:108F90008342F9D1C8E694F862223379012A03F0BA
:108FA000030300F06981012B00F06B81022B00F0BC
:108FB0006981032B00F065810023E360B4E67378D8
:108FC00013F0020340F09781D4E99B210A44D4F8BE
:108FD00068128A4200F2E481E360A5E6D3F8C43265
:108FE0003846DB689847002840F03881337A082BF0
:108FF000194628BF0821E160002B3FF495AE9C4A3A
:1090000001F1100304F110000A4454FA83F312F83A
:10901000011D03F8011D9842F9D185E6D3F8C43249
:109020000DF10202384601A95B689847002840F01C
:109030006E8194F86232022B00F06981BDF8022043
:109040000821206152BA019BA061013B62830C227E
:10905000E174E375190EE2601A0C1B0A2175627542
:109060000222A375227676E6D3F8C43204F519728B
:10907000384604F51A715B689847002840F035813E
:1090800094F86232022B00F03081D4F86832082262
:10909000A082013BE260190E1A0C61F30700190A65
:1090A00062F30F20B4F8642261F3174052BA63F3FD
:1090B0001F60E282206137E694F80890B9F1000F52
:1090C00040F0FF80D4F81822002A00F0898194F93A
:1090D0001C22002AC0F21482D3F8C43238469B689E
:1090E00098478046002840F0F081D5F8D4323846C1
:1090F00005EB8303D3F8C432DB68984701460028A8
:1091000040F08181D6F80220D5F8D40212BAB030EE
:10911000C4F86C22B6F8073055F820005BBA9BB251
:10912000C4F8703200283FF414AE1A44D0F86862D4
:10913000B24200F2C581B4F8642202FB03F3D4F812
:109140001822934240F0EB80B3F5007F4FF001000E
:1091500004F1100428BF4FF4007304F8080C1A46F9
:10916000D5F8C832C3F888229A79C3F88C1203F56F
:109170001E718242C3F88442A3F8780262D1C3F818
:1091800094425FE0227A002A40F09B80D4F81812C3
:10919000002900F0828194F91C120029C0F220817C
:1091A000D3F8C43238469B689847D5F8D4320028A3
:1091B00040F0598105EB83033846D3F8C432DB68AD
:1091C0009847002840F0F180D6F80230D5F8D41244
:1091D0001BBAB031C4F86C32D6F8062055F821100D
:1091E00012BAC4F8702200293FF4B3AD1344D1F889
:1091F0006802834200F22781B4F8643202FB03F371
:10920000D4F8182293427FF4DFADB3F5007F4FF01E
:10921000010104F1100028BF4FF4007321720024F3
:109220001A46D5F8C832C3F888229A79A3F878127A
:1092300003F51E71012AC3F88402C3F88C4208BFEB
:10924000C3F89402186875F001FC6DE5094A92F8BC
:10925000663063F07F0382F8663083E6054A92F851
:109260006B3063F07F0382F86B30BFE6DC180024BC
:10927000E018002478180024022B3CD0012B7FF446
:1092800098AE002384F8623296E6D3F8C43207EB36
:10929000C7013279D86900EB810003790533934225
:1092A00028BF1346E360002B3FF43EAD03F11002EC
:1092B0000344224413F8011D834202F8011DF9D131
:1092C00032E53946284603B0BDE8F04308E40621FC
:1092D0009A4A04F1160304F11000E16012F8011D2E
:1092E00003F8011D8342F9D11EE53A2202212846E6
:1092F00075F060F82DE524220521284675F05AF80E
:1093000027E520220521284675F054F821E5284656
:109310003A22022175F04EF84FF0FF301BE590F82D
:1093200061320525202403F148020133DBB200F845
:10933000325000EBC202042B948014BF80F86132DB
:1093400080F8611205E5D5F8D432B03355F8232002
:10935000002A3FF4FEAC92F8613202243A2003F175
:1093600048010133DBB202F8314002EBC101042BAA
:10937000888075D082F86132EBE494F86132052080
:10938000202103F148020133DBB204F8320004EB80
:10939000C202042B91807FF4DAAC84F86182D8E4B5
:1093A0002122052175F006F8D3E4D5F8D432B03384
:1093B00055F823208AB192F861320225272003F163
:1093C00048010133DBB202F8315002EBC101042B3A
:1093D000888008BF002382F8613205232372B8E435
:1093E00094F861320525202003F148010133DBB2F6
:1093F00004F8315004EBC101042B88807FF4A7AC42
:1094000084F86122A5E4D5F8D432B03355F823208E
:10941000002A3FF49EAC92F86132022427209EE796
:1094200091F861320525202403F148020133DBB2B3
:1094300001F8325001EBC202042B94807FF4D4ACCB
:1094400081F8610285E491F8613205242120BFE4AE
:109450003A220221284674F0ADFF0523237278E4F6
:1094600082F8618275E4B03355F82320002AB4D025
:1094700092F8613202253A20A1E794F8613203F1B3
:1094800048010133DBB204F8312004EBC1013A2278
:10949000042B8A807FF45BAC7FE794F8613205256A
:1094A000202003F148020133DBB204F8325004EB10
:1094B000C202042B90807FF44AAC84F8611248E425
:1094C00090F86132052521242DE7D5F8D432B03348
:1094D00055F82320002A3FF43CAC92F86132022474
:1094E0003A2003F148010133DBB202F8314002EBCC
:1094F000C101042B88807FF43DAF82F8619228E49B
:1095000094F861320520202103F148020133DBB2D7
:1095100004F8320004EBC202042B91807FF417ACF4
:1095200084F8619215E43A2274F044FF0523237213
:109530000FE491F861320525212475E7D218002443
:10954000D0F8D432B03350F82330CBB110B51A7AFA
:10955000022A07D0033A012A02D80021FFF790FA25
:10956000002010BD03F21F2293F81D120446FFF7DE
:109570002DFB0028F4DA01212046FFF781FAEFE7FE
:10958000002070472DE9F04104464FF41D707FF034
:1095900009F9054600285BD0D4F8D47204EB87079C
:1095A000C7F8C002237CC4F8BC02002B45D040237E
:1095B00002220121204675F0CBF8012240234FF012
:1095C00001082046A4F8782181210222002675F0A6
:1095D000BFF8A4F83880D7F8C43230462E81A5F8F9
:1095E000606285F862621B689847D4F8C84294F8B4
:1095F00094342768434508D03846F9F76BFE414656
:109600003846F9F73FFE84F8946405F504751F2287
:109610000023384604F51E71C4F88C320123C4E9D6
:10962000A152A279A4F878329A4208BFC4F89452A1
:1096300075F00CFA0020BDE8F0814FF400730222AF
:109640000121204675F084F801224FF40073B6E73B
:10965000D4F8D4320220B03344F82350EBE700BFF3
:10966000F8B5D0F8C85201260446002295F8943483
:10967000A5F87862B34227D03146286885F894640B
:10968000002775F073FB40F20113A4F8787132469D
:109690003146286885F894642B8775F067FB85F858
:1096A0009474D4F8D4320025B033258754F82300BD
:1096B00040B17FF07FF8D4F8D432B03344F823506F
:1096C000C4F8BC520020F8BD40F20113A0F8782184
:1096D0002B87E6E738B5D0F8D432B03350F82350B2
:1096E0007DB195F81C32044623B9D5F818320BB178
:1096F0006B7A8BB18121204675F032F96B7A022B9F
:1097000000D038BD2046812175F02AF9204601217C
:10971000BDE8384075F024B9012175F021F92046E3
:109720008121BDE8384075F01BB900BFD0F8D432B4
:10973000B03370B550F8235025B12B7A044683B16D
:10974000012B01D0002070BD05F21F2295F81D12DB
:10975000FFF73CFA0028F5DA01212046FFF790F9DF
:10976000F0E7D5E98523C5F83832D0F8C832C5F816
:109770003422D3F88C321F2B04D12F4BD5F8102272
:109780009A421AD095F861324FF0050C20212046FC
:1097900003F148020133DBB205F832C005EBC20227
:1097A000042B91804FF0020208BF00236A7285F8F3
:1097B0006132FFF78FFF002070BD95F81D1201295F
:1097C000E0D895F81E32013B0F2BDBD805F21F22A3
:1097D000FFF7FCF900282B7A22DB013B022BB1D9E1
:1097E000EE681EB3D4F8D432B03354F823100029F5
:1097F000A8D02046D1F83842D1F8183205F110022D
:10980000A41BB342C1F838424FF0000428BF3346CE
:1098100081F83C4204240C72812175F027FA91E70B
:10982000052B99D02046FFF755FF8BE731462046A0
:10983000FFF726F986E700BF55534243F0B50023F2
:1098400083B0ADF80630D0F8D43200EB8303D3F800
:10985000C0524DB10A78044612F0600036D020287C
:1098600005D0204675F0B8F8032003B0F0BD487865
:10987000FE2849D0FF28F4D14B88002BF1D1CE88A7
:10988000002EEED11006ECD44FF4807381212B8191
:1098900005F50475D4F8C842204676F00DFB204645
:1098A000012176F009FB1F22012304F51E712068B7
:1098B000C4F88452A4F87832C4E9A226A2799A4264
:1098C00008BFC4F8945275F0C1F846E04B780B2BF2
:1098D000C7D801A252F823F05F990408CF99040871
:1098E000639804086398040863980408639804085C
:1098F000639804086398040863980408639804084C
:10990000979904084F9904084E88002EA9D1CF8852
:10991000012FA6D11206A4D5D3F8C4329B6998476B
:10992000022328604FF48071C4F89432D4F8C8320E
:10993000C4E906779A79998203F11401012A5F62DA
:109940001D629E6241D0186875F080F805E094F8B9
:109950009C32032B85D18B786B60002085E794F8CF
:109960009C32032B7FF47DAF0222D4F8C832002052
:10997000C4F8942203F11401C4E906220DF106048F
:109980009862C3E908424FF480729A829A79012A58
:10999000D9D11C63D7E794F89C32032B7FF461AFD5
:1099A000D4F8C8320122022104350020C4F89412F0
:1099B0004FF48071C4E90622C3E908529A7999826A
:1099C00003F11401012A9862BDD11D63BBE794F82D
:1099D0009C32032BC1D14B88002BBED1D4F8C86276
:1099E0008F8896F89434012B0AD001233906306809
:1099F00086F8943410D4F9F76DFC002386F894347B
:109A00006B7A022B0DD03A06A7D5012BA5D00121E8
:109A10002046FFF735F8A0E707F00F01F9F732FC11
:109A2000EBE72046812174F09BFF0121204674F072
:109A300097FF92E72DE9F8430D46D0E90031134432
:109A40008B4220D80446AE18076BCAB14FF000090C
:109A500000F10C0801E0AE4212D0E36A5A1C234424
:109A6000E262202A15F8011B1973F4D14146204601
:109A700017B9F9F77BFC0746AE42C4E90B97ECD166
:109A80003846BDE8F8834FF0FF37F9E72DE9F84F86
:109A9000234B81468A46D3F8BC32D3F81422002ADD
:109AA000FBD1BAF1000F37D009EB0A031D4E09F1C3
:109AB000FF39DFF8788003F1FF3B7027326819F82F
:109AC000011F531C1848C3F30B0381543360EFF399
:109AD000118287F31288D8F80030D2B2316882F34D
:109AE00011888B42A3EB01038CBF0022012203EB00
:109AF0000233012B0ED10BF011FA04460D460BF088
:109B00000DFA001B61EB0501B0F57A7F71F10001E0
:109B1000F5D3DCE7D945D1D15046BDE8F88F00BF79
:109B2000082E0024E8300024C84D0024E43000242E
:109B300002784368022A0FD00B490269D1F87402F7
:109B4000023A184010B4400AD1E99A1404FB02000A
:109B50005DF8044B08447047034AD2E9972102EBB1
:109B6000410202EB53207047E05D00242DE9F04FE5
:109B700083B002F00207834D019308B9002F6AD128
:109B8000D5F86442002C53D14FF0FF3E7E4C4FF08D
:109B9000000CF146F046F246E36994F82A609842D8
:109BA00000F0A080002E3BD0012E05EB0C1B0AD14B
:109BB0009BF88360F30706D416F07E0F03D1F609F5
:109BC00000F09380E0460CF1010C1034BCF1080F5A
:109BD000E2D1BEF1000F04DAB8F1000FC0F29780B5
:109BE000C646D5F8F4400EF1020605EB0E18013416
:109BF00005EB061CC5F8F4400CF1580CCCF80440F9
:109C0000C8E91D040024CCF8084005EB061494F8BC
:109C10006240042C1FD8DFE804F029441A444600AF
:109C2000E6460CF1010C1034BCF1080FB4D1D0E7BA
:109C3000D5E99A3606FB0434A042A5D395F8103234
:109C400013B9012385F81032012385F8593000201B
:109C500003B0BDE8F08F95F81032002B53D00123EC
:109C6000022085F8593003B0BDE8F08F12F00104EE
:109C7000D5F870C072D105EB0610019B4FEAE20CDB
:109C800090F86380032B6CF3C71880F8638063D966
:109C90004FF6FF70834228BF034605EB0610A0F87D
:109CA0006030002F45D1500707D505EB061090F81E
:109CB000633043F0010380F86330D3060AD505EB27
:109CC000061696F86330C3F34502013262F3460389
:109CD00086F863302B6F012003EB4E230B6003B03B
:109CE000BDE8F08FC6B9E6467BE7666A1034B24538
:109CF00088BFE1460CF1010C88BFB246BCF1080FE9
:109D00007FF44AAF65E7012385F81032A7E7B9F180
:109D1000000F9CDBCE4664E7D5F8F4400CF1020658
:109D2000E646013405EB061CC5F8F440CCF85C406F
:109D30006BE7D5F8F800D5F8F43001300133C5F8F9
:109D4000F80005EB0E10C5F8F430836705EB061339
:109D5000042083F86200A6E723469EE7D5F8803208
:109D6000002B3FF474AF5C680CEB4E210023074AD4
:109D7000A04700283FF46BAF05EB0616022386F8D8
:109D8000623064E7E05D0024385E0024657C0408EE
:109D900070B5114D82B00E4695F85830022B16D191
:109DA000020AC4B2D5F85C02002301A910440322C0
:109DB000FFF7DCFE012808D195F85830019A022BF4
:109DC0000CBF22F8146042F8246002B070BDC0F3EA
:109DD000D41200F07F04E5E7E05D00242DE9F04FA8
:109DE000444E0D4683B0174696F858102B68032949
:109DF0003ED0022961D14FEA13294FF4807A5FFAED
:109E000083F8421E012A23D84FF0010B9F421AD932
:109E100001288CBF00240124D6F8D4211AB1D6F829
:109E2000F01199424CD0D6F85C020023092201A916
:109E30004844FFF79BFE012823D0022814D020B10C
:109E40002B689F42E8D803202F6003B0BDE8F08F55
:109E5000B8F1000F13D096F8103213B9012386F829
:109E60001032012386F85930022003B0BDE8F08F8C
:109E70004FF0800AC3F3D41903F07F08C1E7D3463B
:109E8000C4E796F85810022913D00329ECD1019B9E
:109E900053F8282022F07042B2FA82F22B6852095D
:109EA000A2421FD0D8445B44D0452B601DD202296A
:109EB000EDD1019B33F81820EEE74FF4807AD9E713
:109EC000D6F86C12013A02EB41224902B2FBF1F2E0
:109ED0001344B3FBFBF20BFB12320AB15B449B1A37
:109EE0002B60AEE79F42B0D8ADE709F101094FF012
:109EF0000008A6E7E05D00242DE9F04FDFF884912B
:109F00008B4685B0174699F858C00968BCF1020F16
:109F1000D9F85C5240F08280CEB24FF4807305EBEA
:109F20001125A6EB010890449844B94208F1FF3886
:109F3000B8FBF3F84AD200F00103A8446FF0404A9E
:109F40000193BCF1030F07EB0604A8EB05032846B9
:109F500014BF4FF480728022641A03A9944228BF70
:109F60001446944228BF002E14BF012200220A3258
:109F7000FFF7FCFD01282AD199F858C0DBF800E072
:109F8000BCF1020F0EF1010324D0B44255D903985D
:109F900006EB0A02011F00EB820201EB840142F88A
:109FA000043F8A4203F10103F9D1DBF80030A11B21
:109FB00019448F42CBF8001002D1019B002B48D1ED
:109FC0008F4205F101054FF00006BAD8012005B017
:109FD000BDE8F08FB44246D903986FF00042811E6D
:109FE000324401EB440100EB420222F8023F91426D
:109FF00003F10103F9D1A11B71448F42CBF800108A
:10A00000DED1019B002BDBD086466FF000434FF67C
:10A01000FF72012023442EF81320D8E701F07F06B9
:10A02000C1F3D413BCF1030FA6EB01081D4414BF08
:10A030004FF480738023904476E7AEEB060E0EEB70
:10A0400004018F42CBF80010BAD1019B002BB7D08E
:10A0500003986FF040434FF0FF32234440F8232031
:10A06000DBF80010ACE7AEEB060E0EEB04018F42FE
:10A07000CBF80010A4D1019B002BA1D0DDF80CE09F
:10A08000C3E700BFE05D002430B50446C06983B07B
:10A0900010B9012003B030BD0D460023032201A9F1
:10A0A000FFF764FD0128F5D1B4F92020002A19DB5F
:10A0B000019B012D4FEA421103EB421203D0022D06
:10A0C0001BD1E5205854A368D3612378032B04D116
:10A0D0000023137753779377D377636A190C5383ED
:10A0E0009182D6E7064A92F8101209B982F8100256
:10A0F0000123022082F85930CCE7E368E4E700BF8F
:10A10000E05D00242DE9F041044682B00D4694F84C
:10A110003C30042B7ED8DFE803F02B0369493A007A
:10A120003D4E4FF6F777DFF8F48016E0BA425BD881
:10A130006BF0D2FC01284FF0000134D1206BFFF707
:10A1400027FE01282FD1019AD6F87012531E2263E0
:10A150008B4228BF0B46C6F8703296F8582001A9EA
:10A16000236B032A18469AB2E0D14345E0D93BE07D
:10A170006900204601F0FE01FFF786FF01283FD16C
:10A18000636B002B18BF022084F83C00BFE794F8F3
:10A190002830042B02D1002384F82830A36B0BB1A4
:10A1A00020469847012002B0BDE8F0811A4E0021F8
:10A1B000E26AD6F8F03106F5E670C6F8F0219B1A8F
:10A1C000D6F86C2202FB03F3D6F8D42102EB43222B
:10A1D000C6F8D421D6F8D82102EB4322C6F8D821FC
:10A1E000FFF752FF01280BD10420CDE7626B04F189
:10A1F00030010020FFF780FE012801D10320C3E7D2
:10A200000228D0D194F82830042BCCD1002384F834
:10A210002830C8E70220F5E7E05D0024F7FFFF0FD4
:10A2200038B5044694F83430052B60D8DFE803F0E5
:10A2300031251D130D0394F82830082B3FD02D4BEA
:10A240000122022083F8112238BD94F82830082B0F
:10A2500030D0012038BD00212046FFF715FF01282E
:10A2600045D1042084F83400DCE7D4E90B01FFF782
:10A270008FFD01283BD10320F4E74FF0FF31206B25
:10A28000FFF786FD012832D1E36A002BF3D00220CC
:10A29000E8E7184D04F130010120D5F864220232BC
:10A2A000FFF79CFD012813D00238C0B201281ED848
:10A2B0000520D7E70023012084F82830CAE70023CF
:10A2C0000122022084F828300A4B83F81122BBE7D0
:10A2D000E368D5F86C12226B03EB4123C5F87022BA
:10A2E000C4E90332E36A002BBCD16262BAE7002002
:10A2F00038BD00BFE05D0024F8B5044694F838305E
:10A30000032B4CD8DFE803F021180B020021204674
:10A31000FFF7BAFE431EDBB2012B41D9F8BD012085
:10A32000626B04F13001FFF7E7FD01284FF00303F2
:10A33000F0D184F83830E1E700211E48FFF7A4FE91
:10A3400001284FF00203F4D0E4E71B4BE66893F8D2
:10A350005820D3F86C12032AD3F8D451D3F8F00163
:10A3600014BF4FF480728022206102FB01F1871A32
:10A370000244A5EB412506EB4126E660C3F8D45123
:10A38000D3F8D851C3F8F021A5EB4121C3F8D81177
:10A39000E36AC4E90C025BB960620123C9E70220E9
:10A3A00094F82830062BB9D1002384F82830F8BD62
:10A3B0002763F2E7AC5F0024E05D00244368C3F349
:10A3C00008020A44B2F5007F2DE9F041054682B04B
:10A3D0000C4605D223446B60012002B0BDE8F08139
:10A3E00090F91A10481C0AD0474A02EB011292F861
:10A3F000831021F0010182F88310FF22AA7695F9DB
:10A400001B20511C16D0404E023206EB021191F86F
:10A410006310C1F34501012944D9013901F03F011D
:10A4200006EB0212FF2692F8630061F3460082F801
:10A430006300EE762A78022ACCD0334ED6F86C220E
:10A44000B4EB422F4FEA42282EDCD6F874721F403C
:10A450007A42A24228DCE2192869424513D32A7EB7
:10A4600012072DD5D6F8F021411C8A421ED300D107
:10A4700000214344A4EB080868610846DB1B08EB95
:10A48000070429616B600028A6D096F85820032A9B
:10A4900035D080B24FF6F77290429DD81A461444D8
:10A4A0006C6099E70021BBE7002096E796F8102240
:10A4B0000ABB012386F8103286F859306B68D8E75A
:10A4C00001A96BF009FB0128EED16B68A4EB08042D
:10A4D00028699844297868613C44A8EB07030198EF
:10A4E00002291A466B602861CDD1D6F87C12B3EBF5
:10A4F000412FD4D370E7012286F85920B9E7034AE7
:10A5000090423FF669AFC9E7E05D0024F7FFFF0F17
:10A510002DE9F0474FF0010882B0044694F8383036
:10A52000032B00F2A680DFE803F055170C02002091
:10A53000236C84F8280003B19847022002B0BDE8DC
:10A54000F0870022236C84F828200BB1204698471E
:10A55000012002B0BDE8F08723786768022B03D0A2
:10A56000454BD3F874321F40C7F34F272046FFF7FF
:10A57000DFFA414E3F1A0546BFB207EB050C022237
:10A5800001A9002328461FFA8CF9FFF7EFFA0128EA
:10A590004FF400724FF00001D0D101987EF0D2F953
:10A5A000E3694FF4007120460BB16368EBB1D6F854
:10A5B0006C325A1E914547D20135FFF7FFFE002845
:10A5C000DBD196F8103213B9012386F8103286F8E1
:10A5D0005980D2E72046FFF723FE012802D0022847
:10A5E00047D1032084F8380098E7019B4FF02032D0
:10A5F0004FF0100E4FF02E0C42F62E6AC3F80120D9
:10A60000C3F80520A3F8092083F800C0D4F824C0BB
:10A61000A3F820A083F80BE0C3F82220C3F826207B
:10A6200083F82A20E26BA3F81AC02CFA0EFC5A8792
:10A6300022FA0EF2A3F814C09A8683F82BE0D6F81B
:10A640006C325A1E9145B7D3C3EBC353204659020F
:10A6500001F50071FFF7B2FE28B996F8103223B168
:10A66000012386F859300220BCE7012386F8103216
:10A67000F6E7002062E700BFE05D0024B1F9043096
:10A680000F2B2DE9F0410D4682B00446164632D01C
:10A690002046FFF74DFA94F91B80B8F1FF3F3BD0FD
:10A6A0005B4F07EB08135B6F984212D097F810329C
:10A6B000002B6ED0012387F859302378022B5ED00F
:10A6C0002269002A73D100230120336002B0BDE863
:10A6D000F081396F01EB4821002966D0AB88204614
:10A6E00001331BB201EB4311AB803160FFF720FA5D
:10A6F00028600120EAE74FF40071FFF75FFE0028B1
:10A7000043D04FF6FF732046AB80FFF711FA94F960
:10A710001B80B8F1FF3FC3D12378022B3DD02269C3
:10A72000002AD0D03A4F97F85830032B66D093B216
:10A730004FF6F7718B4294BF00230123002BC0D149
:10A7400030B997F81032002B4BD0012387F85930DD
:10A750000023112201A9FFF709FA012825D1019947
:10A760003B6FCB1A48BF03F2FF13B3F5805F4FEA8C
:10A7700063222CD24FFA82F884F81B80ACE7D7F81A
:10A780007C226368B3EB422F9DD2002002B0BDE86B
:10A79000F081012387F810328CE71D4F6368D7F8EA
:10A7A0007C22B3EB422FCBD38DE7237886E797F853
:10A7B0005830032B19D093B24FF6F772934294BFDF
:10A7C00000230123002B7FF47EAF0020DEE797F803
:10A7D000103213B9012387F81032012387F859305A
:10A7E000CAE7012387F81032AFE70A4B9A4294BFB9
:10A7F00000230123002B7FF466AFE6E7054B9A4266
:10A8000094BF00230123002B7FF45BAF98E700BFC8
:10A81000E05D0024F7FFFF0F10B50378044690F8C1
:10A8200018C0023B012B02D91CF0060F6ED11CF0A0
:10A83000200F44D194F91A20511C0AD03A4BFF2121
:10A8400003EB021393F8832022F0010283F88320A4
:10A85000A17694F91B305A1C16D03349023301EB10
:10A86000031292F86320C2F34502012A4BD9013A40
:10A8700002F03F0201EB031393F8631062F3460109
:10A88000FF2283F86310E2761CF0080F0ED02649F1
:10A8900091F8F431072B06D091F81032002B3DD0FF
:10A8A000012381F85930002381F8F4310023E26A52
:10A8B000237084F8283042B3BDE8104010471B4A8B
:10A8C0000023E069D1691032884206D00133082B99
:10A8D000B0D0D16910328842F8D11349023301EB6C
:10A8E000031292F86320C2F34502012A1AD9013AF1
:10A8F00002F03F0201EB031393F8631062F3460189
:10A9000083F8631096E70022B4E710BD0121FFF73A
:10A91000BBFB0128F9D194F818C088E7012381F81E
:10A920001032BDE70022E5E7E05D0024385E002438
:10A9300038B51A4C94F83C322BB970B190F82820F5
:10A940001AB1184638BD002038BD0146442204F52E
:10A9500005707CF0CFFE012038BD04F50575014679
:10A96000442228467DF0EEFF94F8583003224FF63B
:10A97000FF71022B2846A4F82E1218BF1346D4F8F4
:10A98000781284F82C22102284F81432C4F8381279
:10A9900084F82D226CF0A4FBDDE700BFE05D00240D
:10A9A000304A4FF0FF31F8B5A2F1580C00230C46A5
:10A9B00003E001331032082B14D092F82A00042847
:10A9C000F7D10CEB031090F88300C607F1D4651C97
:10A9D000106A01D08142ECD91C4601330146103285
:10A9E000082BEAD1002C01DA0120F8BD1E4DA61C6F
:10A9F00005EB0613D5F88022B3F86010D9B927010A
:10AA00002F44296FD5F88032786F01EB4421D3B100
:10AA1000DC680023154AA047A8B1022809D1D5F85F
:10AA2000F83005EB06160122013B86F86220C5F8D6
:10AA3000F8300020F8BD05EB04132701586F12B160
:10AA400093689847DCE7D5F8F83005EB0616032144
:10AA50000122013B86F8621085F8FC20C5F8F83029
:10AA6000E7E700BF385E0024E05D0024C97C0408ED
:10AA7000704700BF0369416853EA0102F0B43B4EDE
:10AA80005DD0C56A013390ED067A6A1C876830EEA6
:10AA9000077A0361012AC26280ED067A42D090ED06
:10AAA000075A07EE902AD0ED096A70EE455A3468CD
:10AAB000B8EEE76A611AC5EE867AB94277EE857A12
:10AAC00030EE670AC0ED087AC0ED077AF0EE667ADC
:10AAD000E5EE807AC0ED0A7AC0ED097A01D8F0BCC3
:10AAE0007047012A28DD06EE905AF8EEE66A87EEF6
:10AAF000A66AB5EEC06AF1EE10FA1DDBF1EEC67A79
:10AB0000F4EE677AF1EE10FA16D6D0ED056AF4EE9F
:10AB1000E76AF1EE10FA15D5037BFBB10323F0BC15
:10AB200003707047326880ED080A521A002180EDE8
:10AB3000070ABA424162D2D9DFED0D7AE5E7316802
:10AB400041609EE707EE903A0223F8EE677A0370C1
:10AB5000F0BCC7EE276AC0ED066A70473168002274
:10AB60000361C36241608261B9E700BF44310024E0
:10AB70000000000010B5DFED4F4A844600F1480E9A
:10AB80000346DA6AB1EC017AD3ED067A013277EE48
:10AB9000877A012ADA62C3ED067A71D093ED075AFB
:10ABA00007EE902A93ED096A77EE455AF8EEE77AB8
:10ABB000C5EEA76A76EE857AF0EE466A37EE677ADA
:10ABC000C3ED087AE5EE876AC3ED0A6AC3ED077A3A
:10ABD0001833C3ED036A7345D3D1374C41682268FB
:10ABE0000369521A816801338A42036147D990EDA3
:10ABF000056A0022DFED2F5ADCF82C10F0EE657AA2
:10AC0000DCED0A6A012901F1FF3E11DD07EE90EA51
:10AC1000F8EEE77A86EEA77AB5EEC07AF1EE10FA92
:10AC200045DBF1EEC77AF4EE677AF1EE10FA3ED624
:10AC3000B4EEE76A01320CF1180CF1EE10FA26D4EA
:10AC4000022AD9DDB4EEE76AF1EE10FA1FD407EE5E
:10AC5000903AD0ED066A90ED0C7A0223F8EE677A0E
:10AC6000D0ED125A037086EEA76AC7EE276A85EE0A
:10AC7000A77A80ED066AC0ED0C6A80ED127A10BDED
:10AC8000F0EE477A83ED087AF0EE646A9EE7037B84
:10AC900013B10323037010BD002221680361C36256
:10ACA00041608261026343648264C36510BDDFED6D
:10ACB000017ABDE70000000044310024B0EEC06A14
:10ACC000F0EEE05AF0EE407AF4EEC65AF1EE10FAE9
:10ACD0000EDCB5EE400AF1EE10FA4AD0F4EEC65A98
:10ACE000F0EE466AF1EE10FA4FD5B0EE655A03E089
:10ACF000F0EE656AB0EE465A85EE267A9FED242A7C
:10AD00009FED243A9FED244ADFED244ADFED242A0B
:10AD1000DFED243AB7EE005ADFED236AF4EEC65AAF
:10AD2000F1EE10FAA7EE023AE7EE223AA7EE034A56
:10AD3000A7EE235AE7EE044AE7EE246AB1EE667AFC
:10AD400087EE050A10D4F5EEC00AF1EE10FA03D52D
:10AD50009FED167A37EE400AF5EEC07AF1EE10FA62
:10AD600048BFB1EE400A70479FED117A37EE400AB6
:10AD7000E9E7F5EEC00ADFED0F7A9FED0F0AF1EE7D
:10AD800010FA58BFB0EE670A7047B0EE465AB3E704
:10AD900039094E3DE3B59EBE88FA16BE45FE7FBF1B
:10ADA00099FB243F69A2163EA7DFA8B4DB0F4940F8
:10ADB000DB0FC93FA7DFA834DA0F4940D1ED007A95
:10ADC000F7EE002AD0ED043A90ED054AE7EEA73AF7
:10ADD000D0ED064A90ED075AD0ED085A90ED096A79
:10ADE000D0ED0A6A90ED0B7AC0ED043A91ED003A8D
:10ADF000D1ED013AD0ED0C7AA3EE234A80ED054A5D
:10AE0000D1ED003A91ED024AE3EE844AC0ED064AE4
:10AE1000D1ED004A35EE245A80ED075AD1ED014AB2
:10AE200091ED005AE4EE855AC0ED085AD1ED015A71
:10AE3000A5EEA56A80ED096AD1ED015A91ED026A8D
:10AE4000E5EE866AC0ED0A6AD1ED016A37EE267A30
:10AE500080ED0B7AD1ED026A91ED007AE6EE877A09
:10AE6000C0ED0C7A91ED027AD1ED017A90ED0D3AB8
:10AE7000D0ED0E3AA7EE273A90ED0F4AD0ED104AEA
:10AE800090ED115AD0ED127AD0ED135A90ED006A80
:10AE900080ED0D3A75EEA25A91ED023AD0ED016ABD
:10AEA000E3EE033A90ED027AC0ED0E3AD1ED023AAC
:10AEB00034EE234A80ED0F4A91ED004A74EE844A45
:10AEC000C0ED104AD1ED014A35EE245A80ED115AF9
:10AED00091ED025AC0ED135A77EE857AC0ED127AE1
:10AEE000D1ED017AD1ED005A67EEA77A91ED025AC1
:10AEF000E5EEA57AE5EE057AA5EEA76A80ED006A93
:10AF000091ED016AE6EE276AC0ED016AD1ED026AB1
:10AF1000A6EEA77A80ED027A90ED037A77EE277A93
:10AF2000C0ED037A704700BF2DE9F04F4FF00009E4
:10AF3000864600F110050646034689B000F1300848
:10AF4000074648462C468B469C46B246CDF80CE058
:10AF500000283CD10CF1040CA445FBD1032800F1DE
:10AF6000010151D09C46AA46029398B1DCED047AC7
:10AF7000AAEB0903B64601927246F3EC016A0EF1A0
:10AF8000100E92ED007A5345E6EEC77ACCED047AC6
:10AF9000F2D1019ADCED046A0CF1100C15ED047A83
:10AFA0000AF1100AC445C6EE877ACCED007ADCD1EE
:10AFB000029B0436084608F1040814331435103493
:10AFC000103709F104099C46B2460028C2D0DCEDD6
:10AFD000007AD646394601927246F1EC016A0EF1CA
:10AFE000100E92ED007A9942E6EEC77ACCED007A27
:10AFF000F2D10CF1040C019A0AF1040AA445E6D13D
:10B00000032800F10101ADD1DDF80CE00023594621
:10B0100004AD764677460020049305930693079384
:10B02000F2EC017AE5EC017AB0B104AC3B46B4EC49
:10B03000017AF3EC016AE6EEC77AB34245ED017A94
:10B04000F5D1013004280BD0F2EC017A1037143618
:10B05000E5EC017A0028E8D1103714360120DFE74B
:10B0600008AD10310EF1400E042875ED017AA1F102
:10B070000402744641ED017A1ED07346F3EC016A76
:10B08000B1EC017AA342E6EEC77AC2ED007AF5D1BF
:10B090005EED016A013887EEA67A82ED007A17D05C
:10B0A000AEF1140E103C114675ED017A0428A1F1A1
:10B0B000040241ED017AE0D15EED016A103CAEF18F
:10B0C000140E032087EEA67A01ED017A1146EBE714
:10B0D00009B0BDE8F08F00BF60EEA00AE0EE000A04
:10B0E000F5EEC00AF1EE10FA07DBB1EEE00AB4EEBD
:10B0F000400AF1EE10FA00D670479FED010AFBE717
:10B100000000000060EEA00AE0EE000AE1EE010A95
:10B11000F5EEC00AF1EE10FA07DBB1EEE00AB4EE8C
:10B12000400AF1EE10FA00D670479FED010AFBE7E6
:10B1300000000000DFED297AB4EEE70AF1EE10FA24
:10B1400028DD9FED277A30EE470AB4EEE70AF1EEEC
:10B1500010FAF8DCDFED237AB4EEE70AF1EE10FA2C
:10B160002FDD30EE670A37EEC00A60EE007ADFEDC1
:10B170001E5A9FED1E6ADFED1E6AA7EEA56A9FEDBF
:10B180001D7A60EE275AE7EE866AA7EEA67AA5EE4C
:10B19000870A7047DFED187AB4EEE70AF1EE10FA8D
:10B1A000D8D59FED0F7A30EE070AB4EEE70AF1EE3C
:10B1B00010FAF8D4DFED0B7AB4EEE70AF1EE10FAEC
:10B1C000CFDC9FED0E7AB4EEC70AF1EE10FACCD5C3
:10B1D00030EE270A37EE400AC7E700BFDB0F4940D1
:10B1E000DB0FC940DB0FC93F9A7C2E36FAAF4FB94F
:10B1F0003587083CA4AA2ABEDB0F49C0DB0FC9BFB4
:10B2000010B5404CB4FBF2F4A14219D3DFED3E7A05
:10B21000F7EE005AB0EE677AB0EE676AF0EE676A52
:10B220000023C0ED005AC0ED017A80ED027A80ED76
:10B23000036AC0ED046A836143610362C36110BDA8
:10B2400007EE902ADFED315AB7EE006ADFED306A83
:10B25000B8EE677A07EE901AB0EE405AF8EE677AC9
:10B2600027EE257A67EEA67AC6EE076AC7EEA64AEB
:10B27000FDEEE47A17EE902A2032402A3FD8B0EE55
:10B28000640AFFF757FFB0EE404ADFED227A34EE52
:10B29000A70AFDEEC07A17EE902A2032402A29D85C
:10B2A000FFF748FFF8EE006A60EE266A012B1CD01B
:10B2B000B7EE006AF6EE004A36EE406A66EE244AC1
:10B2C00035EE055AF7EE007A84EE057A77EE275AC6
:10B2D00037EEC75A84EEA57AC6EE257A86EEA56AC1
:10B2E000C5EE256AF0EE475A9AE7F7EE004AB0EE4F
:10B2F000666AE5E7DFED086A9FED030AD6E79FED92
:10B30000024AC2E720A1070000000000BD378635D1
:10B31000DB0FC940DB0FC93F00000080DFED077A7B
:10B3200030EE270AFDEEC07A17EE903A2033402B1C
:10B3300000D8FFE69FED020A704700BFDB0FC93F50
:10B34000000000002DE9F84F9DF828408946DDF8FF
:10B350002CB00546002C17461BF8011B0CBF4FF004
:10B3600020084FF030081C1E08463ADB00295CD04C
:10B37000002C53D04FF0000A5B4600E064B313F892
:10B38000016B013C002EF9D1BAF1000F2FD12646F6
:10B3900044B14D454146284600D2B847013CF8D15A
:10B3A0000B9B18780146A0B14FF0FF344FF0000A14
:10B3B00000E09B464D45284600D2B8475B4613F84F
:10B3C000011B0029F5D10B9BF61A5E44BAF1000F60
:10B3D00010D13046BDE8F88FBAF1000F1BD15646A8
:10B3E000E0E7634229B31C464FF0010AC4E7002896
:10B3F000E0D10646002C04F1FF3AEADD54464D4503
:10B400004146284600D2B847013CF8D2013656449E
:10B410003046BDE8F88F30B12646CBE726464FF0E0
:10B42000FF34B246C6E70646D3E72646002CB0D125
:10B43000CFE76FEA040A0E46E0E700BF0FB430B56D
:10B4400083B00C4C06ABD4F87018D4F86C0853F8E1
:10B45000042B01936EF06EF80546D4F8840203685D
:10B460005B6998470028F8D0284603B0BDE8304013
:10B4700004B07047E05D00240EB410B583B00446FC
:10B48000084905AB01A853F8042BCDE900346EF050
:10B4900051F80022019B1A7003B0BDE8104003B0C0
:10B4A000704700BF858004080CB4F0B53C4CADF586
:10B4B000277DD4F87438002B6DD094F87C389942ED
:10B4C0000BD90123D4F880288340134205D10DF510
:10B4D000277DBDE8F04002B07047324B4FF47A71DF
:10B4E000314A1B68A2FB030206A8920901FB123332
:10B4F0002E49FFF7C1FF06ABAC9A064603442C4920
:10B5000001A80193ADAB00936EF014F8019B0A21E2
:10B5100000225D1C01951970019BD4F87458591CC8
:10B5200001911A70ADB12B685B6A1BB12846984730
:10B53000D4F874589DF818100029C8D00DF11904DA
:10B540002B6828461B68984714F8011B0029F7D17F
:10B55000BDE7D4F87878002FB9D0304426ABFD226F
:10B5600006A9841C1846ADF810202246CDF81250CA
:10B57000ADF816507CF0BEF802220346044402A93E
:10B580003846CDE9023435F0E9F90DF5277DBDE8FF
:10B59000F04002B07047D4F87838002B8DD196E790
:10B5A000E05D002444310024D34D6210AC470D0807
:10B5B00079800408184A033010B5D2F8844804EBA7
:10B5C0009003B3F5007F19D8C2F8843802F68802D8
:10B5D00020F00300C3F5007302EB84040F4A9B00C4
:10B5E00002EB810151F8702C10440D4A41F8700CA7
:10B5F00004210020FFF758FF204610BD0021094A12
:10B6000000240846FFF750FF044A2046936943F0A0
:10B610000073936110BD00BFE05D0024D86E00246C
:10B62000B8470D08DC470D0803685A1C02601878FB
:10B63000704700BF03681A46591C016012F8021BCC
:10B640000260587841EA0020704700BF0268134644
:10B65000511C016013F802CB0360D31C51780360C6
:10B6600093781B0443EA0123111D43EA0C03016094
:10B67000D07843EA0060704712B370B5044686463E
:10B6800004E0981B17D114EB0C0C15D01EF8013BED
:10B69000A3F14100A2EB0E0C192811F8010BA0F147
:10B6A000410598BF203300F12006192DE9D91B1A56
:10B6B00004D10028E7D170BD604670BD184670BD4A
:10B6C0001046704703880021184AA3F5FA6C70B53C
:10B6D00003F0030490F802E0154E40F2B5550EF168
:10B6E000FF3E04EB44044FEA9C0C0EEB8403C47849
:10B6F00036F81330013C05FB0C3390F804C02344AA
:10B70000847903EB430322444FF47A740CEBC30CAB
:10B7100043790089CCEB0C1C03EB8C03C3EB0313C4
:10B7200002EB8302C2FB040170BD00BF80436D3891
:10B73000609D0C082DE9F04116461F46404D044619
:10B74000394630464FF47A72002375F063FC3D4B66
:10B7500005443D4F3D4E83FB0510E9172844C1EBDE
:10B76000601183FB0103C8170B44C0EB631087FB18
:10B77000003CC317C3EBAC0386FB03764FEAE37EC2
:10B78000CEEBE61EC1EB0116A5EB860CC0EB001557
:10B790004FEA8E0684F806C0A1EB8501617103EBC8
:10B7A0004301A0EBC10040F2B55101FB1E332071F3
:10B7B000B3F5896F33DA40F2DA218B4237DCB3F527
:10B7C000B77F234FB4BF4FF0000E4FF0010E0EEBCA
:10B7D0004E0175464FEA4E0807EBC101C88A08EBD7
:10B7E0000E0C0B2107EBCC0C0CF1160C01E03CF815
:10B7F000020D984210DD0139F9D1F044012137F8EA
:10B80000380006F5FA6E0133A17075441B1A2281C7
:10B810002580E370BDE8F0810131C9B2F1E703256D
:10B8200040F296500A4F4FF00608AE46D7E7022581
:10B8300040F22940064F4FF00408AE46CFE700BF64
:10B8400080BC92C789888888ABAAAA2A73B06D1673
:10B85000609D0C0830B5304C8DB086460D46EC46E8
:10B860001EF0030F0FCCACE80F000FCCACE80F00BC
:10B8700094E80F008CE80F000FD1284B284A03FBF7
:10B880000EF3B2EBB30F44D3264AB2EB331F34BFEF
:10B8900001220022C2F11D0200E01C220EF1FF3342
:10B8A000019240F26D122048002B194602FB0EF265
:10B8B0001E4CB8BF0EF10201EE4602EBA10280FB66
:10B8C0000310DB17ADF1040101EB8501A3EB60155B
:10B8D000C3EBE0132A441A44253284FB0230D31709
:10B8E0001044C3EBA003C3EBC303D31A5EF8040FE9
:10B8F000C218714584FB023C4FEAE2739444C3EBE7
:10B90000AC03C3EBC303A2EB0303EFD1C01A0DB02A
:10B9100030BD1D22C2E700BFC09D0C08295C8FC24C
:10B92000285C8F020AD7A3001F85EB51932449920C
:10B930000D4B10B5D3E9084354EA03020AD101467E
:10B94000002340F2011218460B80C1F802208B71CF
:10B950000B8110BD054A1268121943F10003FFF76D
:10B96000E9FE012010BD00BFD86E00244431002440
:10B9700030B5134D83B00446D5E9081351EA0302EC
:10B980000AD1002340F2011218462380C4F8022095
:10B99000A371238103B030BD0A4A1268521843F1E3
:10B9A0000003FFF7C7FE2B8D20460DF1060221464E
:10B9B000ADF8063069F0F0FF012003B030BD00BFE4
:10B9C000D86E0024443100242DE9F047044688B0A5
:10B9D00094F83030042B11D8DFE803F050136103E2
:10B9E0005A00237E9A0640F1F8800023112204A910
:10B9F000E069FEF7BBF8012800F0EF8008B0BDE871
:10BA0000F087C44D03AE04F11C0705F505793246F5
:10BA100039464846FEF732FE012800F0F980022838
:10BA2000ECD195F92E325F1C0AD005EB0313FF21F0
:10BA300093F8832085F82E1222F0010283F88320E8
:10BA400095F92F325E1C17D0023305EB031292F8E2
:10BA50006320C2F34502012A40F25A81013A02F002
:10BA60003F0205EB031393F8631062F34601FF22D4
:10BA700083F8631085F82F22042306E0A6486BF0B4
:10BA80002FFB4FF6FF720123228484F830309FE7AA
:10BA90000020E36A207008B0BDE8F04718479D4DCC
:10BAA00095F83C32002BA9D104F11C0705F5057867
:10BAB00003AE324639464046FEF7E0FD012840F02D
:10BAC0001581039B002B00F0F0801A780AB1E52A5B
:10BAD000EFD12A6F9A1A48BF02F2FF12B2F5805FC7
:10BAE0004FEA622180F0498109018C4A0A44917B26
:10BAF00004290CD0D5F8F4100131C5F8F4105160C8
:10BB000004219173D5F8F8200132C5F8F82095F991
:10BB10002E22501C0AD005EB021292F8831021F05D
:10BB2000010182F88310FF2285F82E2295F92F2239
:10BB3000511C17D0023205EB021191F86310C1F3CA
:10BB40004501012940F26181013901F03F0105EB16
:10BB50000212FF2085F82F0292F8630061F346007D
:10BB600082F863002022002118467CF0EBFED4F816
:10BB700031100346D4F8352005A819605A6094F8AE
:10BB80003B20B4F839109A721981627E0193DA72FF
:10BB9000FFF7EEFE019B002800F0D8809DF816000C
:10BBA0009DF817209DF8191042EA4012BDF81400C4
:10BBB0004901A0F2BC7042EA40229DF81A0041EA15
:10BBC00050019DF8180092B241EAC02188B2D98193
:10BBD0001A821A83D882032357E720466BF080FA33
:10BBE0002369002B00F08780237E03F0F70213F017
:10BBF0000403227640F09480122A00F0AA800022EA
:10BC0000E36A204684F8282008B0BDE8F0471847CA
:10BC1000DDF80C80B8F1000F00F0BB8098F8003020
:10BC2000002B00F0B68098F80BA01AF0080F7FF4F4
:10BC3000EEAE0B2204F1310140467BF0D7FC002828
:10BC40007FF4E5AE637E8AEA0303DF0640F1E1801C
:10BC500095F92E325E1C0AD005EB0313FF2193F8F1
:10BC6000832085F82E1260F3000283F8832095F973
:10BC70002F22511C3FF400AF023205EB021393F860
:10BC80006330C3F34503012B40F20681013B03F00F
:10BC90003F0305EB021292F8631063F34601FF23A2
:10BCA00082F8631085F82F32E6E695F814320922FF
:10BCB000022B3FF4E1AE95F83C32002B7FF4DCAE72
:10BCC00085F84C32404685F8483285F83C22C5E973
:10BCD0009433D5F82832C5F84032D5F87032C5F81B
:10BCE0004432FEF715FC01283FF4E3AE02287FF44E
:10BCF00085AE0423C9E6237E1B0780D5054B93F848
:10BD0000F421002A7FF47AAE072283F8F42176E743
:10BD10000022A6E6E05D0024F45F0024545E0024C7
:10BD20000023A5682046E66A294684F82830FEF7F5
:10BD300045FB002863D194F82830002B7FF45EAED9
:10BD40000223C4E90B6584F8283057E644F2817277
:10BD50003EE7E06A0421626AA063204684F83C3032
:10BD600084F8281063636362C4E90B22C4E90233D8
:10BD700008B0BDE8F0476BF0B3B995F8102212B9DE
:10BD8000012285F8102201226FF00F0185F8592059
:10BD9000ABE695F92E32591C0AD005EB0313FF21AF
:10BDA00093F8832085F82E1222F0010283F8832075
:10BDB00095F92F325A1C16D0023305EB031292F874
:10BDC0006320C2F34502012A21D9013A02F03F0261
:10BDD00005EB031393F8631062F34601FF2283F827
:10BDE000631085F82F22237EDB067FF545AE2C48B5
:10BDF0006BF076F94FF6FF720223228445E6002E9F
:10BE00003FF4FCAD2046334645E600219FE6002284
:10BE1000DEE7B8F81420B8F81A3043EA0243D5F840
:10BE20006C2263625202D8F81C30B3FBF2F102FBC1
:10BE30001131A36009B113445B1AE36084F819A0BF
:10BE400095F92E325A1C0AD005EB0313FF2193F803
:10BE5000832085F82E1222F0010283F8832095F9C1
:10BE60002F22531C3FF4B7AE023205EB021393F8B6
:10BE70006330C3F34503012B10D9013B03F03F03AB
:10BE800005EB021292F8631063F34601FF2382F878
:10BE9000631085F82F329EE60023FAE60023EFE7D1
:10BEA000F45F00242DE9F04390F8283083B0044675
:10BEB000013B082B0BD8DFE803F0393D1F24052A8E
:10BEC0000A2F34000121FEF71DF9012802D003B02A
:10BED000BDE8F08300222378216C84F82820002B11
:10BEE000F5D00322E162D4E9010384F828208342DB
:10BEF00038BF03462046A36003B0BDE8F043FEF719
:10BF00008BBC002103B0BDE8F043FEF7FBB803B0E3
:10BF1000BDE8F043FEF7F0B903B0BDE8F043FEF72B
:10BF20007FB903B0BDE8F043FEF7F2BA03B0BDE855
:10BF3000F04349E5DFF830914368D9F87462026B49
:10BF400019461E40D9F86C0294F800C0B518470293
:10BF5000B5EB402F41D34FF6F778BCF1020F14D068
:10BF600025692846002D5AD16168A3680020E26A3D
:10BF70008B4284F8280038BF0B46A360002AA6D065
:10BF8000204603B0BDE8F04310476168D9F87C0251
:10BF9000B1EB402F5CD22069217E090732D5D9F858
:10BFA000F011451CA9422AD299F81012002943D158
:10BFB000012389F8103289F85930226B636894F8AC
:10BFC00000C0D21B3B4432449B1B002697421946BB
:10BFD00063602263C4E90450BFD9BCF1020F37D0BB
:10BFE0002569002DC1D099F85830032B36D0ADB259
:10BFF0004FF6F7739D42B8D811446160B5E7E0D1C0
:10C000000025DEE701A969F067FD01287FF45FAF35
:10C010002069019D94F800C06368226BD1E799F80C
:10C02000581003290ED0A9B2414594BF0021012127
:10C030000029B1D06168D4E7012189F8591094F83A
:10C0400000C0BEE707498D4294BF00210121EFE700
:10C05000D9F87C32B1EB432FCED386E7014B9D421A
:10C0600083D8C9E7F7FFFF0FE05D002488422DE980
:10C07000F04198464FF0010439D301FB04F4B0FBC2
:10C08000F4FC8C45F9D264B30025BCF1000F04FB2D
:10C090001C00B4FBF1F7D4BF002601266DB966B9C8
:10C0A000A142354619D9C6460CF1300C0EF801CB29
:10C0B00000238EF80030BDE8F081BCF1090F18DDD7
:10C0C000002A0CBF57233723C6466344A14205F11B
:10C0D00001050EF8013BF046EAD83C46B0FBF7FC00
:10C0E000D3E7C64600238EF80030BDE8F0818446D1
:10C0F000CAE73023E8E700BF2DE9F04104461546C2
:10C1000008469442B4FBF2F607D205FB1644134BE3
:10C110001B5D00F8013BBDE8F0819642B6FBF2F7EB
:10C120000CD20E4B05FB176705FB1644DA5D1B5D51
:10C1300000F8012B00F8013BBDE8F081BA42B7FBE3
:10C14000F2F807D905FB1878044B13F8082000F81B
:10C15000012BE7E74046FFF7CFFFF3E7EC470D0879
:10C16000B5EEC00ADFED357A0023F1EE10FA30B5F6
:10C17000C8BF30EE270A87B0D8BF30EE670ADFEDC0
:10C18000307A054603A9029320EE270ACDE9003351
:10C19000FDEEC07A17EE904A84EAE470A0EBE470FA
:10C1A0006AF020FD002C03A8B4BF2D2320238DF8B6
:10C1B000003074F015F901282AD0022834D0032861
:10C1C0001ED003A968467DF07DFA684674F008F930
:10C1D000044669462846033CE4B222467BF08AFACC
:10C1E000002328462B5574F0FBF82E22431C0DEB40
:10C1F00004012A54E8187DF0DAFA284607B030BD69
:10C20000302303A968468DF801307DF05BFADCE746
:10C2100043F23002302303A96846ADF801208DF8BF
:10C2200003307DF04FFAD0E743F2300303A96846AC
:10C23000ADF801307DF046FAC7E700BF6F12033A50
:10C2400000007A440378202B03D110F8013F202B03
:10C25000FBD0092BF9D02D2B63D02B2BB7EE000A86
:10C2600008BF01300278A2F13003D9B2092961D8A0
:10C27000F2EE046ADFED4D7A07EE103A10F8012F66
:10C28000B8EEC77AA2F13003D9B2A7EEA67A09298F
:10C29000F0EE477AF0D92E2A50D0037803F0DF036E
:10C2A000452B3BD110B442782D2A73D02B2A62D073
:10C2B000A2F130030130092B63D80024002303EBE3
:10C2C000830302EB430310F8012FA2F13001303B4E
:10C2D0000929F4D9B3F59A7F1A46B7EE007A28BF38
:10C2E0004FF49A72072B09D91346DFED316A083BE8
:10C2F00027EE267A072BFAD802F007022AB1F2EECF
:10C30000046A013A27EE267AFBD1002C3BD0C7EE17
:10C31000877A5DF8044B20EE270A704720EE270A43
:10C32000704742780130BFEE000AA2F13003D9B263
:10C3300009299DD92E2ADFED1D7AAED1437801302F
:10C34000A3F13002D1B20929A8D8B2EE047AF0EEF6
:10C35000475A06EE902A10F8013FB8EEE66AA3F1BC
:10C360003002D1B2C6EE076A092927EE257A77EEA8
:10C37000A67AEED992E782780230A2F13003092B37
:10C380009BD9B7EE007A67EE877A5DF8044B20EE12
:10C39000270A704782780230A2F13003092B01D8B6
:10C3A00001248BE7B7EE007AB1E700BF0000000080
:10C3B00020BCBE4C0378092B01D0202B05D110F8EE
:10C3C000013F202BFBD0092BF9D02D2B09D0017870
:10C3D0004FF0010CA1F13002D3B2092B0AD9002091
:10C3E0007047417801304FF0FF3CA1F13002D3B2E9
:10C3F000092BF4D8002310F8011F03EB830302EB91
:10C400004303A1F13002D1B20929F4D90CFB03F0A6
:10C41000704700BFAB4BAC4A2DE9F04F4FF0000A1C
:10C4200097B09E1A41F221051F462C2200210DEBE8
:10C4300002007CF087FAA44AA44B0892CDE9097661
:10C44000DA68D10707D5A24A5A6002F188325A60E9
:10C45000DB68DC070DD49D4BD3F80C21D20708D53F
:10C460009B4AC3F8042102F18832C3F80421D3F8AF
:10C470000C31002101227E2308A8149105A98DF812
:10C4800054208DF81430FDF7D5FA0028C0F2298128
:10C4900008214FF4FC4303E05B0001399BB207D055
:10C4A0001AB2002AF8DA85EA4202013993B2F7D1CA
:10C4B000884AADF81630884B934280F051819846F7
:10C4C0000DF11809CDE902A7B8F802204FF0000CD1
:10C4D000B8F80030C2F30B0B10048DF81DC00BF13F
:10C4E0000601ADF81810C3F30B014FEA1333ADF892
:10C4F0001A108DF81C3000F191800622494608A8D8
:10C50000FDF798FA0028C0F2FD80BDF816404946B4
:10C510000DF11E0011F8013B082284EA032403E018
:10C520006400013AA4B207D023B2002BF8DA85EAFE
:10C530004303013A9CB2F7D18842EBD15A46D8F86E
:10C54000041008A8FDF776FA0028C0F2DB80D8F8BE
:10C55000041001EB0B00814215D00139013811F8AC
:10C56000013F082284EA032403E06400013AA4B2F4
:10C5700007D023B2002BF8DA85EA4303013A9CB2D4
:10C58000F7D18142EBD1ADF8164008F11408514BB8
:10C59000984599D3DDE902A700230222494608A85D
:10C5A000ADF81830FDF746FA0028C0F29A80BDF8C1
:10C5B00016300DF11A0041F2210119F8012B08245F
:10C5C00083EA022303E05B00013C9BB207D01AB26E
:10C5D000002AF8DA81EA4202013C93B2F7D14845D9
:10C5E000EBD102220DF1160108A8ADF81630FDF7C7
:10C5F00021FA002875DB1398002840F089801498F0
:10C6000000286EDB9DF85420002A40F09780002817
:10C610000DBF012200220123002364E0E2466746A9
:10C62000019601370622494608A8FFB28DF81D7011
:10C63000FDF700FA002851DBBDF8164049460DF120
:10C640001E0011F8013B082284EA032403E0640081
:10C65000013AA4B207D023B2002BF8DA85EA4303EB
:10C66000013A9CB2F7D18842EBD1D8F804105A466F
:10C6700008A801EB0A063146FDF7DCF900282DDB9E
:10C6800006EB0B00864215D0711E013811F8013FF0
:10C69000082284EA032403E06400013AA4B207D02C
:10C6A00023B2002BF8DA85EA4303013A9CB2F7D1B2
:10C6B0008142EBD1032FDA44ADF81640B1D1019E8F
:10C6C00063E700BF000004080000020800200052D9
:10C6D0002301674544040E0890FE0D08DDE9016A58
:10C6E000039F012300220AF1010ABAF1020F02DCC2
:10C6F000002B7FF49AAE12B1FBF7D2FC28B90520CB
:10C7000008F068FCDDE902A7EBE717B0BDE8F08FA1
:10C71000089B099A03449342E3D80BABC0F1200273
:10C72000214618447CF00EF9149818B90BA908A8F2
:10C73000F6F71CFE00221490139261E70A4AD168B2
:10C7400041F00101D160D168C9077FF560AFD2F82F
:10C750000C1141F00101C2F80C11D2F80C2156E77E
:10C760000DF1180918E700BF00200052007970474A
:10C770000079C0F34010704700794009704700BF4E
:10C7800090F83C20034602F0FF0012B1002283F82B
:10C790003C2070474FF48053838170474FF400630F
:10C7A000838170474FF40063838170474FF40063C7
:10C7B000838170474FF4006383817047074B10B447
:10C7C00003F11001002453F8042B824208BF43F800
:10C7D000044C8B42F7D15DF8044B704720D80024FD
:10C7E00070B5374CE08B238AB4F928501B1AA08B04
:10C7F000B4F916C000FB03F3B4F92600666B05EB31
:10C80000E335C00290FBF5F000EBE330B4F92230E1
:10C81000A0F57A6EE0620EFB0EF50EFB0CFC2D13FC
:10C820004FEAEC2C05FB03F30CEBE32CB4F92030BE
:10C8300005FB03F3B4F918501B140EFB05F503EBCD
:10C840006533B4F9145002330CEB850CB4F9305055
:10C850009B10648B0CFA05FC03F500430CF1020CF1
:10C8600004FB03F34CF25034A6EBAC0C2C41DB0B75
:10C8700004FB0CF4002C1EDB6400B4FBF3F389B161
:10C880001C1240F6DE3504FB04F405FB04F40D4DE8
:10C89000241403FB05F504EB254404F6CF6403EBF5
:10C8A00024130B602AB100EB800040000830001117
:10C8B0001060012070BDB4FBF3F35B00DFE700BF45
:10C8C00020D8002443E3FFFF012070470120704778
:10C8D0002DE9F04F734D85B00F46A86BAB8F0092DA
:10C8E000C3EB2014B5F940205B00B5F948E004FB28
:10C8F00004F4B5F84280C3EBE003CDF80CE0241358
:10C90000B5F94A60B5F94C1002FB04F4B5F93E20C4
:10C91000029602FB03F3A413B5F9442004EBE324CD
:10C92000AB6DA4F5FA300193B5F9463080FB00EA0F
:10C930004FEAE37B82FB002C03FB0AF94FEA0C3C35
:10C940006C650EFB0B99A3FB0E3B4CEA125C1203C9
:10C95000CB441B0A43EA0B639B184CEB2B2BA3FB2A
:10C9600008320BF5004B08FB0B2B4FEAEB734FEA39
:10C970006B0953EA6B0B00F09280029E01FB0AFAEE
:10C98000019A86FB0008039EC2F5801C4A464FEAC6
:10C9900048484FEAE17948EAD0380EFB09A940043B
:10C9A000A1FB0E1E4118F1444FF000000CF0004EA8
:10C9B00049EB08094EEA5C0E41184FEACC7C09EBC2
:10C9C000C609BCEB010C6EEB090E1CEB0C084EEB20
:10C9D0000E0118EB0C084EEB01014FEA88104FEAEC
:10C9E000811918EB000049EA986941EB09018900B7
:10C9F00041EA9071800010EB0C004EEB01018900C0
:10CA000041EA9071800010EB0C004EEB010174F0D4
:10CA100001FBB5F952304FEA613884464FEA503E87
:10CA2000B5F94E204FEAE37A03FB08F94EEAC14E0E
:10CA3000B5F950000EFB0A99A3FB0E35A94403FB80
:10CA400008F50EFB0955A3FB0E3E75445B0E4FEA3D
:10CA5000E07E43EAC51313EB0C0341EB656500FB75
:10CA600001F10EFB0C11A0FB0C0C6144C00C40EA60
:10CA700041301B1845EBE1451B0A43EA056303EB14
:10CA800002130FB11B0A3B60009B23B104EB84042B
:10CA9000803424121C60012005B0BDE8F08F002313
:10CAA000EFE700BF20D8002431B10A4BD3ED1E7A46
:10CAB000FDEEE77AC1ED007A52B1064B9FED067AA2
:10CAC000D3ED1F7A67EE877AFDEEE77AC2ED007A42
:10CAD0000120704720D800240000C8422DE9F04F03
:10CAE0005F4D934685B0B5F88E30D5F880001B02B7
:10CAF000B5F88CE0B5F88A40C21AB5F888300191D3
:10CB000067EB0707AEFB020C1B04B5F886100EFBA3
:10CB100007CCC009B5F89060C90340EA4C604FEA01
:10CB2000EC1CC018A4FB023E04FB07EE4FEA1323E3
:10CB30004CF1000C43EA0E634FEA2E2E5B18A6FB65
:10CB4000021406FB07444FEAD1514EF1000E41EAB0
:10CB50004421E41511F5FA6844F10006B8F5FA6FBE
:10CB6000029676F1000630DA01FB04F60394A1FB8D
:10CB7000014A0AEB460AA6004FEA8A09361949EA31
:10CB80009479384C4AEB09094FEA560AB6084AEA42
:10CB9000C97A46EA8976B0EB0A0A6CEB690C9E1BEF
:10CBA00050466EEBA90E3346A045029E4FF0FF346F
:10CBB000A64126DB02FB07F7A2FB022101EB47019E
:10CBC000D20F42EA4102B8EB0208019C84B1D5F8C9
:10CBD0009410A1FB033201FB0E225B0D43EAC2233A
:10CBE00052151B1A62EB0C02DB0B43EA4243236033
:10CBF000BBF1000F01D0CBF80080012005B0BDE8EB
:10CC0000F08F40F6AC56039C891944F1000401FBF7
:10CC100004F4A1FB016101EB4401F4004FEAC109F6
:10CC2000341B49EA567961EB090924184CEB090CCD
:10CC30002046B41941EB0109A41941EB09094FEA57
:10CC4000890949EA9479A400A41B69EB01096108E8
:10CC500041EAC971591A6EEB690E0B46AAE700BF8B
:10CC600020D8002424FAFFFF01207047104B10B495
:10CC7000104C1B68D4F898001B1AFA2B0BD811B172
:10CC8000D4F8A0300B6012B1D4F8A43013600120A6
:10CC90005DF8044B7047084A00211368084684F881
:10CCA0009C1023F004035DF8044B1360704700BF31
:10CCB0004431002420D8002414A50024012070470A
:10CCC000064B002200210120C3F8A820C3F8AC20A5
:10CCD000C3F8B020C3F8B410704700BF20D80024B8
:10CCE000104B11491A680346D1F8B400121AFA2AF7
:10CCF00016D8D1ED2A6A012091ED2B7AFDEEE66A75
:10CD0000D1ED2C7ABDEEC77AFDEEE77A16EE902AC9
:10CD1000DA8617EE102A1A8717EE902A5A8770477C
:10CD2000002070474431002420D800240F4B70B5F8
:10CD300093F8B83082B00191ABB90D4B1D6895B135
:10CD40002B681A687AB19B686BB1044628469847ED
:10CD500048B1019922462E6828460B46316802B038
:10CD6000BDE87040084702B070BD00BF20D8002465
:10CD7000C0A900240B4B70B51E688EB133681A68C9
:10CD800072B19B6863B1054630460C46984738B18E
:10CD900031682A46234630460968BDE87040084796
:10CDA00070BD00BFD8A90024024BD3F8BC305B682B
:10CDB000184700BF20D80024024B0830D3F8BC30FD
:10CDC0009B68184720D80024012070470120704735
:10CDD00001207047012070470120704731B10C4B92
:10CDE000D3ED307AF8EEE77AC1ED007A72B10849F6
:10CDF000084BD1F8C410DFED086A0B4407EE903AF7
:10CE0000F8EEE77A87EEA67A82ED007A704700BFE7
:10CE100020D800244D95FFFF0000C8420120704734
:10CE2000012070477A4A014600239446104610B408
:10CE300090F904400C30012C4DD00133082BF7D170
:10CE4000734C002394F904000C34022858D00133A9
:10CE5000082BF7D16E4C002394F904000C340328FE
:10CE60006BD00133082BF7D1694C002394F90400EF
:10CE70000C34052877D00133082BF7D1644C0023FC
:10CE800094F904000C34062800F083800133082B49
:10CE9000F6D1002392F904000C32072800F09380A9
:10CEA0000133082BF6D15B4B1B68DC0340F1A180FA
:10CEB000594B086803F58C7403E01433A34200F067
:10CEC00098801A689042F8D1DA68D201F5D501202D
:10CED0005DF8044B704703EB43035CF8233023B346
:10CEE0004E480B7990F8D14090F8D000984218BF86
:10CEF0009C420CBF01200020A2D15DF8044B70477A
:10CF000003EB43035CF823308BB145480B7990F871
:10CF1000D04090F8D100984218BF9C420CBF01202D
:10CF2000002097D15DF8044B7047394C8AE7384CA4
:10CF300094F904000C34032893D103EB43035CF809
:10CF40002330002B3BD037480B7990F8D04090F835
:10CF5000D100984218BF9C420CBF0120002083D111
:10CF60005DF8044B704703EB43035CF8233043B395
:10CF70002D480B7990F8D04090F8D100984218BF16
:10CF80009C420CBF012000207FF478AF5DF8044B79
:10CF9000704703EB43035CF82330002B3FF47AAF78
:10CFA00022480B7990F8D04090F8D100984218BFF1
:10CFB0009C420CBF012000208AD003466AE7144C33
:10CFC00054E7134C5CE703EB43035CF82330002B7E
:10CFD0003FF469AF164A0B7992F8D10092F8D0204D
:10CFE0009A4218BF98420CBF012000207FF45BAF2B
:10CFF0006EE70B79312B04D82F2B94BF0020012032
:10D0000066E7343B012B8CBF0020012060E700BFA6
:10D010008C890024B86F00242403002464070024B2
:10D020003C0A0024140D0024EC0F0024C412002438
:10D030009C1500240B4B8446002010B503F58C7E14
:10D0400002E014339E450BD01A686245F9D1DA68C4
:10D05000441C8A42F5D0D9601433E0B29E45F3D126
:10D0600010BD00BF24030024704700BF40F2FF72D0
:10D07000044B914203EBC003A8BF1146A3F8CC10A8
:10D08000704700BF20D80024112807D8044B03EBB9
:10D090008003D3F828310BB19B68196029F0F8BAE6
:10D0A00020D80024112807D8044B03EB8003D3F8C1
:10D0B00028310BB19B681960704700BF20D800244D
:10D0C0002DE9F04103EB4306964686B0034602EB9A
:10D0D0004606754612F9067BA3EB070C92F8008012
:10D0E000BCF1000FA3EB0804B8BFCCF1000C002C7E
:10D0F000B8BF6442644502DA15464FFA88F7063233
:10D10000B242E9D1688803E00EF1060E764518D0E8
:10D110009EF800208446BA42F6D10A1ABEF8028070
:10D12000002AA1EB0804B8BF5242002CB8BF6442E9
:10D130009442E9DA75460EF1060E4046C44676453D
:10D14000E6D16879CDF808C02A7804902879019250
:10D150000390012000910321034AFEF7A5F9284618
:10D1600006B0BDE8F08100BFD84C0D0838B50568A1
:10D170000446EB69F3B1987800B938BDB3F90A20D9
:10D18000012007EE902AF8EEE77AC4ED057AB3F9AC
:10D190000C2007EE902AF8EEE77AF1EE677AC4EDFC
:10D1A000047AB3F90E3007EE903AF8EEE77AC4ED60
:10D1B000067A38BD09211420FEF7FCF90346E86120
:10D1C000D9E700BF38B505680446EB69E3B1987844
:10D1D00000B938BDB3F90420012007EE902AF8EE1B
:10D1E000E77AC4ED047AB3F9062007EE902AF8EE48
:10D1F000E77AC4ED057AB3F9083007EE903AF8EE15
:10D20000E77AC4ED067A38BD09211420FEF7D2F979
:10D210000346E861DBE700BF38B505680446EB6903
:10D22000E3B1987800B938BD9A880120D2BA07EEE8
:10D23000902AF8EEE77AC4ED047ADA88D2BA07EEDB
:10D24000902AF8EEE77AC4ED057A1B89DBBA07EE7F
:10D25000903AF8EEE77AC4ED067A38BD0921142039
:10D26000FEF7A8F90346E861DBE700BF38B50568BB
:10D270000C46EB697BB1987800B938BD5B89012019
:10D28000084ADBBA82FB0312DB17C3EB221303F25B
:10D290006D13238038BD09211420FEF78BF9034656
:10D2A000E861E8E77978787870B506680D46144645
:10D2B000F069A0B3D0F80130CDB1D0F80520B7EEB9
:10D2C000006A9FED1A7A07EE902ADFED195ADFED1A
:10D2D000196AF8EE677A77EEC77A77EEA77A87EE63
:10D2E000A57A77EE467A67EEE67AC5ED007AACB1BC
:10D2F00007EE903A9FED107ADFED105AF8EEE77ADC
:10D300009FED0F6ADFED0F6A67EE877A87EEA57AE9
:10D3100077EE467A77EEA67AC4ED007A70BD0921E1
:10D320001420FEF747F9F061C4E700BF9AC9CC4466
:10D330009AC94C460E76D7450000484300E0FF44AA
:10D34000000048423393884370B5066882B00D46AA
:10D350001446F06900284AD0D0F80530F3EE096A87
:10D36000DFED265AB2EE047A07EE903A9FED246A7A
:10D37000D0F80130F8EE677A77EEE57A67EE867AD4
:10D3800067EEA67AF4EEC77AF1EE10FA20DCBAEE78
:10D39000047AF4EEC77AF1EE10FA19D42DB19FEDAC
:10D3A000197A67EE877AC5ED007A7CB107EE903A7C
:10D3B0009FED156ADFED156AB8EE677ADFED147A36
:10D3C000E7EE067A77EEA67AC4ED007A02B070BD79
:10D3D00017EE900A73F070F904460D460D4A0421C9
:10D3E0000320CDE90045FEF75FF802B070BD0921CA
:10D3F0001420FEF7DFF8F061AEE700BF0000004642
:10D40000000080380AD778430319C83D3393884316
:10D41000000048C2144D0D0890F91030F0B503EB30
:10D420004303264E154683B056F83360044683689E
:10D430009A0715D501230DF106028DF80610304626
:10D440000DF10701F6F7D6FF0123002229463046E9
:10D45000F6F7D0FFA3689B0716D5012003B0F0BDF7
:10D4600043691BB19A88186812048261144B154AEB
:10D470001868154BC0005768A3FB0030800953683B
:10D48000DB1B9842FBD2D5E70D4A4FF4FA700E4BE6
:10D4900012680C4900FB02F24868A3FB02329209B1
:10D4A0004B681B1A9A42FBD26369002BD5D01A68CD
:10D4B00001209B88936103B0F0BD00BFC40200242B
:10D4C000486F0024001000E0D34D6210F0B5044610
:10D4D00083B00D461746061D20680379012B19D02D
:10D4E000022B02D0002003B0F0BD83683246FF213A
:10D4F000DB075CBF3246FF21FFF78EFF0028F1D02B
:10D5000015B12379DB07E7D4002FECD023793B70EA
:10D5100003B0F0BD8268417C02F0010C90F910006C
:10D52000FF22CDE9006CF6F76FFCE7E770B5044623
:10D53000051D82B020680379012B16D0022B02D082
:10D54000002002B070BD83682A46FF21DE075CBF61
:10D550002A46FF21FFF760FF0028F1D02379DB077F
:10D56000EFD520680379012BE8D18668FF22417C42
:10D5700006F0010690F91000CDE90056F6F744FCDC
:10D58000EAE700BF024630B5044652F8040B83B008
:10D590000379012B0ED0022B01D0002008E0FF21DF
:10D5A000FFF73AFF0028F8D02079C04300F00100CF
:10D5B00003B030BD8568417C05F0010590F910008D
:10D5C0000092FF220195F6F71FFCEBE72DE9F041F1
:10D5D0004FF0B046D6F88050D6F888301D4010D0B5
:10D5E000DFF824800127B5FA85F4C4F11F0458F848
:10D5F000240007FA04F403689847A543C6F8884056
:10D60000F1D1BDE8F08100BFC06F002438B51446E9
:10D61000002944D0344B0D469FED344A93ED5C7A9B
:10D62000D3ED5F6AB8EEC76AB3F98C21B8EEE60AAB
:10D63000D3ED5D7A04EE902AB3F98821C6EE046A30
:10D6400093ED607A05EE902AB3F98A2105EE102A4F
:10D65000B3F98621B3F98431F8EEE44A06EE102AD4
:10D66000F8EEE55AF8EEE77AB8EEC55AB8EEC77AA2
:10D67000C7EE843A07EE903AB8EEC66AE6EEA45AD0
:10D68000F8EEE77AA6EE856AA6EEA57AE6EE867A49
:10D69000A6EE870AA3EEA70A76F0CEF828600CB3B0
:10D6A000114BF6EE005A9FED115AD3ED5D6AB3F9B6
:10D6B0007A21F8EEE66AB3F9783107EE102A9FED89
:10D6C0000C6A07EE903A86EE850AB8EEC77AF8EE55
:10D6D000E77A20EE070AA7EEA50A20EE060A76F002
:10D6E000ABF82060012038BD20D800240000F04AAB
:10D6F0000000C8420C4B03EBC00310B5D3F8C84080
:10D7000082B001916CB107EE901A94ED047A94ED19
:10D71000030AF8EEE77AA7EE870A76F08DF8A36899
:10D72000186002B010BD00BF20D80024F8B5544BDB
:10D730000D4614462DED048B1B7F022B18D09FED58
:10D74000510A7DB120EE000ADFED4F7ADFED4F6A1E
:10D750009FED4F7A20EE270AC0EE267A77EE877A81
:10D76000C5ED007A0CB14B4B2360BDEC048BF8BDCA
:10D77000494B4A4E1B6896F8901103F00202C1B95A
:10D780005B0516D4B2B1464BB3F9182001EE102A4E
:10D79000B3F91620B3F9143000EE902AB8EEC11A8E
:10D7A00000EE103AF8EEE00AB8EEC00AFDF7AAFC67
:10D7B000C7E722B9D6F8A03193ED330AC1E7D6ED19
:10D7C000658A96ED669AF0EE680AB0EE490AFDF7B2
:10D7D00075FAB5EEC00AB0EE408AF1EE10FA47D401
:10D7E000B0EE680A2F4FF0EE490AFDF775FCDFED49
:10D7F0002E7ADFED2E6AF0EE408A28EE278AD7F8DF
:10D80000EC239FED2B6A9FED2B7AC8EE267AFCEE77
:10D81000E77A17EE903A9BB29B1A07EE903AF8EE31
:10D82000E77A67EE867AA7EEA67AFDEEC77AB0EEC3
:10D83000470A17EE903A2033402B1ED8FDF77AFCAA
:10D84000F0EE407A1C4BB97CA3F12C021846443B05
:10D85000D6ED670A90ED000A002918BF1346A8EE1E
:10D86000E70AD3ED057A70EEA70AFDF735FC68E705
:10D87000DFED127A30EE278AB2E7DFED027AE1E7D8
:10D88000D8A5002400000000CDCC9C3F00409C4661
:10D8900082E6C54733139043D874002420D800246F
:10D8A0002C8A0024608A00240000C84235FA8E3C8D
:10D8B0000AD7233CDB0FC93F608E0024DB0FC94031
:10D8C00070B545880B4604460021C5F30B05184684
:10D8D0002A467BF037F80A4A21690346914206D36B
:10D8E000084A914206D31846BDE87040084700290F
:10D8F000F9D170BD2A46BDE8704079F0FBBE00BF8B
:10D9000044040E087B090E0810B5037982B08E46D8
:10D91000012B0DD0022B02D0002002B010BD836875
:10D92000DB0758BF41F0800102B0BDE8104073E54D
:10D93000816814467246009401F00104417C90F91C
:10D9400010000194F6F760FA02B010BD10B504465D
:10D95000C06900B110BD09211420FDF72BFEE06164
:10D9600010BD00BF10B1036882889A61704700BF84
:10D9700018B1838802681B0493617047174B53F8F2
:10D98000200038B300EB400003EB800292F9A5C100
:10D99000BCF1FF3F1FD092F8AD01D8B103EB0C00F2
:10D9A000002310B590F8F8E18C2092F8AC11142205
:10D9B00000FB0CFC0A4C0CEB0100013A714434F8FA
:10D9C000100013FA80F3F6D1064AA2FB0320C0F33D
:10D9D0000F1010BD70470020704700BF20D80024F2
:10D9E000C0300030CDCCCCCC30B50D4683B0032058
:10D9F0001446FFF7C3FF01909DB107EE900ADFEDDB
:10DA00000B5AB0EE006ADFED0A6AF8EE677AB8EEFC
:10DA1000047A67EEA57AA7EE867A67EE267AC5EDD8
:10DA2000007A0CB1034B236003B030BD6740533A1A
:10DA300000007A4433139043104B70B5104CA3424E
:10DA400019D2054602E00C33A34214D293F805C064
:10DA50008C45F8D193F804C00DB1AC45F3D1D87919
:10DA60009042F0D1186890F804E0E645EBD10668E2
:10DA70009E42E8D170BD002070BD00BFA00200082A
:10DA8000800400080379022B00D0704790F9102021
:10DA900008311C4802EB420210B41B4C83B050F812
:10DAA000322000946944194C11F808CCA24224D0C9
:10DAB00017498A4223D001F580618A4205D0154B6F
:10DAC0009A420CBF03234FF0FF33116803EB43036B
:10DAD00021F0010100EBC30011600169936851F866
:10DAE0002C1023F0E0430B439360136843F00103D1
:10DAF000136003B05DF8044B70470023E5E7012392
:10DB0000E3E700BFC402002400010203003001402B
:10DB1000003800400034014090F91030F0B503EBBC
:10DB20004303284E154683B056F833600446836895
:10DB30009A0719D501230DF106028DF8061030461B
:10DB40000DF10701F6F756FC01230DF106020DF168
:10DB5000070130468DF80650F6F74CFCA3689B078A
:10DB600016D5012003B0F0BD43691BB19A8818682F
:10DB700012048261144B154A1868154BC00057688F
:10DB8000A3FB003080095368DB1B9842FBD2D1E72E
:10DB90000D4A4FF4FA700E4B12680C4900FB02F26A
:10DBA0004868A3FB023292094B681B1A9A42FBD2C7
:10DBB0006369002BD5D01A6801209B88936103B05C
:10DBC000F0BD00BFC4020024486F0024001000E034
:10DBD000D34D621010B5037984B084468E46012B74
:10DBE0000DD0022B02D0002004B010BD8368DB07EB
:10DBF00058BF01F07F0104B0BDE810408CE7816898
:10DC00000DF10F001446724601F001018DF80F402E
:10DC1000CDE900019CF811109CF91000F5F7D8FE31
:10DC200004B010BD70B5B42282B00446FF21006874
:10DC3000FFF7D0FF10B9002002B070BD2068251D8D
:10DC40000379012B13D0022BF5D183682A46FF21DB
:10DC5000DE075CBF2A46FF21FFF7DEFB0028EAD083
:10DC60002379DB07E8D520680379012BEBD186689F
:10DC7000FF22417C06F0010690F91000CDE9005624
:10DC8000F6F7C2F8EAE700BF70B50A4682B004466C
:10DC9000A5210068FFF79EFF10B9002002B070BDFB
:10DCA0002068251D0379012B13D0022BF5D1836841
:10DCB0002A46FF21DE075CBF2A46FF21FFF7ACFBA7
:10DCC0000028EAD02379DB07E8D520680379012B07
:10DCD000EBD18668FF22417C06F0010690F9100026
:10DCE000CDE90056F6F790F8EAE700BF002A34D0F5
:10DCF000F0B5044683B00E46051D8F1816F8012BAB
:10DD0000A5212068FFF766FF90B9002003B0F0BDA1
:10DD10008268417C02F0010C90F91000FF22CDE9ED
:10DD2000005CF6F771F80028EFD02379DB070FD5F8
:10DD300020680379012BEBD0022BE6D183682A46B9
:10DD4000FF21DB075CBF2A46FF21FFF765FBEAE7FF
:10DD5000B742D3D1012003B0F0BD0120704700BF0E
:10DD6000F0B5962283B00E460446FF210068FFF707
:10DD700031FF10B9002003B0F0BD251D20680379E4
:10DD8000012B1DD0022BF5D183682A46FF21DF0726
:10DD90005CBF2A46FF21FFF73FFB0028EAD023792A
:10DDA000DB07EBD4E12220681146FFF713FF0028C0
:10DDB000E0D03246FF21206803B0BDE8F040A3E583
:10DDC0008768FF22417C07F0010790F91000CDE938
:10DDD0000057F6F719F8E0E7002A42D0F0B50446FC
:10DDE00083B00E46051D8F189622FF212068FFF78D
:10DDF000F1FE90B9002003B0F0BD8268417C02F0D2
:10DE0000010C90F91000FF22CDE9005CF5F7FCFF52
:10DE10000028EFD02379DB070FD520680379012B89
:10DE2000EBD0022BE6D183682A46FF21DB075CBFDB
:10DE30002A46FF21FFF7F0FAEAE7E12220681146BF
:10DE4000FFF7C8FE0028D5D03246FF212068FFF733
:10DE50005BFD0028CED00136B742C5D1012003B00A
:10DE6000F0BD0120704700BFF0B50B4605461646D1
:10DE7000044683B087211A4655F8040BFFF7AAFE23
:10DE800020680379012B19D0022B02D0002003B0A7
:10DE9000F0BD83682A46FF21DF075CBF2A46FF21C9
:10DEA000FFF7BAFA0028F1D02379DA07E8D4002E78
:10DEB000EDD0C3F34013337003B0F0BD8768FF2289
:10DEC000417C07F0010790F91000CDE90057F5F704
:10DED0009BFFE7E7F0B5782183B0164604460022A1
:10DEE0000068FFF777FE10B9002003B0F0BD251DD4
:10DEF00020680379012B13D0022BF5D183682A46C1
:10DF0000FF21DF075CBF2A46FF21FFF785FA0028C3
:10DF1000EAD02379DA07EBD45B09337003B0F0BDA4
:10DF20008768FF22417C07F0010790F91000CDE9D6
:10DF30000057F5F769FFEAE770B5CC2282B00446D6
:10DF4000A5210068FFF746FE10B9002002B070BDA1
:10DF50002068251D0379012B13D0022BF5D183688E
:10DF60002A46FF21DE075CBF2A46FF21FFF754FA4D
:10DF70000028EAD02379DB07E8D520680379012B54
:10DF8000EBD18668FF22417C06F0010690F9100073
:10DF9000CDE90056F5F738FFEAE700BF70B5B422C7
:10DFA00082B00446FF210068FFF714FE10B900207C
:10DFB00002B070BD251D20680379012B21D0022BF2
:10DFC000F5D183682A46FF21DE075CBF2A46FF2180
:10DFD000FFF722FA0028EAD02379DA07EBD4CC2124
:10DFE0002046FFF751FE0028E1D002E02379DB074D
:10DFF000DED52A46FF212068FFF786FC0028F5D1F0
:10E00000D5E78668FF22417C06F0010690F91000F2
:10E01000CDE90056F5F7F8FEDCE700BF70B582B039
:10E020000446CDE90023FFF7FDFD10B9002002B042
:10E0300070BD5522A5212068FFF7CCFD0028F5D042
:10E04000251D2A46FF212068FFF75EFC0028EDD041
:10E050002379DB07F5D40DF1FF350DF1070615F82F
:10E06000011F2046FFF710FE0028DFD0B542F6D191
:10E07000DDE700BF2DE9F04F82468DB000209046CD
:10E080000AF10407089106900A930790069B5046F0
:10E09000DC0008EBC3030593FFF7C4FD28B941E09A
:10E0A0009AF8043013F0010208D03A46FF21DAF85A
:10E0B0000000FFF729FC0028F2D133E003929A0711
:10E0C0000B9040F1CC80F0215046FFF7DDFD48B3C6
:10E0D000083CDDF80C9008EB040301240993254665
:10E0E000089B003B18BF01230493049B082D8CBFA1
:10E0F000002303F001039B46002B5DD06E1E089B9E
:10E1000043FA06F606F00106F2017821DAF800007B
:10E11000FFF760FD30B1DAF800000379012B3FD042
:10E12000022B07D000220A9B1046069919700DB0E9
:10E13000BDE8F08F83683A46FF21DB075CBF3A46B3
:10E14000FF21FFF769F90028ECD09AF8043013F0AA
:10E150000102E0D199094FEA531E4FEAD31C01EAAC
:10E160005313DB074BD4664502D0BBF1000F73D1CC
:10E17000BCF1000F2DD0059911F80930234301F8A7
:10E1800009306400013514F0FF04EDB2ADD109F19E
:10E1900001095FFA89F9B9F1080F30D00124A4E729
:10E1A0008268417C02F0010C90F91000FF22CDE959
:10E1B000007CF5F729FEC6E7069BD3B1079BAB426F
:10E1C00017D9099B13F809301C4214BF01260026F9
:10E1D0009AE74EEA0101039B11F0010F059908BF70
:10E1E0002B46039311F8093023EA040301F80930A0
:10E1F000C7E7079B5E1BB6FA86F6760984E7402DD3
:10E2000007D80A9B069A1B7893423FF63FAF024617
:10E2100089E7059BDD795C1E9E1D14F801CF08215E
:10E2200082EA0C0301394FEA5C0C43F3000311F05E
:10E23000FF0123F0730383EA5202D2B2F0D1A64267
:10E24000EBD19542DDD1069B0133DBB20693039BF4
:10E25000002BDCD00793D4E70B9E324663E70646DB
:10E26000324660E7F0B5046883B0002107466426B3
:10E270002046FFF707FC15227E212046FFF7AAFC67
:10E2800006F04CFE04460D4606F048FE001B61EB0E
:10E290000501B0F57A7F71F10001F5D3013EEFD1B0
:10E2A000052611227E213868FFF794FC06F036FE21
:10E2B00004460D4606F032FE001B61EB0501B0F589
:10E2C0007A7F71F10001F5D3013EEFD10DF1070224
:10E2D00003213868FFF718FB9DF8073003F03C0373
:10E2E000142B40F09B800C2240213868FFF772FC11
:10E2F00006F014FE04460D4606F010FE001B61EB0E
:10E300000501B0F57A7F71F10001F5D3454C092381
:10E31000B96B454A97F83500B4FBF1F189B2FEF7C5
:10E32000CFFE0346422138685A88B4FBF2F43C64BD
:10E330001A79FFF74FFC06F0F1FD04460D4606F092
:10E34000EDFD001B61EB0501B0F57A7F71F1000175
:10E35000F5D3082241213868FFF73CFC06F0DEFDCA
:10E3600004460D4606F0DAFD001B61EB0501B0F531
:10E370007A7F71F10001F5D3002243213868FFF75D
:10E3800029FC06F0CBFD04460D4606F0C7FD001B38
:10E3900061EB0501B0F57A7F71F10001F5D3102230
:10E3A00051213868FFF716FC06F0B8FD04460D460B
:10E3B00006F0B4FD001B61EB0501B0F57A7F71F149
:10E3C0000001F5D30A2253213868FFF703FC06F059
:10E3D000A5FD04460D4606F0A1FD001B61EB0501FD
:10E3E000B0F57A7F71F10001F5D3802256213868AB
:10E3F000FFF7F0FB06F092FD04460D4606F08EFD99
:10E40000001B61EB0501B0F57A7F71F10001F5D3D6
:10E4100003213868FFF736FB03B0F0BD062006F095
:10E42000D9FD00BF40420F0038A40C082DE9F0418F
:10E430000768642682B0B6227E2180463846FFF700
:10E44000C9FB06F06BFD04460D4606F067FD001B98
:10E4500061EB0501B0F57A7F71F10001F5D3013E62
:10E46000EFD102213846FFF70DFB7B691BB19A887B
:10E47000196812048A6106F051FD04460D4606F043
:10E480004DFD001B61EB0501B0F57A7F71F10001D4
:10E49000F5D37B6913B11A689B8893610A2606F04D
:10E4A0003DFD04460D4606F039FD001B61EB0501FC
:10E4B000B0F57A7F71F10001F5D3013EEFD132461C
:10E4C0007C213846FFF786FB06F028FD04460D4602
:10E4D00006F024FD001B61EB0501B0F57A7F71F1B8
:10E4E0000001F5D3002259213846FFF773FB06F0EF
:10E4F00015FD04460D4606F011FD001B61EB0501FC
:10E50000B0F57A7F71F10001F5D397F910305E21F3
:10E510008D4A03EB43038DF8071052F83340BB6874
:10E520009A0740F1E48001230DF107020021204603
:10E53000F5F760FF4FF4A473844A20460021F5F7F5
:10E5400059FFBB689B0740F1E6800A2606F0E6FC0F
:10E5500004460D4606F0E2FC001B61EB0501B0F538
:10E560007A7F71F10001F5D3013EEFD101225921EB
:10E570003846FFF72FFB06F0D1FC04460D4606F0A7
:10E58000CDFC001B61EB0501B0F57A7F71F1000154
:10E59000F5D38C2240213846FFF71CFB06F0BEFC69
:10E5A00004460D4606F0BAFC001B61EB0501B0F510
:10E5B0007A7F71F10001F5D3032241213846FFF73C
:10E5C00009FB06F0ABFC04460D4606F0A7FC001B59
:10E5D00061EB0501B0F57A7F71F10001F5D35C4C78
:10E5E0000323D8F8382098F83500B4FBF2F291B242
:10E5F000584AFEF765FD43884221B4FBF3F4C8F89E
:10E6000040400279384642F0C002FFF7E3FA06F0D4
:10E6100085FC04460D4606F081FC001B61EB0501FC
:10E62000B0F57A7F71F10001F5D308224321384615
:10E63000FFF7D0FA06F072FC04460D4606F06EFCB9
:10E64000001B61EB0501B0F57A7F71F10001F5D394
:10E65000042258213846FFF7BDFA06F05FFC044655
:10E660000D4606F05BFC001B61EB0501B0F57A7FFF
:10E6700071F10001F5D30A2253213846FFF7AAFAB7
:10E6800006F04CFC04460D4606F048FC001B61EB0E
:10E690000501B0F57A7F71F10001F5D300227C21EC
:10E6A0003846FFF797FA06F039FC04460D4606F0A7
:10E6B00035FC001B61EB0501B0F57A7F71F10001BB
:10E6C000F5D306227D213846FFF784FA06F026FCB2
:10E6D00004460D4606F022FC001B61EB0501B0F577
:10E6E0007A7F71F10001F5D302B0BDE8F0817B695A
:10E6F0001BB11A689B881B049361174B17491A6852
:10E70000174BD2004868A3FB023292094B681B1AD0
:10E710009A42FBD207E7104A4FF4FA70104B126886
:10E720000E4900FB02F24868A3FB023292094B68D3
:10E730001B1A9A42FBD27B69002B3FF406AF1A6882
:10E740009B88936101E700BFC402002470A40C08F9
:10E7500040420F00B8A50C08486F0024001000E0EC
:10E76000D34D62102DE9F041816B0623654D0446BF
:10E7700007686426644A90F83500B5FBF1F189B268
:10E78000FEF79EFC4388002180463846B5FBF3F532
:10E790002564FFF777F980226B213846FFF71AFAD4
:10E7A00006F0BCFB04460D4606F0B8FB001B61EB0F
:10E7B0000501B0F57A7F71F10001F5D3013EEFD18B
:10E7C0006426072268213846FFF704FA06F0A6FB04
:10E7D00004460D4606F0A2FB001B61EB0501B0F5F7
:10E7E0007A7F71F10001F5D3013EEFD13246642604
:10E7F0006B213846FFF7EEF906F090FB04460D4614
:10E8000006F08CFB001B61EB0501B0F57A7F71F11E
:10E810000001F5D3013EEFD10F2601226B213846CE
:10E82000FFF7D8F906F07AFB04460D4606F076FBB2
:10E83000001B61EB0501B0F57A7F71F10001F5D3A2
:10E84000013EEFD10F2618221B213846FFF7C2F9EF
:10E8500006F064FB04460D4606F060FB001B61EB0E
:10E860000501B0F57A7F71F10001F5D3013EEFD1DA
:10E870000F2618221C213846FFF7ACF906F04EFB94
:10E8800004460D4606F04AFB001B61EB0501B0F59E
:10E890007A7F71F10001F5D3013EEFD10F2698F890
:10E8A00004201A213846FFF795F906F037FB044695
:10E8B0000D4606F033FB001B61EB0501B0F57A7FD6
:10E8C00071F10001F5D3013EEFD1642698F80520DF
:10E8D00019213846FFF77EF906F020FB04460D4665
:10E8E00006F01CFB001B61EB0501B0F57A7F71F1AE
:10E8F0000001F5D3013EEFD138460321BDE8F041D8
:10E90000FFF7C0B840420F00CCA50C082AE700BFB3
:10E91000F0B583B015461C4606460DF107020F46BA
:10E92000FEF7F2FF9DF8072005EA0203A34201D19A
:10E9300003B0F0BD22EA050239463046224303B057
:10E94000BDE8F040FFF746B9F8B50526782200216A
:10E9500007460068FFF73EF906F0E0FA04460D4668
:10E9600006F0DCFA001B61EB0501B0F57A7F71F16E
:10E970000001F5D3013EEFD10526202201213868A0
:10E98000FFF728F906F0CAFA04460D4606F0C6FA63
:10E99000001B61EB0501B0F57A7F71F10001F5D341
:10E9A000013EEFD13246642602213868FFF712F9A2
:10E9B00006F0B4FA04460D4606F0B0FA001B61EB0F
:10E9C0000501B0F57A7F71F10001F5D3013EEFD179
:10E9D0000120F8BD70B52422044641210068FFF7EC
:10E9E000F9F890B9052606F099FA04460D4606F0A6
:10E9F00095FA001B61EB0501B0F57A7F71F100011A
:10EA0000F5D3013EEFD1012070BD202230212068D6
:10EA1000FFF7E0F80028E5D0062231212068FFF753
:10EA2000D9F80028DED0002234212068FFF7D2F880
:10EA3000D8E700BFF8B5052607220A210746006877
:10EA4000FFF7C8F806F06AFA04460D4606F066FAC3
:10EA5000001B61EB0501B0F57A7F71F10001F5D380
:10EA6000013EEFD10526242241213868FFF7B2F894
:10EA700006F054FA04460D4606F050FA001B61EB0E
:10EA80000501B0F57A7F71F10001F5D3013EEFD1B8
:10EA90000526C02242213868FFF79CF806F03EFAAE
:10EAA00004460D4606F03AFA001B61EB0501B0F58D
:10EAB0007A7F71F10001F5D3013EEFD10120F8BD5D
:10EAC00010B50446002221210068FFF783F8FC22DC
:10EAD00020212068FFF77EF8402224212068FFF7DC
:10EAE00079F80C2223212068FFF774F800222221F4
:10EAF0002068FFF76FF8012010BD00BFF8B50122B4
:10EB0000074610210068FFF765F800B9F8BD142624
:10EB100006F004FA04460D4606F000FA001B61EB0D
:10EB20000501B0F57A7F71F10001F5D3013EEFD117
:10EB30003868A0221121BDE8F840FFF74BB800BFAC
:10EB4000F0B5046883B00746002120461426FEF77E
:10EB500099FF0C2225212046FFF73CF80A222621A6
:10EB60003868FFF737F8002263213868FFF732F87A
:10EB7000812227213868FFF72DF806F0CFF90446E7
:10EB80000D4606F0CBF9001B61EB0501B0F57A7F6D
:10EB900071F10001F5D3013EEFD10C222521386837
:10EBA0000A26FFF717F80A2226213868FFF712F81D
:10EBB0000F2263213868FFF70DF88122272138687A
:10EBC000FFF708F806F0AAF904460D4606F0A6F984
:10EBD000001B61EB0501B0F57A7F71F10001F5D3FF
:10EBE000013EEFD10A26032301AA1021384666F020
:10EBF0000DFD06F093F904460D4606F08FF9001B53
:10EC000061EB0501B0F57A7F71F10001F5D3013EAA
:10EC1000EFD19DF804009DF805109DF80620803086
:10EC20002B4B80318032A3F8FC01A3F8FE11252183
:10EC3000A3F800220C223868FEF7CCFF0A22262116
:10EC40003868FEF7C7FF3246632138680A26FEF7A8
:10EC5000C1FF812227213868FEF7BCFF06F05EF96C
:10EC600004460D4606F05AF9001B61EB0501B0F5AC
:10EC70007A7F71F10001F5D3013EEFD10DF103026E
:10EC800001230221384666F0C1FC01230DF1030285
:10EC90000921384666F0BAFC0C2225213868FEF7B7
:10ECA00099FF0A2226213868FEF794FF1222632179
:10ECB0003868FEF78FFF812227213868FEF78AFF28
:10ECC00038680321FEF7DEFE012003B0F0BD00BF6F
:10ECD00020D800242DE9F04180220B21074600684E
:10ECE000FEF778FF1E26804606F018F904460D460A
:10ECF00006F014F9001B61EB0501B0F57A7F71F1A4
:10ED00000001F5D3013EEFD1B8F1000F02D1002090
:10ED1000BDE8F081062229213868FEF75BFF002854
:10ED2000F5D008220B213868FEF754FF0028EED0FA
:10ED30003868CF220A21BDE8F041FEF74BBF00BF83
:10ED400010B5044694220B210068FEF743FF7122A0
:10ED500001212068FEF73EFF002204212068FEF713
:10ED600039FFC82205212068FEF734FF0022062162
:10ED70002068FEF72FFFC82207212068FEF72AFF30
:10ED8000002208212068FEF725FFC82209212068FB
:10ED9000FEF720FF012010BD0A4600212DE9F041B9
:10EDA000DFF8B08084B042F001020446274EFEF73F
:10EDB00011FFD8F80070264DC6F8047218E0022B37
:10EDC0004FF000000BD1A3680DF10F021321204674
:10EDD000DB0702D40DF10F029321FEF71DFB9DF816
:10EDE0000F30287013F0070318D1D6F808222ABB79
:10EDF0002379012BE3D1A2680DF10F0102F001028A
:10EE0000009101921322617C94F91000F4F7FCFF49
:10EE10009DF80F30287013F00703E6D001220B2174
:10EE20002046FEF7D7FE002220461146FEF7D2FE0E
:10EE300001232870184604B0BDE8F081D8F800100E
:10EE400089B2C91B8A42D3D2F4E700BF20D800247C
:10EE50003C2400244431002400680379012B0AD0AB
:10EE6000022B01D0002070478368F022DB0718D501
:10EE7000FF21FEF751BE826890F910C002F0010236
:10EE8000417C60464FF0F00C10B584B00DF10F04DA
:10EE90000192FF228DF80FC00094F4F799FD04B0A1
:10EEA00010BD7F21FEF738BE70B5056884B00446FA
:10EEB0000E462B79012B16D0022B02D0002004B075
:10EEC00070BDAB68E122DB071DD528461146FEF771
:10EED00023FE0028F2D03246FF21206804B0BDE8AE
:10EEE0007040FEF711BDAA68697C02F0010295F935
:10EEF00010000DF10F050192E12200958DF80F2011
:10EF0000F4F766FDE5E761212846FEF705FEE0E738
:10EF100070B5056884B004460E462B79012B17D0D6
:10EF2000022B02D0002004B070BDAB68C32228467B
:10EF3000DB074CBFE1216121FEF7EEFD0028F1D097
:10EF40003246FF21206804B0BDE87040FEF7DCBC0B
:10EF5000AA6895F9100002F00102697C01920DF196
:10EF60000F020092C3228DF80F20E122F4F730FD4A
:10EF7000E4E700BF0068CA43037941EA0211012BAC
:10EF8000CAB209D0022B01D0002070478368DB078A
:10EF900016D5D221FEF7C0BD10B584B0846890F9B3
:10EFA00010C08DF80F200DF10F0204F00104417C18
:10EFB0000092D22260460194F4F70AFD04B010BD1D
:10EFC0005221FEF7A9BD00BF70B5056884B00446A4
:10EFD0000E462B79012B1BD0022B02D0002004B04F
:10EFE00070BDAB68F0222846DB074CBFE1216121F0
:10EFF000FEF792FD0028F1D02246FF2152F8040BC3
:10F00000FEF782FC0028E9D02379337004B070BD8C
:10F01000AA6895F9100002F00102697C01920DF1D5
:10F020000F020092F0228DF80F20E122F4F7D0FCBD
:10F03000E0E700BF00680379012B0AD0022B01D062
:10F04000002070478368B422DB0718D5FF21FEF744
:10F0500063BD826890F910C002F00102417C6046F5
:10F060004FF0B40C10B584B00DF10F040192FF22E3
:10F070008DF80FC00094F4F7ABFC04B010BD7F21F5
:10F08000FEF74ABD00680379012B0AD0022B01D09C
:10F090000020704783680A46DB0716D5A521FEF7D6
:10F0A0003BBD10B584B0846890F910C00DF10F021B
:10F0B00004F001048DF80F10417C60460092A522F7
:10F0C0000194F4F785FC04B010BD2521FEF724BDA2
:10F0D00000680379012B0AD0022B01D00020704771
:10F0E00083689622DB0718D5FF21FEF715BD8268DD
:10F0F00090F910C002F00102417C60464FF0960C7E
:10F1000010B584B00DF10F040192FF228DF80FC0ED
:10F110000094F4F75DFC04B010BD7F21FEF7FCBC49
:10F1200000680379012B0AD0022B01D00020704720
:10F1300083680A46DB0716D58721FEF7EDBC10B5BC
:10F1400084B0846890F910C00DF10F0204F001043E
:10F150008DF80F10417C6046009287220194F4F7ED
:10F1600037FC04B010BD0721FEF7D6BC0068C9010A
:10F170000379CAB2012B06D0022B01D000207047C0
:10F180007821FEF7C9BC10B584B0846890F910C02E
:10F190008DF80F200DF10F0204F00104417C009264
:10F1A000782260460194F4F713FC04B010BD00BF50
:10F1B00000680379012B0AD0022B01D00020704790
:10F1C00083685522DB0718D5A521FEF7A5BC826808
:10F1D00090F910C002F00102417C60464FF0550CDE
:10F1E00010B584B00DF10F040192A5228DF80FC067
:10F1F0000094F4F7EDFB04B010BD2521FEF78CBCA4
:10F2000000680379012B0AD0022B01D0002070473F
:10F2100083682E22DB0718D5F421FEF77DBC8268B7
:10F2200090F910C002F00102417C60464FF02E0CB4
:10F2300010B584B00DF10F040192F4228DF80FC0C7
:10F240000094F4F7C5FB04B010BD7421FEF764BC54
:10F25000154B00681A8E03799201012B02F13402DA
:10F26000D2B209D0022B01D0002070478368DB079F
:10F2700016D5F421FEF750BC10B584B0846890F91F
:10F2800010C08DF80F200DF10F0204F00104417C35
:10F290000092F42260460194F4F79AFB04B010BD8A
:10F2A0007421FEF739BC00BF20D80024006810B5D7
:10F2B000037984B0012B0FD0022B02D0012004B0BF
:10F2C00010BD83683122DB074CBFF4217421FEF7A7
:10F2D00023FC012004B010BD82680DF10F0490F9E9
:10F2E00010C002F00102417C60464FF0310C0192E7
:10F2F000F42200948DF80FC0F4F76AFB012004B0EB
:10F3000010BD00BF00680379012B07D0022B01D08C
:10F310000020704701225821FEF7FEBB8268417C25
:10F3200002F0010210B590F9104084B020460DF1B2
:10F330000F040192582200948DF80F30F4F748FB27
:10F3400004B010BD00680379012B07D0022B01D057
:10F350000020704701224821FEF7DEBB8268417C15
:10F3600002F0010210B590F9104084B020460DF172
:10F370000F040192482200948DF80F30F4F728FB17
:10F3800004B010BD00680379012B07D0022B01D017
:10F39000002070471A460821FEF7BEBB826890F92C
:10F3A00010C002F00102417C60464FF0020C10B523
:10F3B00084B00DF10F04019208228DF80FC0009463
:10F3C000F4F706FB04B010BD00680379012B07D0E9
:10F3D000022B01D00020704701220821FEF79CBBC0
:10F3E0008268417C02F0010210B590F9104084B0AF
:10F3F00020460DF10F040192082200948DF80F3081
:10F40000F4F7E6FA04B010BD10B50446006884B005
:10F410000379012B12D0022B02D0002004B010BDC2
:10F4200001220B21FEF778FB0028F6D01D220921CE
:10F43000206804B0BDE81040FEF7CCBB826890F9AC
:10F4400010C002F00102417C60468DF80F3001923D
:10F450000DF10F0200920B22F4F7BAFAE4E700BFB5
:10F460002DE9F04105461F462848164695F910300B
:10F4700082B003EB430350F83380AB689A0716D58C
:10F4800001230DF106028DF8061040460DF107012B
:10F49000F4F7B0FF3B46324600214046F4F7AAFF9E
:10F4A000AB689B0718D5012002B0BDE8F0816B69FD
:10F4B0001BB19A88186812048261154B1868154BA5
:10F4C000C000A3FB0030144B80095A685C68A4EBB1
:10F4D000020C6045FAD2D3E70D4A4FF4FA700D4B97
:10F4E00012680D4900FB02F24868A3FB0232920940
:10F4F0004B681B1A9A42FBD26B69002BD3D01A6857
:10F5000001209B88936102B0BDE8F081C402002411
:10F51000486F0024D34D6210001000E030B505792B
:10F5200083B084468E46012D0DD0022D02D00020DE
:10F5300003B030BD8468E40758BF41F0800103B0D8
:10F54000BDE830408CE7806814460A46009400F01D
:10F5500001049CF811109CF910000194F4F738FA9A
:10F5600003B030BDF0B5002383B0142607468DF8F4
:10F57000023005F0D3FC04460D4605F0CFFC001B1D
:10F5800061EB0501B0F57A7F71F10001F5D3013E21
:10F59000EFD131460DF102023868FEF7B5F90DF1F1
:10F5A000020280213868FEF7AFF94FF4F8428DF877
:10F5B00006601426ADF80420032301AA60213868F0
:10F5C000FFF7ACFF05F0AAFC04460D4605F0A6FCCB
:10F5D000001B61EB0501B0F57A7F71F10001F5D3F5
:10F5E000013EEFD131460DF1030238688DF803601A
:10F5F000FEF78AF94CF26243142601AA6021ADF8A5
:10F600000430042338688DF806300323FFF786FFA3
:10F6100005F084FC04460D4605F080FC001B61EB00
:10F620000501B0F57A7F71F10001F5D3013EEFD10C
:10F6300031460DF1030238688DF80360FEF764F976
:10F640004FF4E853142601AA6021ADF804300823D2
:10F6500038688DF806300323FFF760FF05F05EFC85
:10F6600004460D4605F05AFC001B61EB0501B0F5A0
:10F670007A7F71F10001F5D3013EEFD10DF1030264
:10F68000314638688DF80360FEF73EF90DF102024D
:10F690001E213868FEF738F9012003B0F0BD00BF25
:10F6A0002DE9F04105461F462848164695F91030C9
:10F6B00082B003EB430350F83380AB689A0716D54A
:10F6C00001230DF106028DF8061040460DF10701E9
:10F6D000F4F790FE3B46002231464046F4F78AFE9E
:10F6E000AB689B0718D5012002B0BDE8F0816B69BB
:10F6F0001BB19A88186812048261154B1868154B63
:10F70000C000A3FB0030144B80095A685C68A4EB6E
:10F71000020C6045FAD2D3E70D4A4FF4FA700D4B54
:10F7200012680D4900FB02F24868A3FB02329209FD
:10F730004B681B1A9A42FBD26B69002BD3D01A6814
:10F7400001209B88936102B0BDE8F081C4020024CF
:10F75000486F0024D34D6210001000E030B50579E9
:10F7600083B084468E46012D0DD0022D02D000209C
:10F7700003B030BD8468E40758BF41F0800103B096
:10F78000BDE830408CE7806814460A46009400F0DB
:10F7900001049CF811109CF910000194F4F734FB5B
:10F7A00003B030BD2DE9F043816B85B0804C06235A
:10F7B000076880467F4A962690F83500B4FBF1F141
:10F7C00089B2FDF77DFC4388002181463846B4FBB1
:10F7D000F3F4C8F84040FEF755F980226B21384613
:10F7E000FEF7F8F905F09AFB04460D4605F096FB86
:10F7F000001B61EB0501B0F57A7F71F10001F5D3D3
:10F80000013EEFD19626032268213846FEF7E2F941
:10F8100005F084FB04460D4605F080FB001B61EB00
:10F820000501B0F57A7F71F10001F5D3013EEFD10A
:10F8300003226B213846FEF7CDF905F06FFB044635
:10F840000D4605F06BFB001B61EB05010F2871F104
:10F850000001F6D310226A213846FEF7BBF905F005
:10F860005DFB04460D4605F059FB001B61EB0501ED
:10F870000F2871F10001F6D300226C213846FEF703
:10F88000A9F905F04BFB04460D4605F047FB001BAC
:10F8900061EB05010F2871F10001F6D399F80520FD
:10F8A00019213846FEF796F905F038FB04460D4657
:10F8B00005F034FB001B61EB05010F2871F100011D
:10F8C000F6D318221B213846FEF784F905F026FBF3
:10F8D00004460D4605F022FB001B61EB05010F28D5
:10F8E00071F10001F6D318221C213846FEF772F997
:10F8F00005F014FB04460D4605F010FB001B61EB00
:10F9000005010F2871F10001F6D399F804201A219E
:10F910003846FEF75FF905F001FB05460C4605F099
:10F92000FDFA8C4208BF8542F9D003213846FEF724
:10F93000A9F8062302AA4321D8F80000FFF70EFF1A
:10F9400028B3BDF80810BDF80A30BDF80C20C9BABC
:10F95000DBBA07EE901AD2BAF8EEE76A07EE102A81
:10F9600007EE903AB8EEC77AF8EEE77AC8ED076A84
:10F9700088ED097AC8ED087AFDEEE77ACDED017AD7
:10F980009DF90430013305D005B0BDE8F083D8ED12
:10F99000087AF1E7D8ED077AFDEEE77ACDED017A46
:10F9A0009DF904300133EFD1062005F013FB00BFB1
:10F9B00040420F00CCA50C0810B582B008210446C7
:10F9C00000686A46FDF7A0FF9DF80030DB0602D410
:10F9D000002002B010BD06236A4600212068FFF710
:10F9E000BDFE0028F4D09DF801209DF80010120201
:10F9F0009DF80230DFED496A02EB01429DF80410E8
:10FA000014024FEA01219DF8034013449DF805209C
:10FA100001EB044148BF03F17F430A44090207EEAA
:10FA2000903A3F4B48BF02F17F42F8EEE77A93ED00
:10FA3000196A07EE102AB3F96820F8EEC65AB3F92E
:10FA40006E10B8EEC77A93F80C4204EE901AB3F930
:10FA50007210112CC7EE263A87EEA67A06EE902A8F
:10FA6000B3F96A20D3ED187A06EE102AB3F96C20A8
:10FA700005EE102AB3F97020F8EEE66A04EE102ABB
:10FA8000F8EEE77AB8EEC66AB3F97420B8EEC55A54
:10FA9000F8EEE44AB8EEC44A66EEA36A27EE232ADB
:10FAA00023D0A7EE045AA7EE246AE5EE075AE5EE46
:10FAB000877A77EEA67AE6EE027AB3F95E20F6EE62
:10FAC000006AC3ED1E7A07EE902AB3F95C10F8EED7
:10FAD000E77A07EE101AB8EEC77A67EEA37AE7EE78
:10FAE000267AC3ED1F7A02B010BD03EE102AF8EE9D
:10FAF000C32A03EE101AB8EEC33AA7EE224AE7EE85
:10FB0000034AA4EE075AA4EE876AE5EE075AE5EE2B
:10FB1000877A77EEA67AE6EE027ACEE7000078489A
:10FB200020D80024F0B5142683B000220A2107460D
:10FB30000068FEF74FF805F0F1F904460D4605F0B0
:10FB4000EDF9001B61EB0501B0F57A7F71F1000161
:10FB5000F5D3013EEFD10A260F220A213868FEF7BD
:10FB600039F805F0DBF904460D4605F0D7F9001B1E
:10FB700061EB0501B0F57A7F71F10001F5D3013E2B
:10FB8000EFD10A26032301AA10213868FFF7E6FD0A
:10FB900005F0C4F904460D4605F0C0F9001B61EB01
:10FBA0000501B0F57A7F71F10001F5D3013EEFD187
:10FBB0009DF804209DF805009DF806108032194B31
:10FBC00080308031A3F8102232460A26A3F81202B0
:10FBD000A3F814120A213868FDF7FCFF05F09EF91E
:10FBE00004460D4605F09AF9001B61EB0501B0F5DE
:10FBF0007A7F71F10001F5D3013EEFD10DF10302DF
:10FC000002213868FDF780FE0DF1030209213868F2
:10FC1000FDF77AFE11220A213868FDF7DBFF01208B
:10FC200003B0F0BD20D80024026830B5137985B048
:10FC30000446012B61D0022B03D00025284605B0D5
:10FC400030BD916802AD1046C9072A464CBF19461F
:10FC50008221FDF7E1FB0028EFD09DF80830DA079C
:10FC6000EBD52A46072303212068FFF777FD0546D9
:10FC70000028E2D011220A212068FDF7ABFF9DF891
:10FC80000E301B07D9D42A49BDF80830B1F810222C
:10FC900013FB02F3274A93423EDBB3F5000F39DA38
:10FCA000002BB8BFFF331B125B421BB2BDF80A200A
:10FCB000E386B1F8123212FB03F31E4A93422FDBA4
:10FCC000B3F5000F30DA002BB8BFFF3343F30F2238
:10FCD000BDF80C30B1F81412228713FB01F3154A5A
:10FCE00093421BDBB3F5000F1CDA002BB8BFFF33C8
:10FCF0001B125B421BB26387A0E7517C02AD92F9F5
:10FD000010009268009502F0010201920222F4F7BD
:10FD10007BF8A0E7084BC9E7084BC7E7074BEAE7C2
:10FD2000064AD5E7044BE6E747F6FF72D0E700BF87
:10FD300020D8002401FF7FFF0180FFFF0080FFFF2C
:10FD4000F0B5142683B000220A2107460068FDF7AB
:10FD500041FF05F0E3F804460D4605F0DFF8001B0F
:10FD600061EB0501B0F57A7F71F10001F5D3013E39
:10FD7000EFD10A260F220A213868FDF72BFF05F084
:10FD8000CDF804460D4605F0C9F8001B61EB0501EE
:10FD9000B0F57A7F71F10001F5D3013EEFD10A266B
:10FDA000032301AA10213868FFF7D8FC05F0B6F844
:10FDB00004460D4605F0B2F8001B61EB0501B0F5F5
:10FDC0007A7F71F10001F5D3013EEFD132460A2668
:10FDD0000A213868FDF7FEFE05F0A0F804460D463E
:10FDE00005F09CF8001B61EB0501B0F57A7F71F11D
:10FDF0000001F5D3013EEFD10DF103020221386875
:10FE0000FDF782FD0DF1030209213868FDF77CFD45
:10FE100001220A213868FDF7DDFE012003B0F0BDA4
:10FE200030B5002385B004460221C0F836300DF10C
:10FE3000070243870068FDF767FD18B19DF807309A
:10FE4000DB0703D40025284605B030BD062302AAEF
:10FE500003212068FFF782FC0DF1070209212068C9
:10FE6000FDF752FD05460028ECD09DF8073013F051
:10FE70000C0FE7D1BDF80820BDF80C30BDF80A1012
:10FE8000C2EB8232C3EB8333206889009B0092006F
:10FE9000218763870A21E2860122FDF79BFE28461F
:10FEA00005B030BD10B50446006882B003796A46DB
:10FEB000022B4FF006030CBF43210321FFF74EFC3A
:10FEC00068B1BDF80010BDF80220BDF8043049BA91
:10FED00052BA5BBAE1866287238702B010BDC4F8CC
:10FEE0003600608702B010BD10B5002386B004460E
:10FEF00000688DF80F300379012B31D0022B02D02E
:10FF0000002006B010BD83680DF10F02D9074CBF69
:10FF10002721A721FDF780FA0028F1D09DF80F30A6
:10FF20001B07EDD5062304AA28212068FFF716FC3D
:10FF300028B3BDF91030002BB8BF03339A10BDF9B8
:10FF40001230002BE286B8BF03339A10BDF914308B
:10FF5000002B2287B8BF03339B10638706B010BD08
:10FF60008268417C02F0010290F910C001920DF10B
:10FF70000F02604600922722F3F746FFCCE7C4F851
:10FF8000360060870020BCE730B54FF0000C044617
:10FF9000006887B0C4F836C0A4F83AC00379012BD2
:10FFA0002AD0022B02D0002007B030BD83680DF1AB
:10FFB0000F02D9074CBF61468021FDF72DFA0028BA
:10FFC000F1D09DF80F301B07EDD5062304AA0121BF
:10FFD0002068FFF7C3FB0028E5D0BDF81430BDF85A
:10FFE0001010BDF812205BBA49BA52BA5B42E186E2
:10FFF0002287638707B030BD85686246417C05F083
:020000040805ED
:10000000010590F9100001950DF10F050095F3F72A
:10001000FBFED4E72DE9F047164F81468A4697F854
:1000200019326BB90024D9F8000097F81A325246F9
:10003000492187F81942FFF791FB0120BDE8F087BD
:1000400004F06CFFD7F82032C51AC5F5FA55002D1B
:10005000E8DD04F063FF04464FEAE5780E4604F05D
:100060005DFF001B61EB0601A84271EB0801F6D3AE
:10007000D8E700BF20D800242DE9F041624C0546A6
:1000800082B0D4F82802C5F8360094F81832B4F8D3
:100090002C22012B6A8777D0022B0FD0002B69D13D
:1000A00001220221284667F0E5F8012394F82E6228
:1000B00084F81832304602B0BDE8F08194F8193265
:1000C00004F50A7705F13608002B6FD169462846FA
:1000D000FFF7A0FF9DF80630064600284AD01B0710
:1000E00048D4B4F8FC21BDF8003013FB02F3474AB2
:1000F00093427EDBB3F5000F70DA002BB8BFFF33FD
:100100001B125B421BB2B4F8FE21EB86BDF8023035
:1001100013FB02F33D4A93426FDBB3F5000F70DA35
:10012000002BB8BFFF3343F30F23B4F800222B8713
:10013000BDF8043013FB02F3344A93425BDBB3F5A2
:10014000000F5CDA002BB8BFFF331B125B421BB2FF
:10015000D5F836006B870023C4F828023046B8F87B
:10016000042084F818320123BA8084F82E3202B0B9
:10017000BDE8F08100231E4684F8183284F82E3240
:10018000304602B0BDE8F08194F8193294F82E623E
:10019000D3B969462846FFF73DFF9DF8003008B106
:1001A0009A071DD1002384F8183283E704F0B6FEC5
:1001B000D4F82032C01AB0F5FA5F87DA94F82E62CC
:1001C000304602B0BDE8F08104F0A8FED4F8203239
:1001D000C01AB0F5FA5FFFF66DAFDAE70C4B92E7A5
:1001E00007220321284667F045F8022384F81832D5
:1001F00060E7084B87E7074BAAE7064B95E7044BF8
:10020000A6E747F6FF7390E720D8002401FF7FFFA1
:100210000180FFFF0080FFFF10B500230446006847
:1002200086B0C4F8363063870379012B23D0022BC4
:1002300002D0002006B010BD83680DF10F02D9076F
:100240004CBF06218621FDF7E7F80028F1D09DF884
:100250000F30DB07EDD5062304AA00212068FFF745
:100260007DFA0028E5D0049ABDF81430C4F8362091
:10027000638706B010BD8268417C02F0010290F9EC
:1002800010C001920DF10F02604600920622F3F7B2
:10029000BBFDDAE710B500230446006886B0C4F859
:1002A000363063870379012B29D0022B02D000203E
:1002B00006B010BD83680DF10F02D9074CBF0921AC
:1002C0008921FDF7A9F80028F1D09DF80F30DB0750
:1002D000EDD5062304AA01212068FFF73FFA002884
:1002E000E5D0BDF81210BDF81020BDF81430494219
:1002F00052425B42E1862287638706B010BD826866
:10030000417C02F0010290F910C001920DF10F0240
:10031000604600920922F3F777FDD4E710B5002379
:100320000446006886B0C4F8363063870379012B31
:1003300012D0022B0DD183680DF10B02DB074CBFED
:100340003421B421FDF768F818B19DF90B30002B6A
:1003500011DB002006B010BD8268417C02F0010272
:1003600090F910C001920DF10B0260460092342208
:10037000F3F74AFDE8E7092303AA24212068FFF7E1
:10038000EDF90028E5D09DF810209DF80F109DF89C
:10039000133012041B0442EA01629DF8121043EA72
:1003A00001639DF80C10C2F30F42C3F30F43228781
:1003B00063879DF80D301B0443EA0163C3F30F43C9
:1003C000E38606B010BD00BF70B5066882B0044673
:1003D000F569002D5CD0002204233046FF212A70ED
:1003E0000DEB0302FFF7BAF910B9002002B070BD9F
:1003F00004236A46FF212068FFF7B0F90028F4D0F3
:100400009DF804309B09023B012BEED9BDF8043066
:1004100043F6FF7CBDF806205BBABDF80010BDF8BE
:100420000240C3F30D066645DFD0002EDDD053BA7F
:1004300040F2FF7EC3F34A1272451346D5D0002A1C
:10044000D3D049BAC1F30D0262451146CDD0002A7E
:10045000CBD064BAC4F34A1272451446C5D0002A00
:10046000C3D0721A002AB8BF5242FF2ABDDC1A1B41
:10047000002AB8BF5242FF2AB7DC23440E445B1067
:100480007610C5F801300123C5F805602B70ADE783
:1004900009211420FBF78EF8F061054626689AE7DB
:1004A00070B5066882B0F469F4B1002104233046C7
:1004B00021700DEB0302FF21FFF750F910B39DF8F7
:1004C00004309B0919D1BDF804200121BDF8063084
:1004D00052BA21705BBA92B2C3F34A13C4F8052032
:1004E000C4F8013002B070BD054609211420FBF7A5
:1004F00061F8F06104462E68D7E7044A042103201E
:10050000FAF7D2FF002002B070BD00BF384D0D08D1
:1005100070B5066882B00546F469002C3ED0337988
:10052000221D012B2DD0022B26D1B368304613F0AB
:10053000010F4FF00C030CBF8C211946FFF7B0F8E8
:10054000A070D8B1B4F9043007EE903AF8EEE77A2B
:10055000C5ED077AB4F9063007EE903AF8EEE77A7F
:10056000C5ED087AB4F9083007EE903AF8EEE77A6C
:10057000C5ED097A02B070BD0023A370002002B05F
:1005800070BDB368717C03F0010396F9100000920E
:1005900001930C231A46F3F737FCD1E70921142005
:1005A000FBF708F8F06104462E68B8E770B50668F6
:1005B00082B00546F469002C3ED03379E21C012B51
:1005C0002DD0022B26D1B368304613F0010F4FF027
:1005D0000D0314BF0C218C21FFF762F8A070D8B175
:1005E000B4F90A3007EE903AF8EEE77AC5ED077AEB
:1005F000B4F90C3007EE903AF8EEE77AC5ED087AD8
:10060000B4F90E3007EE903AF8EEE77AC5ED097AC4
:1006100002B070BD0023A370002002B070BDB368AB
:10062000717C03F0010396F9100000920C220193F3
:100630000D23F3F7E9FBD1E709211420FAF7BAFFFC
:10064000F06104462E68B8E7006810B5037984B0FD
:100650000C46012B1AD0022B02D0002004B010BD92
:10066000836803AA13F0010F4FF0030314BF222184
:10067000A221FFF715F80028EFD0BDF90D3003EBEC
:1006800083031B12E633238004B010BD836803AAE2
:10069000417C03F0010390F91000009222220193A3
:1006A0000323F3F7B1FBE6E770B5066882B00546B1
:1006B000F469002C3ED03379221D012B2DD0022B62
:1006C00026D1B368304613F0010F4FF00E0314BF6C
:1006D0003B21BB21FEF7E4FFA070D8B1A389DBBAB0
:1006E00007EE903AF8EEE77AC5ED077AE389DBBAD0
:1006F00007EE903AF8EEE77AC5ED087A238ADBBA7E
:1007000007EE903AF8EEE77AC5ED097A02B070BDCF
:100710000023A370002002B070BDB368717C03F0A9
:10072000010396F9100000923B2201930E23F3F788
:100730006BFBD1E709211420FAF73CFF0446F06176
:10074000B9E700BF006810B5037984B0012B10D061
:10075000022B01D000200AE003AAF621FEF7A0FF39
:100760000028F7D0BDF80C30094A5BBA138204B0F8
:1007700010BD826803AC417C022302F0010290F9B3
:100780001000CDE90042F622F3F73EFBE8E700BF98
:1007900020D80024006810B5037984B0012B1DD047
:1007A000022B01D0002017E0032303AAF621FEF755
:1007B00077FF0028F6D09DF80D309DF80CC01B0285
:1007C0000D499DF80E2043EA0C431343B1F9302044
:1007D000C2F10802D3404B6304B010BD826803AC81
:1007E000417C032302F0010290F91000CDE90042A0
:1007F000F622F3F709FBDCE720D80024006810B5E7
:10080000037984B0012B2DD0022B07D01C49002086
:10081000D1E98C328A638B6504B010BD062302AA2D
:10082000F721FEF73DFF0028F0D09DF809309DF834
:100830000C209DF808C01B019DF80BE012019DF8EB
:100840000A1043EA0C3342EA0E329DF80DC043EA27
:1008500011130B4942EA1C128B658A63C1E98C3281
:1008600004B010BD826802AC417C062302F0010294
:1008700090F91000CDE90042F722F3F7C5FAD2E76C
:1008800020D80024006810B5037984B0012B1DD056
:10089000022B0FD09DF80D3001209DF80CC01B02DB
:1008A0009DF80E10104A43EA0C430B43C2F8803007
:1008B00004B010BD836803AA13F0010F4FF00303C7
:1008C00014BF00218021FEF7EBFEE3E7826803AC52
:1008D000417C032302F0010290F91000CDE90042AF
:1008E0000022F3F791FAD5E720D80024006810B56C
:1008F000037984B0012B1DD0022B0FD09DF80D3051
:1009000001209DF80CC01B029DF80E10104A43EA0E
:100910000C430B43C2F8943004B010BD836803AAA3
:1009200013F0010F4FF0030314BF00218021FEF7E5
:10093000B7FEE3E7826803AC417C032302F00102C7
:1009400090F91000CDE900420022F3F75DFAD5E7F7
:1009500020D80024006810B5037984B0012B28D07A
:10096000022B01D0002022E0836803AA13F0010FBC
:100970004FF003030CBF83211946FEF791FE0028B8
:10098000F0D09DF80C309DF90C109DF80D201B0443
:1009900000299DF80EC043EA02230D4AACBF002196
:1009A0004FF07F4143EA0C030B43C2F8743104B0AB
:1009B00010BD826803AC0323417C02F0010290F970
:1009C0001000CDE900421A46F3F71EFAD7E700BF40
:1009D00020D80024006810B5037984B0012B28D0FA
:1009E000022B01D0002022E0836803AA13F0010F3C
:1009F0004FF0030314BF00218021FEF751FE0028B1
:100A0000F0D09DF80C309DF90C109DF80D201B04C2
:100A100000299DF80EC043EA02230D4AACBF002115
:100A20004FF07F4143EA0C030B43C2F8703104B02E
:100A300010BD826803AC417C032302F0010290F9EF
:100A40001000CDE900420022F3F7DEF9D7E700BF3E
:100A500020D8002410B50446006884B00379012B27
:100A600043D0022B07D0002213461046C4F836208C
:100A7000638704B010BD836802AA13F0010F4FF022
:100A8000060314BF11219121FEF70AFE0028EAD0C7
:100A9000BDF90C20B7EE086ABDF90A3007EE902ABE
:100AA000BDF908205B4206EE902AF8EEE77A07EEE1
:100AB000103AF8EEE66AB8EEC77A67EE867A66EE26
:100AC000866A27EE067AFDEEE77AFDEEE66ABDEE6F
:100AD000C77A17EE903A16EE902A1BB2E28617EE0E
:100AE000102A6387228704B010BD836802AA417C64
:100AF00003F0010390F910000092112201930623E4
:100B0000F3F782F9C2E700BF10B50023044600687E
:100B100084B0C4F8363063870379012B22D0022BCE
:100B200001D000201CE0836802AA13F0010F4FF0EF
:100B3000060314BF03218321FEF7B2FD0028F0D085
:100B4000BDF90A30BDF80810BDF80C205B4201EB7E
:100B5000410102EB420203EB4303E18662872387F4
:100B600004B010BD836802AA417C03F0010390F930
:100B700010000092032201930623F3F745F9DDE705
:100B800010B54FF0000C0446006884B0C4F836C0BD
:100B9000A4F83AC00379012B18D0022B01D0002011
:100BA00012E0836802AA13F0010F4FF0060314BF8E
:100BB00061468021FEF774FD0028F0D0029ABDF84E
:100BC0000C30C4F83620638704B010BD83686246D9
:100BD000417C03F0010390F910E0019302AB7046F1
:100BE00000930623F3F710F9E6E700BF10B50023E2
:100BF00084B0044600680293CDF80B300279012AD4
:100C00001ED0022A19D1836802AA13F0010F4FF0F7
:100C1000070314BF4E21CE21FEF742FDBDF8091097
:100C2000BDF80B20BDF80D30C9BAD2BADBBA01202D
:100C3000E1862287638704B010BD1A461946F6E79D
:100C4000826802AB90F910C002F00102417C00936F
:100C50006046019207234E22F3F7D6F8DEE700BF85
:100C6000006810B5037984B0012B0BD0022B06D19C
:100C7000012303AAFF21FEF713FD04B010BD0020DD
:100C800004B010BD826803AC417C02F0010290F90F
:100C9000100000940192FF22F3F7B6F804B010BDE3
:100CA0000368DA6B10B5044682B012B1904740B1C8
:100CB00023685B6B1BB1214601A8984718B9FF2335
:100CC000E38202B010BDBDF80630013B9BB2F7E7EE
:100CD000F0B50D4683B00446184616461F466FF021
:100CE0007FFB2844E6732946A0732046256800242C
:100CF0003B46324600946C69A04703B0F0BD00BF8C
:100D000038B58B68044601600D46984700230B4AAE
:100D1000237522612B6B13B1204698472075084B31
:100D200093F838321BB1237D23F001032375002390
:100D30002046E382BDE83840B2E700BF0001FF0073
:100D400020D80024144B30B51C6885B084B12379B9
:100D5000012B10D0022B0BD1A1680246204611F0C6
:100D6000010118BF802105B0BDE83040FCF7D4BEBA
:100D7000002005B030BDA2680DF10F05617C8DF833
:100D80000F0094F9100002F00104802200950194F4
:100D9000F2F71EFE05B030BD80760024F0B5274D79
:100DA00085B02868002846D0B0228021FCF712FFC9
:100DB000286800283FD040228021FCF70BFF2868DC
:100DC000002838D000228021FCF704FF286890B367
:100DD00010228021FCF7FEFE28684FF48064002773
:100DE0000DF10F0670B10379012B10D0022B09D140
:100DF00083680022402113F0010304BF1A464021FA
:100E0000FCF78AFE013CA4B29CB12868EAE782683C
:100E1000013C90F910E002F0010CA4B2417C4022A8
:100E200070468DF80F70CDE9006CF2F7D1FD002C03
:100E3000EBD105B0F0BD0020CFE700BF80760024E5
:100E400010B50C4C2368A3B1A0F1500280211846C4
:100E5000D2B2FCF7BFFE206858B100228021FCF717
:100E6000B9FE206828B110228021BDE81040FCF7AF
:100E7000B1BE10BD80760024A0F12003F0B503EBD5
:100E800083031C4D1C4E85B0EC18053530681D449D
:100E900098B10379012B227816D0022B09D00134A6
:100EA000AC42F7D10022402105B0BDE8F040FCF78C
:100EB00091BE4021FCF730FE30680134AC42E7D1EE
:100EC0000028EFD105B0F0BD8168013490F910C061
:100ED00001F00107417C8DF80F20604601970DF16C
:100EE0000F0740220097F2F773FDAC423068CFD174
:100EF000E6E700BFF0A50C0880760024F0B59B4D16
:100F000085B02868002800F02E81D4228021FCF7CB
:100F100061FE2868002800F0268180221146FCF737
:100F200059FE2868002800F01E81A8228021FCF7C5
:100F300051FE2868002800F016813F228021FCF72E
:100F400049FE2868002800F00E81D3228021FCF79A
:100F500041FE2868002800F0068100228021FCF76D
:100F600039FE2868002800F0FE8040228021FCF72E
:100F700031FE2868002800F0F6808D228021FCF7E1
:100F800029FE2868002800F0EE8014228021FCF75A
:100F900021FE2868002800F0E680A1228021FCF7CD
:100FA00019FE2868002800F0DE80C8228021FCF7A6
:100FB00011FE2868002800F0D680DA228021FCF794
:100FC00009FE2868002800F0CE8012228021FCF75C
:100FD00001FE2868002800F0C68081228021FCF7ED
:100FE000F9FD2868002800F0BE80CF228021FCF7A0
:100FF000F1FD2868002800F0B680D9228021FCF796
:10100000E9FD2868002800F0AE80F1228021FCF77D
:10101000E1FD2868002800F0A680DB228021FCF793
:10102000D9FD2868002800F09E8040228021FCF72E
:10103000D1FD2868002800F09680A4228021FCF7CA
:10104000C9FD2868002800F08E80A6228021FCF7C8
:10105000C1FD2868002800F08680AF228021FCF7BF
:10106000B9FD286800287ED0A6228021FCF7B2FDB9
:101070002868002877D0AE228021FCF7ABFD2868D5
:10108000002870D020228021FCF7A4FD28680028C9
:1010900069D000228021FCF79DFD2868002862D0DD
:1010A000B0228021FCF796FD286800285BD0402202
:1010B0008021FCF78FFD2868002854D00022802171
:1010C000FCF788FD286800284DD010228021FCF70D
:1010D00081FD28684FF4806400270DF10F0628B3C6
:1010E0000379012B2BD0022B04F1FF3215D094B2DF
:1010F000002CF6D181228021FCF76CFD286848B1D4
:10110000C8228021FCF766FD286818B1AF22802133
:10111000FCF760FD012005B0F0BD8268402112F0AF
:10112000010218BF0022FCF7F7FC2868013CA4B2BA
:10113000002CD4D10028DDD1012005B0F0BD82689B
:10114000013C90F910E002F0010CA4B2417C402275
:1011500070468DF80F70CDE9006CF2F739FC286805
:10116000002CBCD1E6E70020B4E700BF8076002465
:10117000FCF72CBAFCF72ABAFCF728BAFCF726BA17
:10118000FCF724BAFCF722BAFCF720BA012070471A
:10119000034620B1026812B1D26902B1104793ED43
:1011A000017AF6EE007A074BB8EEC77AD3ED016A02
:1011B000E7EE267AFDEEE77A17EE900A00F30B00D1
:1011C000704700BFC4A90024034620B1026812B1D1
:1011D000126A02B1104793ED027AF6EE007A074BDD
:1011E000B8EEC77AD3ED026AE7EE267AFDEEE77A2B
:1011F00017EE900A00F30B00704700BFC4A900244B
:10120000034628B102681AB1516A09B193691847B7
:1012100093ED037AF6EE007A064BB8EEC77AD3ED7B
:10122000036AE7EE267AFDEEE77A17EE900A00F3FE
:101230000B007047C4A9002410B5044630B1036800
:1012400023B1DB6813B1BDE81040184703F066FE18
:10125000D4E904239042994134BF0120002010BDFD
:10126000D8B10E4B0E4A70B506680D4682B00446E2
:1012700033449B0A32F8130064F088FCC5F3810301
:101280000022A1883046CDE90032C5F3411305F0B4
:1012900013026EF06BFE02B070BD70470000FEA737
:1012A0003C9E0C08D0B10E4BF0B5076816460D4AAF
:1012B0000D463B4483B004469B0A32F8130064F0A9
:1012C00065FCC5F38103A188384605F01302CDE91A
:1012D00000366B096EF04AFE03B0F0BD704700BFE8
:1012E0000000FEA73C9E0C0810B50409013C042C2C
:1012F00019D80F4A00F00F0332F8140040FA03F235
:1013000012F0010211D0012202FA03F3013B18404E
:1013100078F0DCFA074B084A1B5D184400EB4000EC
:1013200002EB800010BD002010BD104610BD00BFB4
:10133000F09D0C0820A40C086C6000242DE9F04FEF
:101340005422044600218BB0A14877F0FBFAA14952
:10135000621EE01C0E460C4612F8013F5D1E052D74
:1013600088BF0023904244F8043BF5D19A4BA3F187
:10137000100252F8040B012800F01C819342F8D1AE
:10138000944A52F8040B022800F00B819342F8D1E2
:10139000904A52F8040B032800F0FA809342F8D1E7
:1013A00051F8042B042A00F0EA808B42F8D18B4FCD
:1013B00005204FF01A09DFF818824FF0000B07F2F2
:1013C0005C44874EFBF7FAF90620FBF7F7F998F82B
:1013D0000CA0BAF1000F31D0504698F90D50FFF72C
:1013E00083FF28B1052380F80790837100230372DF
:1013F0000321FFF735FF002302E001331C2B3ED011
:1014000014F833205245F8D107EBC303D3F8602416
:10141000F423C8F810200122062103FB05650BF117
:10142000010B88F81610D5F8F43088F8152088F8E4
:101430001430134485F8F020C5F8F43009F101099F
:1014400008F10C085FFA89F9B9F1200FBFD1BBF19F
:10145000000F11D0DFF89CA14FF0000BDFF898913E
:101460009AF8EC306BB90BF1010B0AF1F40A09F5AB
:101470008C79BBF1030FF3D10BB0BDE8F08F0022E4
:10148000C6E7BAF806004FF4403764F07FFBBAF8BD
:10149000040064F07BFBDAF8F030514CF421012BAE
:1014A000CAF82830DAF8002001FB0B41D4BF002332
:1014B00001234FF0030CCAF81020CAF81C30002397
:1014C000CAF838308AF82C30CAF83030CAF82030E0
:1014D0008AF8483004930823CAE905734FF48063FF
:1014E000CAF834304FF48073AAF824304FF4805394
:1014F000CAE90FC38B6E002B65D093689E0003D59D
:101500009168384B0B4093609368DD0014D4364BE0
:1015100036491B689068B3FBF1F33549013301404C
:1015200041F0805191600493049B2BB1049B013BDB
:101530000493049B002BF9D19368D8001CD4F423A6
:101540004FF0010803FB0B43996E41F010019966BF
:10155000D96E41EA0801D966F423916803FB0B4375
:1015600001F00401986E00F01000014346D09A6E1D
:1015700042F010029A6676E74FF00008ECE796F822
:10158000F8313422013386F8D42186F8F8310EE799
:1015900096F8F8213520013286F8C80186F8F8213E
:1015A000FEE696F8F8213120013286F8BC0186F873
:1015B000F821EDE696F8F8213020013286F8B001E6
:1015C00086F8F821DCE6CB668AF8603095E700BF44
:1015D000C4D9002420D8002430D8002438A40C0812
:1015E0003C240024C0FFFF5F00000024400D0300E6
:1015F000C0FFFF6F40240024C0300030996E21F4FA
:10160000817141F0020199669368D90713D4784B30
:101610009A4200F0248303F580739A4200F01F83FE
:10162000744B9B68DF0706D473498B6823F47C13E3
:1016300043F440338B60714B71491B68D368194088
:1016400043F208030B43D3609168936801F00401EF
:1016500003F00803194300F06D82DAF81000DAF89D
:101660001C30012B00F06983036B23F00F0303632D
:10167000F42303FB0B439A6E22F0030242F00102B3
:101680009A66B8F1000F7FF4EEAE9AF86020CDF8BC
:101690001480012A3FF4E7AE8268012196078AF898
:1016A0006010816802D4CD0700F19482F421554A7C
:1016B000554B01FB0B418D6E2A4042F002028A66B7
:1016C0008268134043F00043836083684F4A002BD5
:1016D000C0F2F081F4214E4B4E4D4FF4005701FB08
:1016E0000B414D484FF0030C8A6E22F0030242F08A
:1016F00001028A66DAF80820DAF80C60AA4218BFFC
:101700009A424FF48065CAF878600CBF0123002329
:10171000CAF89CC0824208BF43F0010318308242DD
:1017200008BF43F001031830824208BF43F00103B1
:101730001830824208BF43F001031830824208BFCC
:1017400043F001031830824208BF43F0010300F563
:101750005670824208BF43F001031830824208BF2E
:1017600043F001031830824208BF43F001031830F0
:10177000824208BF43F001031830824208BF43F0A1
